:020000040800F2
:1000000000000420F58A000821310008253100088D
:10001000293100082D3100083131000800000000AE
:100020000000000000000000000000009D470108E3
:1000300035310008000000002948010889480108FE
:10004000458B0008458B0008458B0008458B000850
:10005000458B0008458B00083931000891310008B4
:10006000458B0008458B000841100008B51D0008AD
:10007000DD1D0008051E0008458B00082D1E000828
:10008000391E0008458B0008458B0008458B000889
:10009000458B0008458B0008458B0008013500089A
:1000A000458B0008458B0008458B0008458B0008F0
:1000B000458B0008458B0008458B0008011D000892
:1000C0000D1D0008191D0008251D0008311D000820
:1000D0003D1D0008458B0008491D0008458B0008A0
:1000E000A9310008458B0008458B0008F131000854
:1000F0000932000821320008458B0008611E000803
:1001000000000000458B0008458B0008458B000867
:100110000000000000000000458B0008458B00082F
:10012000891E0008951E0008C91E00083532000807
:10013000458B0008458B0008458B0008458B00085F
:10014000458B0008458B0008458B0008458B00084F
:10015000458B000841320008D51E0008651D0008C7
:10016000458B0008458B00080000000000000000DF
:10017000000000000000000000000000000000007F
:10018000458B0008458B00080000000000000000BF
:10019000458B0008458B00080000000000000000AF
:1001A000000000000000000000000000000000004F
:1001B000458B00080000000000000000458B00088F
:1001C000458B000810B5034B0360044614F086F815
:1001D000204610BDD895010810B5054B03600446B4
:1001E00014F07CF8204615F003FE204610BD00BF39
:1001F000D895010810B5064A064B0260044640F83F
:10020000783F14F06BF8204614F0AAF9204610BD90
:10021000F4950108D895010810B5064A064B02600E
:10022000044640F8783F14F059F8204614F098F945
:10023000204610BDF4950108D895010890F8BE3508
:1002400010B5044623B1D0F8B80508B115F0D2FDB9
:1002500094F8AE3523B1D4F8A80508B115F0CAFD5D
:1002600094F89E3523B1D4F8980508B115F0C2FD75
:1002700094F88A3423B1D4F8840408B115F0BAFD97
:10028000204610BD08B5274C2378BFF35B8FD907F4
:1002900012D5254C2378BFF35B8FDA072FD5234C7B
:1002A0002378BFF35B8FDB0717D5214B01221A7030
:1002B00015F0AEF904F060FB204600F0D5FC0028F4
:1002C000E7D01C4800F0B6FB1B4A1C49194800F057
:1002D000D7FC204600F0CEFCDBE7204600F0C4FC53
:1002E0000028E2D01349164800F0BCF9124A15491B
:1002F000134800F0C5FC204600F0BCFCD5E72046C2
:1003000000F0B2FC0028CAD00A490F4800F0A2F859
:10031000094A0E490C4800F0B3FC204600F0AAFC44
:10032000BDE700BF28020020200200202402002098
:100330008CD9012034040020A90C00083D020008DB
:10034000B0030020190200082C020020F50100086B
:1003500010B5084A084B0260044640F8783F13F095
:10036000BDFF204614F0FCF8204615F041FD204664
:1003700010BD00BFF4950108D895010810B5084AD2
:10038000084B0260044640F8783F13F0A7FF204670
:1003900014F0E6F8204615F02BFD204610BD00BFF6
:1003A000F4950108D895010808B5044600212046B7
:1003B00014F06EF978B9204614F078F906280ED1B9
:1003C000D4F88000032102F0C3FB0021204614F082
:1003D0005FF90028EFD0022003F094F9E6E704F07B
:1003E000CBFA00BF70B5054682B00E4609B3541A69
:1003F0000F2C01940BD8012C006822D10B780370CC
:10040000019C28686C600023035502B070BD002277
:1004100001A915F0FDFC019B2860AB602246314626
:1004200018F0BEF8019C28686C600023035502B0E8
:1004300070BD4AB90068144600236C60035502B0D1
:1004400070BD002CDED0E9E7014815F0DAFC00BFF2
:100450000096010870B5104A86B0044602AE6846A0
:100460000D46A2F10A010096FFF7BCFF032369467F
:100470004FF48062204614F0EFF80098B04201D0AB
:1004800015F0B6FC054B2360C4F88051204614F0EB
:100490002BF8204606B070BD36960108CC960108B0
:1004A0002DE9F041D0F88051284600F01FFB421E94
:1004B00018BF012206460321284602F07FFB324680
:1004C0000121284602F07AFB05F5987002F0FEFF44
:1004D0000FF0AAFA4E480EF0EBFB4E4808227821A6
:1004E0000FF0D8F84C481E2278210FF0D3F84B4873
:1004F0000EF0DEFB012E00F0818004200EF0BCFB2C
:100500004748502278210FF0C5F8002E14BF042070
:1005100000200EF0B1FB6E2278214248DFF8008106
:10052000404F0FF0B7F800200EF0A6FB3E48962291
:1005300078210FF0AFF801220021284602F03EFB9F
:100540000021284602F04AFC022804460ED0042866
:100550004FF0FA0033D0012C12D004F045FA0021FC
:10056000284602F03BFC02280446F0D1FA2004F0B1
:100570003BFA2846314600F0BDFA3046BDE8F0812E
:1005800000220321284602F019FB22462146284674
:1005900002F014FB00200EF06FFB50227821404641
:1005A0000FF078F804200EF067FB6E2278213846B1
:1005B0000FF070F8FA2004F017FA2646C0E701227F
:1005C0000321284602F0FAFA00220121284602F00F
:1005D000F5FA20460EF050FB5022782140460FF0ED
:1005E00059F800200EF048FB6E22782138460FF0B3
:1005F00051F8FA2004F0F8F90026A1E700200EF0E7
:100600003BFB0748502278210FF044F8042080E794
:1006100074E5010838960108509601085CD5010878
:1006200068960108809601089896010830B595B043
:100630000446FFF735FF032301930223054601A972
:10064000204602930623039314F03CF864212046CD
:1006500014F02EF8D4F88001294600F0CFFA15B036
:1006600030BD00BF70B5104A86B0044602AE684681
:100670000D46A2F10E010096FFF7B4FE0223694673
:100680004FF40072204613F0E7FF0098B04201D00B
:1006900015F0AEFB054B2360C4F88050204613F0E4
:1006A00023FF204606B070BDC2960108E0960108FF
:1006B00002484FF4DC310FF00DBE00BF00120020E5
:1006C0004FF0C043C0B21880704700BF4FF0C04326
:1006D0005880704741B100EB41014FF0C04230F803
:1006E000023B53808142FAD1704700BF41B100EB19
:1006F00041014FF0C042538820F8023B8142FAD1B9
:10070000704700BF30B50024A1B02146682206A87A
:100710000194029403940494059417F069FF23460E
:100720002246134913480FF0E3F8F022054611461C
:1007300020460DF05FF8F022114620460DF042F8F9
:10074000204603210EF0B0FB01A928460CF0D9FF8A
:10075000094A0A4B0A4C1194CDE90E23094A159215
:10076000094B0A4A06A928460CF0E9FF21B030BD22
:100770007CF30108C8F10108C1060008CD06000895
:10078000D5060008ED06000809D100086DCA00086A
:1007900030B589B01D4B1E48002400941A6B42F0FE
:1007A00008021A631A6B02F008020092009A019480
:1007B0001A6B42F040021A631A6B02F04002019277
:1007C000019A02941A6B42F020021A631B6B059483
:1007D00003F0200302934FF40063012503A9039360
:1007E000029B04950223069304F0CCFB03A9082383
:1007F00008480393049404F0C5FB202306480393A0
:1008000003A9049504F0BEFB09B030BD00380240D6
:10081000000C0240001802400014024008B5FFF727
:10082000B7FF1F480122202104F0D2FC00224FF420
:1008300000611C4804F0CCFC052004F0D5F801222E
:100840004FF40061174804F0C3FC0A2004F0CCF810
:1008500000224FF40061134804F0BAFC142004F0A5
:10086000C3F801224FF400610E4804F0B1FC0A20E5
:1008700004F0BAF80C4B5B689847852807D00B4BFF
:100880005B6898474FF6FF73984204D008BDBDE8F7
:10089000084002F01BB8BDE8084001F0B9BD00BF38
:1008A00000140240000C02403C0000200400002024
:1008B000012908B503D1FFF7B1FF002008BD4FF0B3
:1008C000FF3008BD00F2644580B5052307460122CC
:1008D0000221284600F01EFB07F27C48284600F063
:1008E00059FB0221404600F011FC134E07F5B56795
:1008F000284600F075FB284600F07AFB01223046BE
:100900004FF4806104F064FC0121284600F094FB60
:1009100040F30F21384600F00FFA002204464FF44E
:100920008061304604F054FC47F6FF73A2B2022106
:10093000404600F001FCDBE70000024080B5DFED3F
:10094000358A9FED35AADFED359ADFF8E490DFEDCB
:1009500034AA9FED349A84B00646B0EE68BA00F52A
:10096000B56800F2D457B7EE008A002468EE0A7A20
:10097000D6F84006FDEEE77A17EE903A19B208F085
:10098000A1FC28EE298A4046BDEEC88A18EE103A2E
:100990001BB21946039300F0CFF9C0EB0011090117
:1009A00089FB01320A44C917C1EBE231054609B29D
:1009B000D6F8440608F086FC2246CDE90045039BA4
:1009C0001949384617F00CFF01343946002003F06E
:1009D00079FFB4F5817F0AD178EE8B8A0024F4EE9A
:1009E000EA8AF1EE10FACCBFDFED0A8A00240EF09D
:1009F000A3FADFED0E7A28EE897A87EE270A07EE52
:100A0000904AF8EEE77A20EE270A15F041FBB0EEA7
:100A1000408AABE70000C8420000704200F87F4601
:100A200000007A44DB0FC940EC96010800007A45CB
:100A30002100048030B56021044687B001F064FADB
:100A4000002504F29443264AC4F884348121A4F892
:100A50008814C4F88C34C4F89034C4F8982541F64E
:100A6000FF73A4F89C15C4F8A02504F5B361C4F87D
:100A7000A42584F88A5404F2844284F89E5504F52F
:100A8000B56000F013F92846C4F83856C4F83C564F
:100A900003F024FE2946204600F024FC20460121D4
:100AA00000F03AFC2046012100F040FC0D4B00957F
:100AB0001A6B0D4842F001021A631B6B039503F099
:100AC000010300934FF48062009B019202230122F4
:100AD00001A90292049304F055FA204607B030BDF4
:100AE000C89701080038024000000240032102F0CC
:100AF00093B900BF0A46032102F084B9F0B5D0F8DB
:100B00003C5685B004460E462DB1284605B0BDE8DA
:100B1000F04009F0CCB809F0A3FB4FF4087303933D
:100B200002230193F0231A46009029460295284695
:100B300008F080FF2A46C4F83C066FF07F4108F0B9
:100B4000CDFF2C49D4F83C06012208F0C7FF032250
:100B50002949D4F83C0608F0C1FFD4F83C0601212D
:100B600008F0D9FF334604F24C624FF4F0714FF4B1
:100B70007F0008F06DFB334604F60C22C4F84006F3
:100B80004FF4F0714FF4004008F062FBD4F8407667
:100B9000C4F8440606463946D4F83C0608F05AFF25
:100BA00038463C2108F0A9FBD4F83C06314608F051
:100BB00051FF3046B42108F0A0FB14230122114656
:100BC000184608F039FAB7EE000AC4F8480608F0EB
:100BD00061FAD4F84816D4F83C0608F05DFFD4F862
:100BE0003C0600952B462A46142108F0ACFF05B0C0
:100BF000F0BD00BF808080004040400008B5054641
:100C00000C46C0F83816B1B90EF00EFF1149204657
:100C100003F058FE1049204603F054FE0F485022BE
:100C200078210EF037FD0E486E2278210EF032FD4D
:100C30002846FFF747FE4FF4F071FFF75FFF0949C1
:100C4000002003F03FFE0449002003F03BFE28464D
:100C5000FFF774FE049701082497010868970108BC
:100C600084970108A49701080078B0FA80F0400941
:100C7000704700BF01230370704700BF704700BF7B
:100C800000207047704700BFFEE70000044A054996
:100C90001368002B08BF0B461844106018467047B5
:100CA00000CA0120A818022000207047F8B50D46A0
:100CB0008979044616461F46C1B92B6803608360D4
:100CC000C360AB8881718380B3791BBBB288A37585
:100CD0003368A2822361A361E361AA882785930810
:100CE00002F00302236262622046F8BDA888400039
:100CF00015F082F8AB79AA882060A060E060A3714B
:100D0000A280002BE0D02968520017F049FCB3798B
:100D1000002BDBD0B088400015F06EF8B379B288B4
:100D20002061A061E061A375A282002BD5D031685B
:100D3000520017F035FCD0E7C3692DE9F04F9A1C3B
:100D4000C2611980D0F81080B0F814900C4608EBFE
:100D500049018A4283B0016A026808BFC0F81C805A
:100D60004FEA4909A9F102098246009102EBC10B41
:100D7000C14401920020002101E0B3F90040B2F922
:100D800002E0B2F90470023B984594BF1E464E46FD
:100D9000B2F9003036F902C9B04594BF35464D4628
:100DA000C3FB840135F90269A84594BF2B464B4625
:100DB000CEFB8C0133F90249B2F906500832C7FB69
:100DC0008601984588BF4B469345C5FB8401D4D125
:100DD000009ADAF82460CAF81830920096B11644E6
:100DE000019A02EB46061A463BF9025B32F90249C8
:100DF00090458CBF4B4613465E45C5FB8401F2D13E
:100E0000CAF81830BAF92820D31716F003FA00B23E
:100E100003B0BDE8F08F00BF10B5034B036004467C
:100E200013F0BAFA204610BDD498010810B5054B4E
:100E30000360044613F0B0FA204614F0D9FF2046B0
:100E400010BD00BFD49801082DE9F041044640F8D8
:100E50000C1B022788B0082200216060A76017F0F1
:100E6000C7FB00251B4B01951A6B25753A431A6386
:100E70001A6BDFF86C803A400192019A02951A6B66
:100E800042F004021A631B6B059503F0040301266C
:100E9000029303A94046029B03960496069504F02C
:100EA00071F80D4B049303A910230C480393069784
:100EB000059604F067F82A4609210A2003F0B8FDD8
:100EC00040463246314604F083F9204608B0BDE87A
:100ED000F08100BF003802400000211000080240ED
:100EE0000004024070B505460C4616462246002115
:100EF000286800F095F900222868114600F090F962
:100F000083B204B970BDB3424FF00A00FAD003F0C7
:100F10006BFDEBE7F8B51746002204460E46006865
:100F200011461D4600F07CF900221146206800F0B1
:100F300077F945F2065211462046FFF7D3FF43F6F4
:100F40004B020021206800F06BF976020022114666
:100F5000206806F47E4600F063F906F14D02002198
:100F6000206800F05DF900221146206800F058F971
:100F700005EB4712D2B212024E320021206800F077
:100F80004FF900222068114600F04AF90123237529
:100F9000F8BD00BF10B540F24F3204460021006892
:100FA00000F03EF900221146206800F039F94FF4B4
:100FB0004C5211462046FFF795FF45F20552114667
:100FC0002046FFF78FFF044813F00EFA034B4FF44F
:100FD00080621A6010BD00BF08CA012000E100E075
:100FE00002484FF0FF3113F0F1B900BF08CA0120E9
:100FF00010B588B00F49019105A9044603AA03233F
:1010000003910068029301A9049300F035F9039B52
:101010002068596801F006FF6268039B000A1060AF
:101020009968206801F0FEFE6368000A586008B005
:1010300010BD00BFDC980108436853F821007047D9
:1010400000B5102083B004F0D1F80A4801A913F0CC
:10105000D9F9019B012B09D14FF0E0234FF08052C9
:10106000C3F8042DBFF34F8FBFF36F8F03B05DF84C
:1010700004FB00BF08CA01202DE9F04188B01F4BD6
:101080001F4F002601961A6B016042F002021A639C
:101090001A6B02F002020192019A02961A6B42F058
:1010A00004021A631B6B03F004030293154B0493B1
:1010B000012504464FF0020803A9134805954FF493
:1010C00080430393CDF81880029B03F05BFF324608
:1010D0000921282003F0ACFC03A9384605960395A6
:1010E0000495CDF8188003F04DFF38462A4629466E
:1010F00004F06EF8204608B0BDE8F08100380240E8
:1011000000080240000021100004024010B5032333
:1011100084B0C943194080228DF806208DF805104F
:1011200000688DF8043001AC02AA0121CDE9024328
:1011300000F0B6F804B010BD10B584B013443031DF
:1011400003220292C3F3072C8DF80C1000688DF86F
:101150000DC003AC01AA012101948DF80E3000F0FE
:101160009FF804B010BD00BF0160704710B5064C79
:1011700000220121204613F04FF92046034A04497A
:10118000BDE81040FFF77CBD08CA0120A90C00088B
:10119000190E000810B5054CA36804F108001B687F
:1011A00098472046FFF738FE10BD00BF60D00120F1
:1011B00010B5054CA36804F108001B689847204649
:1011C000FFF72AFE10BD00BF70D0012010B5054CFE
:1011D000A36804F108001B6898472046FFF71CFE2F
:1011E00010BD00BF08D0012010B5054CA36804F164
:1011F00008001B6898472046FFF70EFE10BD00BF91
:1012000018D0012038B5054CA4F1280554F8083D44
:101210001B6820469847AC42F8D138BD60D0012009
:1012200000B585B0019271B901A9042303AA0E4843
:1012300006F032FE4FF0FF310C4813F0C7F8039868
:1012400005B05DF804FB01A90222094806F0B6FDCD
:1012500041F234234FF0FF310648039313F0B6F800
:10126000039805B05DF804FBD8CE012028D00120FA
:1012700030CF012030D0012008B50AC99B009BB2B5
:101280001268054806F008FEBDE8084003484FF024
:10129000FF3113F09BB800BFD8CE012028D0012029
:1012A00008B559B911680B48928806F087FDBDE86A
:1012B000084009484FF0FF3113F088B8116807481B
:1012C000928806F07BFDBDE8084005484FF0FF31ED
:1012D00013F07CB8D8CE012028D0012030CF0120D7
:1012E00030D0012010B50B46084C094AE45C09488F
:1012F000D25C4FF4806103F06BFF22460548BDE8E5
:1013000010404FF4005103F063BF00BF549901082F
:1013100050990108001402400A1E034818BF012218
:10132000202103F055BF00BF001002400A1E0348F1
:1013300018BF0122402103F04BBF00BF0010024044
:1013400010B58AB0254B00220192196B41F00801BB
:101350001963186B00F00800019001980292186B55
:1013600040F010001863186B00F010000290029813
:101370000392186B40F020001863186B00F02000F7
:10138000039003980492186B40F0400018631B6BA5
:101390001348079203F0400304934FF4405305A908
:1013A0000593012308920693049C03F0EBFD05A925
:1013B00060230C48059303F0E5FD05A942F20C43B8
:1013C0000948059303F0DEFD4FF498430748059361
:1013D00005A903F0D7FD0AB010BD00BF00380240D8
:1013E000000C0240001002400014024000180240AD
:1013F0002DE9F04F8FB00026B04C0296236BB04819
:10140000B04D43F001032363236B03F00103029308
:10141000029B0396636C43F480536364636C03F430
:101420008053A0220227039309A94FF003094FF02C
:10143000050A0992039B0A970B97CDF83090CDF8D7
:1014400034A003F09FFD10239D4809934FF001083D
:10145000122309A90A93CDF82C8003F093FD4023B1
:101460009748099309A90B9603F08CFD964B2B60C6
:101470004FF482736B604FF48023AB610823EB6100
:101480000A23AE60EE602E61C5F814802E626E6293
:10149000AE62EB62284606F04FFC002840F00B815C
:1014A0000490236B894E43F480032363236BF06025
:1014B00003F480030493049B70614023B36003F141
:1014C000804303F5193333604FF0806373604FF44A
:1014D000806333614FF4003333620423B061F06101
:1014E000F0623063C6F828907362304603F024FB44
:1014F0000246002840F0DF80414601903A20DFF8A4
:10150000ECB103F095FA3A2003F0D0FA019ACBF847
:101510000820CBF80C20CBF81420CBF81820CBF8FF
:101520001C20CBF82C20CBF83020694ACBF80020C7
:1015300004234FF0C062CBF82430CBF804204FF4E2
:1015400080634FF440325846AE64B563CBF8103038
:10155000CBF82890CBF8202003F0EEFA06460028BE
:1015600040F0A98002464146382003F061FA382055
:1015700003F09CFA324639462320C5F84CB0CBF82C
:10158000385003F055FA232003F090FA0596236BA8
:101590005048514D43F002032363236B03F00203D1
:1015A0000593059B0696236B43F004032363236B8B
:1015B00003F004030693069B0796236C43F48043D1
:1015C0002364236C0A9703F480430822079309A934
:1015D0000992079B0B97CDF83090CDF834A003F01B
:1015E000D1FC4FF400533D48099309A90B96CDF85F
:1015F00034A003F0C7FC122338480A9309A94FF41A
:1016000080530993CDF834A0CDF82C8003F0BAFCB8
:101610004FF482736B604FF48023AB610823EB615E
:101620000A23EB622E4B2B604FF40043EE602F61D8
:101630006E612E626E62AE62AB60284606F07CFB85
:10164000002838D10890236B43F400132363236BE5
:10165000244C03F400130893089B60604023A360AC
:101660004FF4806323614FF400332362E0601E4B2C
:101670006061A061E0616062E0622063C4F828906C
:101680002046236003F058FA0246A0B94146019073
:101690000F20AC64A56303F0CBF90F2003F006FA2A
:1016A000019A3946242003F0C3F9242003F0FEF9FF
:1016B0000FB0BDE8F08F03F05FF900BF00380240C3
:1016C00000000240D8CE012000300140F0CB0120C4
:1016D000106402400008024030CF012000040240A4
:1016E0000038004050CC01207060024090CB0120B7
:1016F0002DE9F04F8DB07F4C7F4D8048002602963B
:101700000996236C43F400132364236C03F4001341
:101710000293029B0396236C43F480032364236C9F
:1017200003F480030393039B0496236B43F00203AB
:101730002363236B03F00203C02204934FF0120AC9
:101740004FF002094FF0040807A9049B0792CDF857
:1017500020A0CDF82890CDF82C8003F013FC684B26
:101760002B60684B6B606E23EB6028464FF4804320
:10177000AE606E61AE61EE612E622B6103F08CFF94
:10178000002840F0B4800590236B5F4F43F40013B2
:101790002363236BB86003F400130593059B5B4B35
:1017A0003B604FF00073F8607861B861F86178626F
:1017B0007B604FF480664FF4803338463E613B6275
:1017C00003F0BAF90246002840F09180AF63BD6390
:1017D00001904F4F0C210B2003F02AF9019A7A60F7
:1017E000FA607A61BA61FA613A627A624FF0400B4C
:1017F000484A3A6038463E61C7F808B003F09CF9A1
:101800000246002873D101900D210C206F63BD6347
:1018100003F00EF901233948099307A9CDF820A058
:10182000CDF82890CDF82C80079603F0ABFB4FF451
:101830000073394D3148079307A909230B9303F02F
:10184000A1FB304B6B606E23EB604FF48043019A39
:101850002B612846314BAA606A61AA61EA612A625B
:101860002B6003F019FF002841D10690236B43F44D
:1018700000132363236B2A4C03F400130693069B87
:10188000A0604FF480332362264BE0606061A0616A
:10189000E06160624FF060682046C4E9003826616C
:1018A00003F04AF9074610BBAC63A5631E4C024621
:1018B0000C210D2003F0BCF81C4BC4F8048020461A
:1018C000C4F808B0E76026616761A761E761276235
:1018D0006762236003F030F9024640B90C212F20E3
:1018E0006C63A56303F0A4F80DB0BDE8F08F03F0BE
:1018F00043F800BF0038024030CE0120000402400F
:1019000000540040801A060010CA012010600240F6
:1019100070CA01202860024084CE01200058004097
:10192000D0CA01204060024030CB0120B8600240A4
:101930002DE9F04188B000253F4E0095336B3F4CB8
:101940003F4843F001033363336B03F0010300931B
:10195000009B0195336C43F400333364336C03F420
:10196000003301930223049301230C2705930323DF
:1019700006930DEB070107230793019A039703F0E2
:1019800001FB304B236020464FF4E1336360A560D8
:10199000E56025616761A561E56106F0D5FE002877
:1019A00047D10290336B284D43F400133363336BFC
:1019B000A86003F400130293244BE8606861A861F7
:1019C000E861286268624FF0006828464FF480673B
:1019D000C5E90038029A2F6103F0AEF8064640BB15
:1019E00002460D2110206563AC63194D03F020F809
:1019F000102003F05BF84023AB602846154BC5F878
:101A00000480EE602F616E61AE61EE612E626E62E7
:101A10002B6003F091F8024658B90D21112025637F
:101A2000AC6303F005F8112003F040F808B0BDE8FE
:101A3000F08102F0A1FF00BF0038024088CF0120F2
:101A40000000024000440040B0CC01208860024009
:101A500010CD0120A06002402DE9F04F8BB0674C03
:101A600067484FF00008CDF80480236B43F004036F
:101A70002363236B03F004030193019BCDF80880DB
:101A8000236B43F040032363236B03F04003029373
:101A9000029BCDF80C80636C43F020036364636C9D
:101AA00003F02003022601254FF0030A4FF0080936
:101AB000039305A94027039B079506960597CDF844
:101AC00020A0CDF8249003F05DFA4FF400734D4848
:101AD000079505A94C4D05930696CDF820A0CDF8A5
:101AE000249003F04FFA4FF440534648059305A95C
:101AF000CDF820A0CDF824900696CDF81C8003F0F8
:101B000041FA0C236B61414B2B60414B6B604FF4EE
:101B10004073AB6128464FF40043C5F80880C5F810
:101B20000C80C5F81080EB6106F00EFE002863D132
:101B30000490236B43F480032363236B354C03F43D
:101B400080030493049B344BA0604FF0206AC4E9E7
:101B5000003AE0606061A061E061E06220634FF400
:101B6000003320464FF480694FF00408A662C4F8A1
:101B700010902362C4F8248002F0DEFF8346002820
:101B80003AD1024606216C63A5633920234C02F04A
:101B90004FFF392002F08AFF214AA6624FF48033BA
:101BA0002046C4F804A0A760C4F81090C4F82480AC
:101BB000C4F80CB0C4F814B0C4F818B0C4F81CB021
:101BC000C4F82CB0C4F830B02260236202F0B4FF35
:101BD000064688B90246062146202C63A56302F01A
:101BE00027FF462002F062FF32460A21472002F01A
:101BF0001FFF0BB0BDE8F08F02F0BEFE00380240C0
:101C00000008024000180240C8CF01200014014023
:101C100080841E0070CD012028640240D0CD0120B8
:101C2000B864024030B5044683B001F08BFC40F24A
:101C30000E2204F5AA700021C4F85021C4F84C010A
:101C4000012516F0D5FC02F095FE1549009580237C
:101C500004F55972002002F055FE002811DA2046E2
:101C6000FFF76EFB2046FFF7C3FB2046FFF740FD62
:101C70002046FFF75DFE2046FFF7EEFE204603B04C
:101C800030BD08490095802304F57972284602F09A
:101C900039FE0028E3DB0449002002F013FEDEE7F2
:101CA000E8980108F89801080899010802680849AD
:101CB0001368884223F04003136003D0054B984219
:101CC00003D07047044801F015BA044801F012BA75
:101CD000D8CE012030CF012028D0012030D00120E3
:101CE000054B984200D0704702680448136823F0FF
:101CF0004003136001F0FEB9D8CE012028D00120A6
:101D0000014804F047B900BF30CE0120014804F07B
:101D10000DBE00BF30CE0120014804F03BB900BF2A
:101D200084CE0120014804F001BE00BF84CE012012
:101D3000014806F057BA00BFD8CE0120014806F08E
:101D400051BA00BF30CF012008B5044806F076FD37
:101D5000BDE80840024801F0CDB900BF88CF01209E
:101D600060D0012070B5104C94F83A5094F8393096
:101D7000EDB22046DEB206F061FD222D0BD0212E01
:101D800000D070BD94F83930202BFAD1BDE87040F6
:101D9000064801F0AFB994F83A30202BF1D1BDE8F4
:101DA0007040034801F0A6B9C8CF012078D00120C7
:101DB00070D0012010B5074C204602F0EFFF94F8D8
:101DC0003530012B00D010BDBDE81040024801F0B5
:101DD00091B900BF10CA012008D0012010B5074CEE
:101DE000204602F0DBFF94F83530012B00D010BD07
:101DF000BDE81040024801F07DB900BF70CA012063
:101E000010D0012010B5074C204602F0C7FF94F80F
:101E10003530012B00D010BDBDE81040024801F064
:101E200069B900BFD0CA012018D00120014802F0D2
:101E3000B5BF00BF50CC012010B5074C204602F0C2
:101E4000ADFF94F83530012B00D010BDBDE8104037
:101E5000024801F04FB900BFB0CC012060D0012092
:101E600010B5074C204602F099FF94F83530012B4D
:101E700000D010BDBDE81040024801F03BB900BFE2
:101E800030CB012020D00120014802F087BF00BFE5
:101E900090CB012010B5094C204602F07FFF94F84A
:101EA0003530012B00D010BD054B06482022BDE87F
:101EB000104083F8392001F01DB900BF70CD01201A
:101EC000C8CF012070D00120014802F067BF00BFD9
:101ED000F0CB012010B5094C204602F05FFF94F8CA
:101EE0003530012B00D010BD054B06482022BDE83F
:101EF000104083F8392001F0FDB800BFD0CD01209B
:101F0000C8CF012078D0012010B50446FFF78AFE23
:101F1000214604F26440FEF797FF214604F27C401C
:101F2000FFF7AAF8214604F59060FFF71DF9204657
:101F300010BD00BF38B5002201213048304C12F0EE
:101F40006BFA304A30492D48FEF79AFE00220121F3
:101F50002E4812F061FA2B4A2B492C48FEF790FECE
:101F6000002201212A4812F057FA002201212948B3
:101F700012F052FA234A28490020FEF781FE00227F
:101F80000121264812F048FA00220121244812F0CB
:101F900043FA1C4A23490020FEF772FE0022012169
:101FA000214812F039FA00220121204812F034FAB7
:101FB000144A1F490020FEF763FE002201211D483C
:101FC00012F02AFA002201211B4812F025FA0D4ACC
:101FD0001A490020FEF754FE04F12805204600228D
:101FE0000121083412F018FAAC42F7D1BDE83840AC
:101FF000044A13490020FEF743BE00BF28D0012049
:1020000038D00120A90C0008190E000830D001209A
:1020100060D0012068D001209511000870D0012007
:1020200078D00120B111000808D0012010D0012083
:10203000CD11000818D0012020D00120E91100089E
:1020400005120008B420704710B4B328144C94BF94
:1020500084464FF0000CA4F800C0B329114C94BF83
:102060008C464FF0000CA4F800C01418B42CDCBF50
:1020700002F1FF32801803EB0102D4BF80B2B3201B
:10208000B42ADCBF03F1FF33C918074C074B20808B
:10209000D4BF89B2B3215DF8044B1980704700BFEB
:1020A00080D0012082D0012000000020020000200A
:1020B00008B501F0D9FB4FF6FF7008BDB42070479A
:1020C00008B5292001F05AFCBDE80840382001F08D
:1020D00055BC00BF08B5282001F050FC142001F0C9
:1020E00059FC102001F04AFCBDE80840962001F0A0
:1020F00051BC00BF2DE9F041C0B282B0002600F112
:102100001E02A0F12F030DF105042A2088468DF848
:1021100004608DF805208DF806608DF8073002AF59
:1021200001F02CFC2546304601E015F8010B01F0CA
:102130001FFCBD42F9D15FFA88F1A1F14D032B20BC
:102140008DF805108DF8073001F018FC002001E033
:1021500014F8010B01F00CFCBC42F9D102B0BDE84F
:10216000F08100BF38B5D50802F4784305F0FC05CE
:102170001D441446ADB2FFF7BDFF2C2001F0FEFB5D
:10218000284601F0F5FBE00200F47840BDE8384055
:1021900001F0EEBB2DE9F8430546C60A05F01F081D
:1021A000F60008461F4606EBC826C5F34513114640
:1021B0004FEAC80805F4784505EB830508EB83284A
:1021C000FFF798FF2C20B6B2ADB21FFA88F801F0E5
:1021D000D5FB8FB107F1FF390024284601F0C8FB79
:1021E000304601F0C5FB4C45404601D001F0C0FB34
:1021F0000234A4B2A742F0D8BDE8F88338B504464B
:102200000D46FFF777FF29462046FFF773FF2E2084
:1022100001F0B4FB01F0B8FB01F0B6FB044601F09D
:10222000B3FBC4F38502C0F3C42303EB421304F4ED
:102230007840184480B238BD2DE9F0410F4605467C
:10224000114638461E461446FFF754FF2C2001F075
:1022500095FBEEB14FEAD50805F4784308F0FC0889
:1022600026449844ED02B6B21FFA88F8ADB2214672
:102270003846FFF73FFF2C2001F080FB0134404639
:1022800001F076FBA4B2284601F072FBA642EED123
:10229000BDE8F0812DE9F04F0446151983B02C20DC
:1022A0000F46994601F06AFBA54219DD254EDFF87D
:1022B0009C80DFF89CA0244A4FF0000B3188A1429B
:1022C0000AD8B8F80010B94206D8BAF80010A142EE
:1022D00002D31188B94206D20234A4B2AC42EDDB7B
:1022E00003B0BDE8F08F39F81B10C80800F0FC00FF
:1022F00001F4784108444FEA4B03023380B2019362
:1023000001F036FB019B39F81B0039F80310C002BD
:10231000C90A00EBC10080B201F02AFB691EA1428C
:10232000094A0BF1020BD7D0019B39F80310C80002
:10233000C0B2490900EB812080B201F019FB024ACA
:10234000CAE700BF80D001200200002082D0012017
:10235000000000202DE9F0431A4E1B4C33882688DC
:1023600055889488558901339B1B9EB2174BB3F84F
:1023700000C0174B1B880CF1010CACEB030C11FADD
:102380008CFC9389ADB28C4583B00F46804645EAFC
:10239000034513D915444FEA46090CF1FF34A1B2A5
:1023A00040460191FFF7A6FE2B4601993246404672
:1023B000FFF770FFBC42A4464D44EED803B0BDE821
:1023C000F08300BF0000002080D001200200002028
:1023D00082D001202DE9F043CF18B94283B00C46DA
:1023E0000646904611D20A9D4FEA4209A1B23046F4
:1023F00001910134FFF77EFE2B460199424630469B
:10240000FFF748FFBC424D44F0D303B0BDE8F08372
:10241000F0B583B001F028FA352001F0AFFA0020C2
:1024200001F0A6FA3A2001F0A9FA062001F0A0FA7C
:10243000B02001F0A3FA012001F09AFAFE2001F089
:1024400097FAB12001F09AFADE2001F091FA2120EA
:1024500001F08EFAB72001F091FA052001F088FA18
:10246000332001F085FAB82001F088FA052001F048
:102470007FFA332001F07CFAC82001F07FFA0420B3
:1024800001F076FA032001F073FAC92001F076FA20
:102490005E2001F06DFA082001F06AFACA2001F00E
:1024A0006DFA0A2001F064FA0C2001F061FA0220B2
:1024B00001F05EFACC2001F061FA032001F058FA35
:1024C000042001F055FAD02001F058FA0C2001F058
:1024D0004FFAB32001F052FA022001F049FAC0206D
:1024E00001F04CFA532001F043FAC52001F046FAFE
:1024F000002001F03DFA452001F03AFAC22001F037
:102500003DFA032001F034FA122001F031FA0026DE
:10251000DD208DF8046001F031FA304601F028FA30
:10252000B42001F02BFA112001F028FA962001F0D6
:1025300031FA0DF105051E22D1232A208DF8052040
:102540008DF806608DF8073002AF01F017FA2C46BF
:10255000304601E014F8010B01F00AFAA742F9D164
:102560000026B3232B208DF805608DF8073001F08D
:1025700005FA304601E015F8010B01F0F9F9A54222
:10258000F9D1362001F0FAF9832001F0F1F9292080
:1025900001F0F4F9382001F0F1F92C2001F0EEF906
:1025A0004BF6D854002001F0E3F9013CFAD1142095
:1025B00003B0BDE8F04001F0EDB900BFF020704776
:1025C00010B4EF28144C94BF84464FF0000CA4F8CC
:1025D00000C0EF29114C94BF8C464FF0000CA4F8BA
:1025E00000C01418F02CDCBF02F1FF32801803EB9E
:1025F0000102D4BF80B2EF20F02ADCBF03F1FF3329
:10260000C918074C074B2080D4BF89B2EF215DF871
:10261000044B1980704700BF84D0012086D0012070
:102620007400002076000020F020704708B501F00B
:102630001BF9042001F0A2F901F0A6F901F0A4F9B8
:10264000C0B208BD08B5292001F098F9BDE80840DE
:10265000112001F093B900BF08B5BD2001F08EF93B
:10266000FE2001F085F9102001F088F9BDE808404E
:102670000A2001F08FB900BF2DE9F041C3B282B04A
:102680000026A3F111022A200DF1050488468DF8D9
:1026900004608DF805308DF806608DF8072002AFD4
:1026A00001F06CF92546304601E015F8010B01F008
:1026B0005FF9BD42F9D15FFA88F1A1F111032B2036
:1026C0008DF805108DF8073001F058F9002001E071
:1026D00014F8010B01F04CF9BC42F9D102B0BDE88D
:1026E000F08100BF10B51446FFF7C6FF2C2001F0A3
:1026F00045F92046BDE8104001F03AB970B50646EC
:10270000084611461D46FFF7B7FF2C2001F036F9A9
:102710003DB1002401343046A4B201F029F9A542AC
:10272000F8D170BDF8B50E460746114630461D4635
:102730001446FFF7A1FF2C2001F020F97DB12544BC
:10274000ADB221463046FFF797FF01342C2001F04F
:1027500015F9A4B2384601F00BF9A542F1D1F8BD44
:102760002DE9F04F0446151983B02C200F469946E9
:1027700001F004F9A54219D9124EDFF84C80DFF8B8
:102780004CA0DFF84CB000233288A2420BD8B8F836
:102790000020BA4207D8BAF80020A24203D3BBF8FF
:1027A0000020BA4205D20134A542EDD803B0BDE8FD
:1027B000F08F39F81300019301F0DAF8019B01332F
:1027C000F1E700BF84D0012086D0012074000020F2
:1027D000760000202DE9F0431A4E1B4C33882688E2
:1027E00055889488558901339B1B9EB2174BB3F8CB
:1027F00000C0174B1B880CF1010CACEB030C11FA59
:102800008CFC9389ADB28C4583B00F46804645EA77
:10281000034513D915444FEA46090CF1FF34A1B220
:1028200040460191FFF728FF2B460199324640466A
:10283000FFF796FFBC42A4464D44EED803B0BDE876
:10284000F08300BF7400002084D0012076000020B7
:1028500086D001202DE9F043CF18B94283B00C4651
:102860000646904611D20A9D4FEA4209A1B230466F
:1028700001910134FFF700FF2B4601994246304693
:10288000FFF76EFFBC424D44F0D303B0BDE8F083C8
:1028900038B504460D46FFF7EFFE29462046FFF700
:1028A000EBFE2E2001F06AF801F06EF801F06CF8F2
:1028B000044601F069F8C4F38502C0F3C42303EBB6
:1028C000421304F47840184480B238BDF0B585B0A6
:1028D00000F0CAFF102001F051F80A2001F05AF868
:1028E000012001F04BF8C82001F054F8112001F04C
:1028F00045F8782001F04EF8362001F03FF800202E
:1029000001F036F83A2001F039F8052001F030F8EE
:10291000212001F033F80026EF232A200DF10105D4
:102920008DF800608DF801608DF802608DF803303D
:1029300001AF01F023F82C46304601E014F8010BFA
:1029400001F016F8BC42F9D12B2001F017F82C4603
:10295000002001E014F8010B01F00AF8BC42F9D1A3
:102960000C263323B2208DF800608DF801608DF8BD
:1029700003308DF804300DF1050700F0FFFF2C4601
:10298000304601E014F8010B00F0F2FFBC42F9D12F
:10299000B72000F0F3FF352000F0EAFFBB2000F085
:1029A000EDFF1F2000F0E4FFC02000F0E7FF2C2027
:1029B00000F0DEFFC22000F0E1FF012000F0D8FFB0
:1029C000C32000F0D5FFC42000F0D8FF202000F085
:1029D000CFFFC62000F0D2FF0F2000F0C9FFD020AB
:1029E00000F0CCFFA42000F0C3FF082311228DF8D3
:1029F00001308DF802208DF803300C2239238DF838
:102A000004208DF80630152250238DF805208DF80E
:102A10000830332213238DF807208DF80A30362230
:102A20002923D0268DF809208DF80C3014222D236F
:102A3000E0208DF800608DF80B208DF80D300DF141
:102A40000E0700F09BFF2C46304601E014F8010B06
:102A500000F08EFFA742F9D106238DF804308DF8DF
:102A600005305123102144228DF8083016238DF8AB
:102A700002108DF807200B212F228DF80A30E1205B
:102A800031238DF809108DF80C208DF80D3000F0F1
:102A900075FFD02001E015F8010B00F069FFAC4292
:102AA000F9D1292000F06AFF112000F067FF3520DE
:102AB00000F064FF002005B0BDE8F04000F058BF12
:102AC00070B5012882B00BD002280BD060243620CC
:102AD00000F054FF204602B0BDE8704000F048BF4F
:102AE0000024F4E700250122F02333208DF8005064
:102AF0008DF801508DF802208DF803308DF80450C8
:102B00008DF805506C4600F039FF0DF1050628469A
:102B100001E014F8010F00F02BFFA642F9D1372095
:102B200000F02CFF002000F023FF502000F020FFD9
:102B3000C024CCE738B5054CA4F1280554F8083D6D
:102B40001B6820469847AC42F8D138BD38D20120E6
:102B500010B5E9B1012926D0164C174A002332F8E6
:102B60001110E1604FF44862204662602361A36067
:102B700005F052FD0246D0B90E212C2001F058FF7D
:102B8000204605F003FCBDE810402C2001F08EBF6C
:102B9000032000F0ABFD2C2001F096FFBDE81040B3
:102BA000044805F003BC032000F094FDF3E701F0B6
:102BB000E3FE00BFCCD00120589901080329F8B5E5
:102BC00014461FDD1B4D1C4F012C05F10C064FF068
:102BD00000030AD0022C0ED1F85C00F093FDB54240
:102BE00008D0012C55F8043BF4D1F85C00F072FDDC
:102BF000B542F6D1F8BD0CB101F0BEFEF85C00F0B4
:102C000075FDECE7012A0FD0022A07D0002AF3D184
:102C1000094B585CBDE8F84000F068BD064B585CB5
:102C2000BDE8F84000F06EBD034B585CBDE8F840CD
:102C300000F050BD6C99010864990108F0B44FF0A0
:102C400060434FF0E025D3F8000ED5F8FC4D154E4B
:102C5000154F44F08074C5F8FC4D4FF0010C134C37
:102C6000C3F8B04F0CFA02F2114C20EA0200002522
:102C700001394FF0020CC3F8000E0243C3F8805E26
:102C80000C48C4F8F0C021614FF48071C3F8405E75
:102C90003760C4F80413C3F8800EF0BCC3F8002EEC
:102CA000704700BF001000E0FE03004055CEACC5E9
:102CB000000004E00D000100F0B5A5B0364A374B26
:102CC00000240194106C40F080501064126C02F0EB
:102CD00080520192019A02941A6842F440421A60AA
:102CE0001B68119103F4404302930224012304253D
:102CF00002980A930D214FF4A0224FF4800608A8F1
:102D0000CDE90812CDE90E46CDE912450D93109597
:102D1000149404F003FD00283BD14FF48053059038
:102D200007900F27032103A806930397049404F048
:102D3000C3FA034668BB032218921D934FF48072B6
:102D4000229368231C9215934FF00062482315A824
:102D5000199416951F92179304F090FB0446C0B97E
:102D60003146024604F020FA04F06CFA04F03EFB0F
:102D70000B4BA3FB0030800901F0B6FE284601F0A2
:102D8000CFFE224639464FF0FF3001F051FE25B00C
:102D9000F0BD01F0F1FD00BF0038024000700040BE
:102DA000D34D621038B505462D200C4601F08CFE3F
:102DB000002001F093FC44B930BF2D2001F076FED5
:102DC000BDE83840012001F089BC0121002003F05A
:102DD00079FE60212846FFF76FFFEEE738B5FFF771
:102DE000E1FF074D01242846002111F0EFFA0835D4
:102DF00020B90134052CF6D1062038BD204638BD57
:102E000018D20120132908B501D9022008BD04F009
:102E1000C9FE002008BD00BF132901D9002070475A
:102E200004F0C6BE08BA704770B588B0184C19488F
:102E300000250195236B43F010032363236B069554
:102E400003F01003019303A90126019B04960F23AD
:102E50000393059602F096F8284600F047FC3046AA
:102E600000F044FC022000F041FC032000F03EFC96
:102E70000295236C084A094943F080032364236CBC
:102E8000116003F080030293029B08B070BD00BF85
:102E90000038024000100240CCD00120001C00404D
:102EA0002DE9F0438BB00024394B01941A6B0227B3
:102EB0003A431A631A6B3A400192019A02941A6BD0
:102EC00042F020021A631A6B02F020020292029A68
:102ED00003941A6B42F040021A631A6B02F040022C
:102EE0000392039A04949A6B3A439A639B6B0697F6
:102EF0003B400546032604934FF009082548CDF8CA
:102F00002480C02305A905934FF00A09049B079468
:102F1000089602F037F84FF440731E48059305A950
:102F2000069707940896CDF8249002F02BF81A48DB
:102F3000CDF8248005A94FF0040806970794089659
:102F4000CDF8148002F01EF840231448059305A91B
:102F5000069708960794CDF8249002F013F8104BCA
:102F60002B63102217236C63C5F83880EA632B6447
:102F70006C64AC64EC642C6505F1300003F078FE01
:102F800020B901F07DF90BB0BDE8F08301F0F4FC4D
:102F900000380240001402400004024000180240C1
:102FA000001000A000B583B00B4B002201925A6BB9
:102FB00042F040025A635B6B084A40F87C2F03F0F2
:102FC00040030193019B04F063FD10B903B05DF869
:102FD00004FB01F0D1FC00BF00380240000806509D
:102FE00070B588B00026184B02961A6C174C42F444
:102FF00080721A641B6C03F480730D46029301A95E
:1030000003A8029B04F018FA04F0F6F9104A2260B3
:1030100043001048266140F2E732E260A0FB032340
:103020009B0C013B20466360A66005F0F5FA042284
:1030300029462D2001F0FCFC2D2001F037FD204613
:1030400005F0A4F908B070BD003802400CD1012091
:103050000020004083DE1B4338B504460D4601F0D6
:1030600009FB214B1A6842F400721A601A6842F494
:1030700080621A601A6842F480721A60032001F0BC
:10308000C5FC0F212046FFF7ABFF29462046FFF77E
:1030900013FE04F0D7F8002208212046FFF7CEFDEA
:1030A000012000F03BFB2046FFF7BEFE2046FFF765
:1030B000F7FE2046FFF776FF0C4A0D480121C2F8C3
:1030C0003C1E00237F21FF22C4E90003A160E260CF
:1030D00023616361A361204604F0F6FC08B9204631
:1030E00038BD01F049FC00BF003C024000004742EF
:1030F0000028004000B583B001A911F083F958B150
:10310000019B4BB14FF0E0234FF08052C3F8042DE8
:10311000BFF34F8FBFF36F8F03B05DF804FB00BFA9
:10312000FEE700BFFEE700BFFEE700BFFEE700BF0F
:10313000FEE700BF704700BF70B5124D012002F0DE
:1031400055F800F073FB2B78BFF35B8FDB07044669
:1031500008D50D4E30680D4BBDE8704003EBC00044
:10316000FFF7C8BF2846FDF77FFD074E0028F1D0C6
:10317000002C0CBF0023042328463360FDF77AFDA2
:10318000E8E700BF88D0012038D2012010D201200A
:1031900008B5022002F02AF8BDE808400148FFF710
:1031A000A9BF00BF18D2012008B50E4B5B695A04B5
:1031B00004D40C4B5B691B040BD408BD4FF4804056
:1031C00002F014F80848FFF795FF064B5B691B04F3
:1031D000F3D54FF4004002F009F8BDE80840034879
:1031E000FFF788BF003C014028D2012020D20120F7
:1031F00008B5034805F0FAF8024B01221A7008BD21
:103200008CD001200CD2012008B5044805F0EEF85E
:10321000BDE80840032000F075BA00BFCCD0012003
:1032200008B5034805F0E2F8BDE8084001F0CABB64
:103230000CD10120014801F0B1BD00BF4CD10120EB
:10324000014801F0ABBD00BFACD1012038B5094C3D
:1032500004F12805204600220121083411F0DCF891
:10326000A542F7D1BDE83840034A04490020FDF7E4
:1032700007BD00BF10D20120A90C0008352B0008A3
:1032800010B54FF6FF7000F08DFD002000F0DEFC61
:103290004FF6FF7000F0E0FC084800F0E3FC084A3D
:1032A00001236421002000F0E3FCBDE81040054A42
:1032B00001237821002000F0DBBC00BF800000204B
:1032C000789901088499010870B504460D4603E019
:1032D000237883B101F088FB204601F097F803467C
:1032E0006420002BF6D1002DF2D0012DF2D12378ED
:1032F000013B012BEED801F071FB86B2204601F0B4
:1033000085F80028FAD175B92378013B012B0FD934
:1033100001F064FB6438B0424FF0640010D9BDE89E
:10332000704001F061BB012DF2D12378002BEFD169
:10333000642001F059FBBDE87040642001F054BBEB
:1033400001F052FBDAE700BFF8B5174C34F8115022
:10335000044600201E46174600F078FC2946142239
:10336000284600F0D5FD4FF6FF7000F06FFC0A22F2
:103370002946284600F0CCFD20460121FFF7A4FF96
:1033800063883B80E388338000212046FFF79CFF61
:103390004FF6FF7000F05AFC294628461422BDE87B
:1033A000F84000F0B5BD00BF049A010838B500210F
:1033B0000446C068FFF730FD034668B1020C638223
:1033C000E068A2820121FFF727FD50B1030CE082E3
:1033D00023830120207438BDE0680121FFF71CFD24
:1033E00098BB2046FFF74CFF00F020FC054600F09C
:1033F00025FC012281B2A8B200F0DAFF054640BBED
:10340000234604F1120203F8140B01462046FFF78D
:103410009BFF638AA28AE068294603EB0242FFF71A
:10342000F1FC234604F1160203F8185B2046012143
:10343000FFF78AFF228BE38AE06803EB0242012157
:10344000FFF7E0FC0120207438BD030CE0822383E9
:10345000C7E74FF6FF7000F0FFFB4FF4784000F035
:10346000F5FB154A01239121002000F001FC134ACD
:103470000123A021002000F0FBFB012D15D0022D1F
:1034800009D000F0DBFB413881B20D4A0123002056
:1034900000F0EEFB9DE700F0D1FB413881B2094A14
:1034A0000123002000F0E4FB93E7074A2B46AF21FD
:1034B000002000F0DDFB8CE7909901089899010845
:1034C000EC990108D8990108BC99010838B505465E
:1034D00000F0F2FD0CF0E2FA00F0A8FB044600F068
:1034E000ADFB022281B2A0B200F062FF00B138BD94
:1034F0002846FFF75BFFBDE8384001F01DB800BF6C
:1035000010B50E4B5C6982B0202001F06FFEA3065F
:1035100001D402B010BD0A4801A910F073FF019B4D
:10352000012BF6D14FF0E0234FF08052C3F8042D69
:10353000BFF34F8FBFF36F8F02B010BD003C01404F
:103540003CD2012010B582B00446FFF785FD002172
:103550000B4B01911A6B84F8401142F48052C4F86D
:103560003C411A631B6B03F480530193019B10F0E1
:103570009DFE042006F04CFC204602B010BD00BFAA
:103580000038024010B5064C00220121204610F000
:1035900043FF2046034A0449BDE81040FDF770BBD5
:1035A0003CD20120A90C0008190E000830B5464B8A
:1035B000464C83428BB04FF0000544D00395236BFB
:1035C000434843F002032363236B079503F0020390
:1035D00003934FF48063059312230693022305A9F6
:1035E00008930423039A099301F0CCFC4FF4007371
:1035F00005A9059336480923099301F0C3FC0495F6
:10360000236C43F480032364236C03F4800304934A
:10361000049B236A43F480032362236A23F4800318
:1036200023622A460F21212001F002FA212001F015
:103630003DFA2A460F21222001F0FAF9222001F05A
:1036400035FA0BB030BD0195236B214843F00203DE
:103650002363236B079503F0020301934023059333
:1036600012230693022305A908930423019A0993C0
:1036700001F088FC05A980231548059301F082FC20
:103680000295236C43F400132364236C03F40013AA
:103690000293029B236A43F400132362236A23F4F8
:1036A000001323622A460F211F2001F0C1F91F20B9
:1036B00001F0FCF92A460F21202001F0B9F9202061
:1036C00001F0F4F90BB030BD44D2012000380240C3
:1036D000000402400246034B034833F82210002244
:1036E00001F076BD149A0108001002400246034B17
:1036F000034833F82210012201F06ABD149A010830
:10370000001002400246034B034833F8221001F038
:1037100063BD00BF149A0108001002402DE9F04774
:103720008CB00223002409930A93DFF8F4803A4E08
:103730003A4DDFF8F0A0DFF8F09007460123F4B12E
:10374000012C4FF0000235D0022C4FD0032C58D062
:1037500006922A6B42F040022A632A6B02F0400272
:103760000692069A0793BFB1012F2ED00134052C83
:1037700006F104061AD038F8023B002CE0D102947E
:103780002A6B42F001022A632A6B079302F00102BE
:103790000292029A002FE7D13068089707A90134F6
:1037A00001F0F0FB052C06F10406E4D100200CB07A
:1037B000BDE8F08703922A6B42F040022A632A6B2D
:1037C00002F040020392039ACCE73068CDF820A0C3
:1037D00007A901F0D7FB14F90900019000220F217D
:1037E00001F026F9019801F061F9BFE704922A6B14
:1037F00042F020022A632A6B02F020020492049A0B
:10380000B0E705922A6B42F020022A632A6B02F08D
:1038100020020592059AA5E72C9A0108003802407B
:103820000A9A010800001110249A010870B50B488B
:103830000B4E0C4D0121002401F0C4FC50B90134A1
:10384000052C09D056F8040B35F8021B01F0BAFC20
:103850000028F4D0E0B270BD204670BD00000240E8
:10386000309A01080A9A010830B53C483C4AADB08C
:103870004FF02045CDE9185009200A9024200C90E3
:103880000720002313901020CDE91C304FF4805006
:1038900022904FF480400124022124904FF4001024
:1038A000CDE92803CDE90E11CDE91A33CDE91E3358
:1038B000CDE9203310931493159116911793239308
:1038C0002593269327930B940D94119412940193AE
:1038D000906B20439063906B20400190019802937D
:1038E000106B40F008001063106B00F008000290AD
:1038F00002980393106B40F010001063106B00F0FF
:103900001000039003980493136B164843F02003B0
:103910001363136B069103F020030493049B079435
:103920000C23032205A909934CF2B3730892059363
:1039300001F028FB4FF6807305A90B48059301F0B1
:1039400021FB05A90948059401F01CFB11AA0AA94D
:1039500018A804F0EDFC2DB030BD00BF040100A09C
:1039600000380240000C02400010024000140240E7
:103970004FF0C0435880BFF34F8F70474FF0C043A4
:103980001880BFF34F8F70474FF0C043588880B204
:10399000704700BF01F028B810B50E4C204603F068
:1039A0008DF80346A0B90C480C49A360C4E9000196
:1039B0004FF480422046E36022616361A361E361CA
:1039C0002362FFF7F3FD2046BDE8104001F064BE1E
:1039D00010BD00BF44D2012000540040A086010069
:1039E00010B586B04FF47A73174C029394460123B6
:1039F0000A4601460DF117000090019320468DF80C
:103A000017C001F02BFF08B906B010BD204601F029
:103A10000BFF204603F052F803460028F4D10B496F
:103A20000B48A360C4E900014FF480422046E360E4
:103A300022616361A361E3612362FFF7B7FD204662
:103A400001F02AFE06B010BD44D20120A08601007C
:103A50000054004030B587B01A4C0A4600210123BB
:103A60004FF47A758DF8171001460DF1170000908C
:103A700002950193204601F09FFF18B99DF81700A9
:103A800007B030BD204601F0CFFE204603F016F807
:103A900003460028F2D10C490C48A360C4E9000198
:103AA0004FF480422046E36022616361A361E361D9
:103AB0002362FFF77BFD204601F0EEFD9DF8170025
:103AC00007B030BD44D20120A08601000054004060
:103AD00030B5184D85B04FF47A74CDE900230294C7
:103AE0000A4601230146284601F066FF044610B944
:103AF000A0B205B030BD284601F096FE284602F07F
:103B0000DDFF03460028F3D10B490C4AAB60C5E941
:103B1000001228464FF48042EB602A616B61AB6172
:103B2000EB612B62FFF742FD284601F0B5FDA0B224
:103B300005B030BD44D2012000540040A0860100F1
:103B40002DE9F04FDFF8DCA08BB0DAF808300691F1
:103B500099880890D8880491CB1DDB100393C1EBA2
:103B6000C303DBB20590079300284CD000230193D8
:103B7000DFF8B4B002924B1E0993069B019A9F187E
:103B8000039B012BBFB241D0022B42D0029A567840
:103B90001378360246EA034693781E43049B43B3E8
:103BA000099B079A089C9D18049B4FF00108A5EB00
:103BB00003090BE05B693946204613B1BAF80020CF
:103BC0009847013D01344D45A4B212D008FA05F3DF
:103BD0003342DBF80030EDD15B6920463946002BDB
:103BE000EFD0BAF80420013D984701344D45A4B206
:103BF000ECD1029A0399019B0A440292059A01337F
:103C000093420193B9D10BB0BDE8F08F029B1E78AF
:103C1000C4E7029B1E785B7846EA032676BAB6B202
:103C2000BCE700BF98D20120A4D2012008B5024B06
:103C30001B689B6A984708BDA4D2012008B5024BB7
:103C40001B68DB6A984708BDA4D20120014B1860AD
:103C5000704700BF98D20120014B5860704700BFE9
:103C600098D20120014B9860704700BF98D2012084
:103C70002DE9F84F1546164615F8014B8246884641
:103C80009B462CB1002415F8011B01340029FAD100
:103C9000DFF8B0902A4FD9F800309B6A9847BA688D
:103CA000BBF1010F9388B0FBF3F040D0BBF1020FE2
:103CB00006D1001B10FB03F0A0EB0A0A1FFA8AFAD8
:103CC0000FFA8AF3002B06F1FF36D8BF4FF0010A36
:103CD000002410E03378D5881268203B05FB03F3FD
:103CE0000EFB0322FFF72CFFBB6898880134824447
:103CF000A4B21FFA8AFAD9F8003016F8015F9B6A5D
:103D0000003D18BF01259847BA68B2F804C00346C1
:103D10000CFB14339BB20CF1070E63455046414631
:103D20004FEAEE0E01D3002DD4D1BDE8F88F001B71
:103D300003FB00F00AEB500A1FFA8AFAC0E700BF43
:103D400098D20120A4D201202DE9F047DFF850A03D
:103D5000DAF800502C6A07468846164644B10F4AE6
:103D600033461088A4460A463946BDE8F047604706
:103D70008AB1DFF8289001E0DAF800506B6907EBB0
:103D8000040C41461FFA8CF0013413B1B9F800203D
:103D90009847A642F0D1BDE8F08700BF98D2012035
:103DA000A4D201202DE9F041DFF838800C4ED8F87C
:103DB00000303768DB6A30609847054660B1002400
:103DC000D8F800309B6A9847A1B20246013400201F
:103DD000FFF7BAFFAC42F3D1BFB23760BDE8F08164
:103DE00098D20120A4D201202DE9F04F530087B0D2
:103DF000C3F10303CDE90001424F434E049315463E
:103E0000002409E0049B621B0A33013D013403EBEB
:103E10008203A542049371D33B685B69002B61D098
:103E20000099A2B201EB020B01990392A8B2091A00
:103E30001FFA8BFB89B23288029058460591984749
:103E40003B68039A00995B69A1EB020A1FFA8AFAA0
:103E50003288002B46D00599504698470298009921
:103E60003B6832885B6900EB010901980399411AAC
:103E70001FFA89F989B2002B34D04846059198473A
:103E80003B68009A02985B69A2EB00081FFA88F869
:103E90003288002B26D0059940469847019B02980E
:103EA000328818443B685B6981B2DBB158460291A5
:103EB00098473B6832885B69A3B10299504698479E
:103EC000019B0399328819443B685B6989B24BB105
:103ED0004846029198473B6832885B6913B1029962
:103EE00040469847094BB360049B002B8ADA06339F
:103EF00003EB84030134A54204938DD207B0BDE8DF
:103F0000F08F00BFA4D2012098D2012078000020B9
:103F10002DE9F04FDFF8B8A05500BAF80030CAF824
:103F2000003083B0914680460F46C5F10305164622
:103F30000024C6B97CBB002D05F1060345DBA31B9D
:103F40000A3505EB8305013E0134A642F1D2BAF8E9
:103F50000030CAF800304A463946404603B0BDE852
:103F6000F04FFFF741BFB2B21FFA84FBA8EB02008B
:103F700007EB0B01520080B292B289B2019200901D
:103F8000FFF7E2FEA7EB0B01019A009889B2FFF759
:103F9000DBFE002CCFD0A2B21FFA86FBA8EB0200FA
:103FA000A7EB0B01520080B292B289B2019200904D
:103FB000FFF7CAFE0BEB0701019A009889B2FFF7E1
:103FC000C3FE002D05F10603B9DA03EB8405BBE758
:103FD00098D201202DE9F0412F4D304BAB600024E9
:103FE0004FF6FF7780466F602C60FCF7D1FB2C48C2
:103FF0002C4E0122202101F0EBF822464FF4006103
:10400000294801F0E5F8052000F0EEFC01224FF40C
:104010000061254801F0DCF80A2000F0E5FC2246AA
:104020004FF40061204801F0D3F8142000F0DCFCCC
:1040300001224FF400611C4801F0CAF80A2000F088
:10404000D3FC73689847852810D0184E736898473A
:10405000B84202D00120BDE8F081154A33681660ED
:104060009847144BAB602046BDE8F081104A336896
:1040700016609847B8F1000F07D0B8F1020F04D0CE
:104080000C4BAB600020BDE8F0814046FEF718FD08
:10409000084BAB600020F6E798D201208800002092
:1040A000001402403C000020000C024004000020EC
:1040B000A4D20120780000200220FFF78BBF00BFB0
:1040C00030B595B00022034601214FF480750524D8
:1040D0004FF08070CDE90E20CDE90021CDE912220C
:1040E0000C9506940D920B92119204920391102557
:1040F0004FF480046A4606A904480295059402F02C
:104100008DFE003818BF012015B030BDA8D20120A7
:1041100010B594B04FF48071062200230C910692E2
:1041200016480D9341F2883206A9CDE90E33CDE948
:1041300012330B93119302F011FE034610B10120CC
:1041400014B010BD0222CDE9002210220493029285
:1041500001244FF480034FF08072039405930F9273
:1041600006A9052441F288336A460448069402F001
:1041700055FE003818BF012014B010BDA8D2012090
:104180002DE9F0418AB03A4B3A4D3B480024019466
:104190009A6B42F002029A639A6B02F00202019259
:1041A000019A9A6942F002029A619A6922F0020227
:1041B0009A6102941A6B4FF0400842EA08021A63AF
:1041C0001A6B02EA08020292029A03941A6B42F0F6
:1041D00002021A631A6B02F002020392039A049419
:1041E0001A6B42F020021A631B6BCDF8148003F0A7
:1041F0002003049302230693049B01230A2705A9A5
:104200000793032308930926099700F0BBFE05A92D
:1042100004231A4805930794099600F0B3FE05A9F4
:1042200028464FF480730593099700F0ABFE05A96B
:1042300028464FF400730593099700F0A3FE8023EE
:1042400005A928460593099600F09CFE05A9284675
:10425000CDF81480099600F095FE22460F215C20CF
:1042600000F0E6FB5C2000F021FC0AB0BDE8F08124
:1042700000380240001402400018024000040240CE
:1042800070B5494C494B236090B0204602F052FD76
:10429000054610B1012010B070BD01462046FFF761
:1042A0006FFF04221023A260E36065604FF0807608
:1042B00096FAA6F3B3FA83F3013B4FF480622046EB
:1042C00023616261A561E561256202F0D1FC0028ED
:1042D000E0D1CDE90A00CDE90E004FF480756623E8
:1042E000099007900D9041F2883202A92046089566
:1042F000029302F033FD10B1042010B070BD992379
:1043000041F2883202A92046029302F027FD0028DC
:10431000F2D141F28830FFF7D3FE0028ECD185239B
:10432000CDE90A06CDE90E0002930990012307901A
:104330000D9041F2883202A9204608950C9302F0B4
:104340000DFD0028D8D141F288320DF10701204639
:1043500002F0A8FE0028CFD1FFF7DAFE0028CBD16B
:1043600081230293F02292FAA2F29DF807300A20EC
:10437000B2FA82F200FA02F203F00F03134302A929
:1043800041F2883220468DF8073002F0E7FC002821
:10439000B2D141F288320DF10701204602F006FE4B
:1043A00000283FF478AFA7E7A8D20120001000A0B2
:1043B000F8B5124C124E236830781546984763685A
:1043C00070209847CD2801D00320F8BD0D4F7023F1
:1043D00033703C600C4B55B906221A70A3687020EC
:1043E00098473B683078DB6898470020F8BD022D7D
:1043F0000CBF08220C221A70F0E700BF94000020C6
:10440000F4D20120F8D20120900000202DE9F04FD5
:10441000DFF8D8B0324ADBF8003005461B69107867
:1044200083B098472870002850D06946DFF8C080D4
:104430002C4F01AE05F1020A4FF000090C46DBF8E3
:104440000030274A5B691078214632469847264B50
:104450001A7810073ED420883388910703D5C0F11D
:10446000EF0080B22080520703D5C3F1EF039BB267
:104470003380D8F800C0396860458CBFA0EB0C02CF
:10448000ACEB00028B428CBFA3EB010EA1EB030E41
:1044900092B21FFA8EFE7244052AD2BF1FFA8CF028
:1044A000C8F800003B602AF8020BD8BF8BB2AAF80C
:1044B00002302B7809F101094B4504F1020406F1A1
:1044C000020608F1040807F10407B8D8002003B079
:1044D000BDE8F08F2388308820803380BDE700BF9F
:1044E000F4D2012004D3012090000020F8D2012052
:1044F000FCD2012070B586B00C4B0D4C0D4800224B
:1045000000921A6B42F040021A631B6B029403F094
:104510004003009301220223202501A9009E01955A
:104520000392049300F02EFD06B070BD00380240E7
:10453000000021100018024008B5FFF7DBFF0F2133
:104540000022172000F074FA172000F0AFFA044B95
:10455000044A1B6810789B699847002008BD00BF7B
:10456000F8D20120F4D20120704700BF002070472C
:1045700010B50446FFF710FAA821E0B2FFF76AFA77
:1045800080B210BD10B582B000240221C0B28DF8F7
:104590000740FFF75FFA8DF807009DF8073003F03A
:1045A0000F038DF807309DF80730022B88BF8DF878
:1045B00007409DF80710044B9DF807005970002232
:1045C0009A7002B010BD00BF0CD3012070B5164C1C
:1045D0001546A37862789A4282B00E461FD903B37B
:1045E000012B14BF0021092104230DEB0302C0B2EB
:1045F000FFF76EFA9DF804309DF805209DF807102E
:104600001B0203F470631A439DF8063032801B02CC
:10461000A27803F470630B4301322B80A27002B0C6
:1046200070BD0321E0E700BF0CD301200122A421CB
:10463000C0B2FFF7D5B900BF0022A421C0B2FFF776
:10464000CFB900BF064A1378834204D0517888421C
:1046500001D013B101B170470123D054FFF79CB9C9
:1046600010D30120704700BF0022A421C0B2FFF781
:10467000B7B900BF10B4174A116885B04FF0E023F6
:10468000490400910099D3F8244D2143C3F8241D17
:104690001168890401910199D3F8244D2143C3F88D
:1046A000241D12680C4912010292029AD3F8144D8B
:1046B0002243C3F8142D0A686FEAC2020392039AD8
:1046C000D3F8141D0A40C3F8142D05B05DF8044B4F
:1046D000704700BFC0000020BC000020012882B04D
:1046E0000BD00B4B1B684FF0E022DB430093009B89
:1046F00011690B40136102B07047064B4FF0E02286
:104700001B680193019B11690B43136102B0704751
:10471000BC000020C0000020F0B5C56886684FF0DE
:10472000000E04694368A6EB050CA54204F1FF34B2
:1047300028BFA4199445A4EB050428BF94466445FA
:1047400028BF6446A644121B2F1954B1013D2B44C7
:1047500001EB040C11F8014B03F8014F8C45F9D122
:104760008668B74214BF3D460025C560002AD8D1EF
:104770007046F0BD70B4C6688568AB1B93420ED915
:104780004368B51842B1013E33448C1811F8012B2F
:1047900003F8012FA142F9D1C56070BC704744688D
:1047A000C3B106F1FF3C0B44A44411F8014B0CF8D3
:1047B000014F9942F9D144683244551BECD0621E36
:1047C0005C1913F8011B02F8011FA342F9D1C5605F
:1047D00070BC70470B46EFE710B5124C124A1349F4
:1047E000A2610320206160611148E0614FF48060A4
:1047F000206210486066102000232266A066042212
:10480000E01DA3626362E3622367E366636713F0FC
:10481000C7FE094B93E803002022A2712060A1800B
:1048200010BD00BF14D3012044C8010850C80108BE
:10483000BCD30120BCD7012054C8010838B5204B97
:1048400000EB400403EBC40E0130DEF82C4000EB1B
:104850004000012C8C46154603EBC00005D0022C0D
:1048600029D0ACB10024204638BDDEF82830DEF86F
:10487000242093429CBFDEF820401B19013B9C1A68
:10488000AC4228BF2C462246FFF774FF204638BDB5
:10489000DEF82830DEF8242093429CBFDEF820109A
:1048A0005B18013B9B1A9D42DDD82A466146FFF703
:1048B00061FF2C46D7E7BDE83840FFF72DBF00BFAA
:1048C00014D3012070B5054682B008460C4613F09B
:1048D000A7FF0B4B1B7802466BB1EFF311864FF02D
:1048E000200181F3118821462846FFF7A7FF86F3B0
:1048F000118802B070BD0190FFF76EFF019AECE7DE
:1049000014D301202DE9F041194D1E462B780446A1
:104910008846174633B32B69A34226D9EFF3118398
:104920004FF0200181F3118854B92046044405EB6F
:10493000C405069AEA6283F311880020BDE8F0817D
:10494000601C00EB4000C00004EB440205EBC20217
:1049500045F800802844002147601662600091629B
:104960005162E3E7FFF738FFD5E74FF0FF30E5E7A7
:1049700014D30120FFF730BFFEE700BF38B50E4A61
:104980000E4B12781B6805464FF47A70B0FBF2F0BC
:10499000B3FBF0F000F0A8F8044608B90F2D01D9D8
:1049A000012038BD024629464FF0FF3000F040F8A4
:1049B000034B20461D6038BDC4000020CC00002001
:1049C000C8000020034A044B11681B780B44136095
:1049D000704700BFCCD70120C4000020014B1868ED
:1049E000704700BFCCD7012038B50446FFF7F6FF6B
:1049F000631C054602D0044B1B781C44FFF7EEFFF6
:104A0000431BA342FAD338BDC40000200749CA683B
:104A100003024FF6FF0003F4E0630240134343F048
:104A2000BF6343F40033CB60704700BF00ED00E08C
:104A30001C4BDB68C3F3022300B5C3F1070EBEF1C4
:104A4000040F03F1040C28BF4FF0040EBCF1060F55
:104A50001BD9033B4FF0FF3C0CFA03FC22EA0C028B
:104A60004FF0FF3C0CFA0EFC21EA0C0199400028A3
:104A700041EA02010CDB00F16040090100F56140F0
:104A8000C9B280F800135DF804FB00221346E7E783
:104A9000054B00F00F0009010344C9B219765DF817
:104AA00004FB00BF00ED00E0FCEC00E0002808DDA6
:104AB0004109044A00F01F00012303FA00F042F804
:104AC0002100704700E100E0002809DD43090549A5
:104AD00000F01F000122203302FA00F041F8230009
:104AE000704700BF00E100E00138B0F1807F10B4F2
:104AF0000FD24FF0E023094C58614FF0F00C84F8CE
:104B000023C00022072110469A615DF8044B196109
:104B1000704701205DF8044B704700BF00ED00E0D6
:104B20004FF0E022042813690CBF43F0040323F084
:104B300004031361704700BF38B50446FFF74EFF0A
:104B40000546002C66D02368022284F835201A68B6
:104B5000002122F0010284F834101A6005E0FFF70A
:104B60003DFF431B052B39D823681A68D107F6D4BB
:104B7000A0686268E168256902430A436169A06927
:104B80002A430A43E1691D6802430A433349294025
:104B9000256A2A430A43616A042926D01A605A69A1
:104BA00022F007021143D8B22D4A59611038A2FBF6
:104BB000005212092B4923F47F73895CE16523F0CD
:104BC00003035F2888BF04333F228A40A365002087
:104BD0009A600123606584F8353038BD03232022B4
:104BE0006265184684F8353038BDE56A216B294383
:104BF0000A431A605969A26A21F00701114341F082
:104C00000401002DCFD038B9012A23D032F002029E
:104C1000C9D108E0012038BDB0F5005F0CD0022AF0
:104C200003D9032ABFD1EA01BDD501234022626521
:104C3000184684F8353038BD032AB4D801A050F89E
:104C400022F000BF2B4C0008274C00082B4C00081A
:104C5000554C0008B5F1C07FA5D1E6E73F8010F0C4
:104C6000ABAAAAAA5CC8010870B490F83440856D5C
:104C7000012C35D090F835404FF0010C644580F898
:104C800034C005D0002380F8343070BC0220704757
:104C9000022680F83560046800264665266826F4FA
:104CA0008026266063608368402B0EBFA260A160EF
:104CB000E260C26D08BFE1603F239340AB602368B0
:104CC000026C43F0160323601AB1236843F0080313
:104CD0002360236843F001030020236070BC704709
:104CE000022070BC704700BF70B50446866DFFF7A8
:104CF00075FE94F83530022B054606D0802200233D
:104D0000626584F83430012070BD23681A6822F08F
:104D100016021A605A6922F080025A61226C32B37C
:104D20001A6822F008021A601A6822F001021A605A
:104D300005E0FFF753FE431B052B0FD823681B68C4
:104D400013F00103F5D1E16D3F228A400121B260E9
:104D5000184684F8343084F8351070BD03202022C2
:104D60000023626584F8343084F8350070BDA26C8D
:104D7000002AD5D1D8E700BF90F83530022B03D0F8
:104D800080234365012070470268052380F8353091
:104D9000136823F001030020136070472DE9F041F0
:104DA00082B0744A866D156800230193C36D346820
:104DB00008229A402242804604D001680F68780792
:104DC00000F18A8001229A40224204D0D8F80010D3
:104DD0004969090678D404229A40224204D0D8F8BE
:104DE000001009688F0767D410229A40224204D02D
:104DF000D8F800100F68380749D420229A40224280
:104E000017D0D8F800100C68E00612D5B26098F8F8
:104E10003520052A73D00B6813F4802F0B6800F03F
:104E20009080190340F19B80D8F83C300BB140468C
:104E30009847D8F854303BB3D8F85430DA071BD52C
:104E4000D8F800204C49052388F835301368A1FBB9
:104E5000051523F00103AD0A136002E01368DB07B8
:104E600004D5019B0133AB420193F7D90022012302
:104E700088F8342088F83530D8F84C3023B14046D3
:104E800002B0BDE8F041184702B0BDE8F081B26061
:104E90000A6812F4802F0A682AD1D70503D40A6859
:104EA00022F008020A60D8F84020002AA5D0404627
:104EB0009047D8F85C30A0E7B260D8F8542042F0B0
:104EC0000402C8F854208FE7B260D8F8542042F0AA
:104ED0000202C8F854207EE70F6827F004070F602D
:104EE000B260D8F8542042F00102C8F8542069E7B3
:104EF0001203D8D5D8F84820002AD8D17DE70A680F
:104F000022F016020A604A6922F080024A61D8F84B
:104F1000402052B30A6822F008020A603F2202FAD7
:104F200003F3D8F85010B3600022012388F834202E
:104F300088F835300029A7D0404602B0BDE8F041DE
:104F4000084713F480737FF46FAF0A6822F01002F1
:104F50000A60012288F8343088F8352064E7D8F8F0
:104F60004430002B7FF463AF63E7D8F84820002A71
:104F7000D0D1D3E7CC000020B5814E1B90F835008E
:104F8000704700BF2DE9F04F00220D68DFF830A216
:104F900085B0134605E00133102B02F1020200F048
:104FA0009B8001249C4005EA040BAC43F3D14F687D
:104FB00027F0100E0EF1FF34012C40F29080D0F853
:104FC0000CE08C684FF0030C0CFA02FC94402EEAC3
:104FD0000C0E44EA0E04C4606FEA0C04D0F800C062
:104FE0000CEA040C07F00304944044EA0C04046047
:104FF000FC00D0D500240394DAF84440694E44F410
:105000008044CAF84440DAF8444004F480440394ED
:10501000039C23F0030404F1804404F59C3403F062
:10502000030ED4F808804FEA8E0E4FF00F0C0CFAE6
:105030000EFCB04228EA0C0C1FD006F58066B04288
:1050400000F08D80584EB04200F09080574EB04234
:1050500000F09380564EB04200F09680554EB0421C
:1050600000F09980544EB0420CBF4FF006084FF04C
:10507000070808FA0EFE4CEA0E0CC4F808C04F4CA4
:1050800024686FEA0B0CFE034C4E54BF0CEA040478
:105090004BEA040434607468BE03484E54BF0CEA03
:1050A00004044BEA04047460B468FE02434E54BF27
:1050B0000CEA04044BEA0404B460F4680133BE0251
:1050C0003E4E54BF0CEA04044BEA0404102BF46077
:1050D00002F102027FF465AF05B0BDE8F08FD0F8B1
:1050E00008C0CC688E684FF0030909FA02F92CEA6F
:1050F000090C944044EA0C048460446824EA0B0CD4
:10510000C7F300149C4044EA0C044460C46806FAE7
:1051100002FC24EA09084CEA080CBEF1020F6FEA0F
:105120000904C0F80CC07FF459AF4FEAD30E00EB6E
:105130008E0E03F00708DEF8206001960E694FEA34
:10514000880806FA08FC4FF00F09019E09FA08F8D2
:1051500026EA08094CEA090CCEF820C03EE74FF0D9
:10516000010808FA0EFE4CEA0E0C86E74FF0020822
:1051700008FA0EFE4CEA0E0C7FE74FF0030808FA1F
:105180000EFE4CEA0E0C78E74FF0040808FA0EFE0B
:105190004CEA0E0C71E74FF0050808FA0EFE4CEAD7
:1051A0000E0C6AE70000024000080240000C0240BA
:1051B000001002400014024000180240003C014070
:1051C000003802400369194214BF012000207047D3
:1051D00002B9090481617047436931EA030308BFDA
:1051E00009048161704700BF704700BF044A5169DC
:1051F000014208B500D108BD5061FFF7F5FF08BDB9
:10520000003C01402DE9F8430D46814617461E46F5
:105210004FEA1148D9F8002001E0731C13D1B8F10E
:10522000010F0BBF5369946925EA030C25EA040CAE
:105230001FFA8CFCBCFA8CFC4FEA5C1CBC45ECD021
:105240000020BDE8F883FFF7C9FB089BC01AB042F5
:1052500001D8002EDED100222023C9F8302089F8A1
:105260003D3089F83E20D9F8403089F83C2043F0A1
:105270002003C9F840300120E3E700BF2DE9F843DF
:1052800081460E4617469846D9F8005004E06C69EE
:1052900062050AD47B1C22D16C6926EA0404A4B2FC
:1052A000002CF4D12046BDE8F8832B6843F400734A
:1052B0002B6000226FF4806120236961C9F83020DF
:1052C00089F83D3089F83E20D9F8403089F83C20F3
:1052D00043F00403C9F840300120BDE8F883FFF72C
:1052E0007DFBA0EB0800B84201D8002FCCD10022F2
:1052F0002023C9F8302089F83D3089F83E20D9F8BC
:10530000403089F83C2043F02003C9F840300120A8
:10531000C9E700BFF8B506460D46174608E06269C2
:10532000D2061BD4FFF75AFBC01BA84207D835B1E1
:105330003468636913F04003F1D00020F8BD002207
:105340002023326386F83D3086F83E20336C86F8A1
:105350003C2043F0200333640120F8BD6FF01001BE
:1053600020226161336386F83D2086F83E30326C3E
:10537000326486F83C300120F8BD00BFF8B5054620
:105380000E4617462C6801E0731C19D1636913F0AF
:10539000800313D160694205F6D56FF48061202245
:1053A00061612B6385F83D2085F83E302A6C85F8D5
:1053B0003C3042F004022A640120F8BD0020F8BD10
:1053C000FFF70CFBC01BB04201D8002EDAD100223F
:1053D00020232A6385F83D3085F83E202B6C85F824
:1053E0003C2043F020032B640120F8BDF8B50546AE
:1053F0000E4617462C6801E0731C19D1636913F03F
:10540000040313D160694205F6D56FF48061202250
:1054100061612B6385F83D2085F83E302A6C85F864
:105420003C3042F004022A640120F8BD0020F8BD9F
:10543000FFF7D4FAC01BB04201D8002EDAD1002207
:1054400020232A6385F83D3085F83E202B6C85F8B3
:105450003C2043F020032B640120F8BD2DE9F04FE0
:10546000056883B099462B680C9EDDF834A043F4A0
:10547000807307468B4690462B606C69E10720D508
:105480000BF0FE032B613149534632463846FFF795
:10549000F5FE20BB3B680190596901919B6901931E
:1054A000524631463846019BFFF768FFA0B9B9F173
:1054B000010F3B6833D15FFA88F21A6103B0BDE88F
:1054C000F08F721CD9D0FFF789FAA0EB0A00864250
:1054D00009D346B13D68D0E73B6C042B2ED00120A8
:1054E00003B0BDE8F08F002320223B6387F83D2006
:1054F00087F83E303A6C396842F020023A640A6814
:1055000087F83C30D30506D54FF4007303203B6485
:1055100003B0BDE8F08F032003B0BDE8F08F4FEA81
:1055200018201861524631463846FFF727FF0028F9
:10553000D2D13A685FFA88F31361D1E73A68136809
:1055400043F4007301201360CAE700BF02000100AA
:105550002DE9F0479946036890461A6842F4806244
:105560001A601A6884B042F480720C9D0D9F1A6014
:1055700006468A465C69E00744D50AF0FE021A61D5
:1055800043493B462A463046FFF778FE5FFA8AFADF
:10559000002844D133680390596903919B690393B0
:1055A0003A4629463046039BFFF7E8FE002833D1F0
:1055B000B9F1010F4FD133685FFA88F21A613A46A8
:1055C00029463046FFF7DAFE30BB024630680168F4
:1055D00041F4807101602B4600974FF00111304675
:1055E000FFF710FE00284DD1326829494AF0010327
:1055F000136130463B462A46FFF740FE003818BF8D
:1056000001200DE0691CB5D0FFF7E8F9C01B854209
:1056100009D345B13368ADE7336C042B2BD001209F
:1056200004B0BDE8F08700232022336386F83D20D4
:1056300086F83E30326C316842F0200232640A68EB
:1056400086F83C30D20502D54FF400733364032052
:1056500004B0BDE8F08733684FEA18221A61294682
:105660003A463046FFF78AFE0028D5D132685FFA05
:1056700088F31361A3E73268136843F400730120D1
:105680001360CDE733681B68DB05E0D5DCE700BFBE
:1056900002000100704700BF70B50446002800F00A
:1056A0009D8090F83D3003F0FF02002B00F09880C1
:1056B0002368242284F83D201A6822F001021A602F
:1056C0001A6842F400421A601A6822F400421A6012
:1056D00001F092FE63684E4A93424FD84D4A904281
:1056E0007CD94D4D5A00A5FB0035431EB3FBF2F3A8
:1056F0002268506820F03F0040EA95405060A90CB5
:1057000001F1010C116A21F03F0141EA0C01116223
:10571000D16940F6FC7E013321F44F4113EA0E0FAC
:1057200021F0FF0161D104230B43D3611168206A8A
:10573000E36921F0C00103430B4313609168E06803
:10574000236921F40341034321F0FF010B439360DC
:10575000D168A069636921F0FF0103430B43D36063
:105760001168002341F0010120201160236484F8B6
:105770003D002363184684F83E3070BD274A9042AE
:105780002CD9254D264EA5FB002C2268556825F006
:105790003F0545EA9C4555604FEA9C414FF496759C
:1057A00005FB01F1A6FB0151156A890925F03F05AA
:1057B000013129431162D169A56821F44F4121F0DB
:1057C000FF01ADB9013803EB4303B0FBF3F3013341
:1057D000C3F30B03D3B143F40043A5E7012070BD2D
:1057E00080F83C20FFF756FF62E7C3F30B039BE70B
:1057F00003EB8303013803EB8303B0FBF3F30133C3
:10580000C3F30B0313B143F440438DE701238BE74C
:10581000A08601007F841E0083DE1B43FF083D003D
:10582000D34D6210704700BF10B50446A0B10268A6
:10583000242380F83D30136823F001031360FFF741
:10584000F1FF0023236484F83C3084F83D3018468F
:10585000236384F83E3010BD012010BD2DE9F04FC8
:10586000044683B09946BDF834A00E9E0F4690467C
:10587000FFF7B4F894F83D30202B054608D00220FD
:1058800003B0BDE8F08FFFF7A9F8401B192874D8C2
:10589000206883696FEA030C1CF0020BF3D094F8C4
:1058A0003C30012BEBD003680122DB0784F83C205D
:1058B00071D53946076827F4006707600C98606265
:1058C00021200195009684F83D00402084F83E0098
:1058D00000202064A4F82AA0608D20853548E0626D
:1058E0004B4642462046FFF7B9FD002841D1238DA3
:1058F000002B2BD02A4631462046FFF73FFD0028DB
:105900004DD1676A2068B4F828C039460CF1FF32DF
:1059100011F8013B0361638D013B9BB26385D0F8B5
:1059200014E0616293B21EF0040F23850CD06BB1BA
:105930007A780261628DACF10203013A9BB20237C0
:1059400092B2676223856285002BD3D12A46314605
:105950002046FFF74BFD10BB22681368202143F45B
:105960000073136084F83D1084F83C0084F83E0016
:1059700086E7012003B0BDE8F08F2023C4F830B0E3
:1059800084F83D3084F83EB0236C84F83CB043F09A
:105990002003236473E703681343036089E7236CE0
:1059A000042BE6D12268136843F4007301201360CE
:1059B00066E700BF0000FFFF2DE9F04F044687B007
:1059C0009946BDF844A0129E0F469046FFF706F890
:1059D00094F83D30202B05460AD04FF0020840468F
:1059E00007B0BDE8F08FFEF7F9FF401B19284AD831
:1059F000206883696FEA030C1CF0020BF3D094F863
:105A00003C30012BE9D003680122D90784F83C20FF
:105A100047D53946076827F4006707601098606229
:105A200022200195009684F83D00402084F83E0035
:105A300000202064A4F82AA0608D20858448E062BC
:105A400042464B462046FFF783FD8046A8B9238D8A
:105A50005BBB236802905A6902929A690292029A89
:105A60001A6842F400721A600023202284F83D2054
:105A700084F83C3084F83E30B1E74FF001084046EE
:105A800007B0BDE8F08F2023C4F830B084F83D3073
:105A900084F83EB0236C84F83CB043F020032364C8
:105AA0009BE7036813430360B3E7012B00F0BF805B
:105AB000022B00F08480226805905169059192695B
:105AC0000592059A634F032B4DD8012B00F0A2805D
:105AD000022B009533464FF00002394620467ED017
:105AE000FFF790FB02460028C7D12368196821F40C
:105AF000806119601969636A1970616A638D013187
:105B00006162013B218D9BB263854B1E2385394623
:105B1000009533462046FFF775FB0028ADD123687A
:105B2000616A1A6842F400721A601B690B70638D17
:105B3000626A2168013B9BB26385531C09696362F9
:105B4000238D013B23855170238D628D616A013B5A
:105B5000013A01319BB292B2616223856285002BCA
:105B600082D0032BB1D92A4631462046FFF7D2FB1B
:105B7000002882D12268636A12691A70628D2068D7
:105B8000238D616A013A92B262854269013B9BB200
:105B900001F1010C52072385C4F824C0DFD5036945
:105BA0004B70628D238D013A92B26285626A013B2D
:105BB0009BB2013223856262002BD2D154E7226866
:105BC000116821F480611160116841F40061116075
:105BD00004905169049192690492049A72E7FFF764
:105BE00011FB00287FF449AF2368616A1A6842F408
:105BF00000721A601B690B70638D626A013B9BB275
:105C00006385238D013B23852368511C1B696162D9
:105C10005370C6E72A4631462046FFF77BFB002833
:105C20007FF42BAF23681A69636A1A70B9E7226898
:105C3000116821F4806111600390516903919169A9
:105C400003910399116841F4007111603AE700BFB4
:105C50000000FFFF04000100704700BF704700BF55
:105C6000704700BF704700BF704700BF704700BF5C
:105C7000704700BF90F83D20016D10B50346D2B2C9
:105C800059B9C26C0168012A826C29D0C2F307227B
:105C90000A61026D0132026510BD016D012925D036
:105CA000016D0229F8D1222A2CD0418D89B229BB5D
:105CB000418D89B20029EFD1212AEDD102685468C3
:105CC00024F4E0645460146844F4007414602022E6
:105CD000016380F83D2080F83E10FFF7C9FF10BD3A
:105CE000D2B20A61026D0232026510BD826C016897
:105CF000D2B20A61026D0132026510BD212A07D0BD
:105D00005B8D10BD0268136843F48073136010BD8F
:105D1000416A026811F8010B10615A8D5962013A0B
:105D200092B25A8510BD00BF704700BF704700BFD8
:105D3000704700BF70B53A4B3A491B68806B82B020
:105D4000DB080022A1FB031301921B0A90F83D100F
:105D5000026803EB8303C3EBC303C9B2019305E0FD
:105D6000019B013B019313689B0506D5019B002B0A
:105D7000F6D1036C43F020030364446B4CB3836B94
:105D80000025E563F3B11668DD6326F480661660CE
:105D90004585256500241C65136823F00103136005
:105DA00090F83D30602B2AD001F02801282919D025
:105DB0002022002380F83D2080F83E30FFF7B6FF18
:105DC00002B070BD156825F48065156043852365B4
:105DD000E2E7836BF3B11568DC6325F48065156039
:105DE0004485D7E7136843F0010313601368002468
:105DF00043F480631360046380F83D10DEE7002302
:105E0000202280F83D2080F83E300364FFF790FFA9
:105E100002B070BD146824F4806414604385BBE74D
:105E2000CC00002089B5F81490F83D2090F83E3061
:105E3000102B10B5D2B20446D9B238D0402936D092
:105E400002F0280128293DD023685968080507D4A5
:105E5000602A05D02021002284F83D1084F83E20DD
:105E6000002222635A6812F4006234D194F83D1083
:105E7000602975D05A69500605D5626A1B6913708E
:105E8000636A013363622046FFF750FF236C1907F2
:105E900004D02268536823F4E063536094F83D30E3
:105EA000226C5207DBB201D5282B2FD010BD222A3D
:105EB000C6D123681A6822F400621A605A68120573
:105EC000C8D5CDE700232363236884F83D105A68C2
:105ED00012F40062CAD05A68606B22F400625A6001
:105EE00090F83530012B1ED0284B0365FEF744FF98
:105EF0000028CBD02268606B1368202123F00103B7
:105F00001360036D84F83D109847BFE700232049D4
:105F1000E16220222363204684F83D2084F83E304D
:105F2000FFF7A4FE10BDA06B184B0365FEF724FF1E
:105F30000028ABD023685A69510606D5626A1B69EE
:105F40001370626A2368013262621A68A06B22F0E1
:105F5000010220211A60036D84F83D10984795E7EF
:105F6000202184F83D1022645A69520606D5626ADF
:105F70001B691370626A2368013262621A6822F038
:105F8000010220461A60FFF7D3FE7FE7355D000867
:105F90000000FFFF70B5036804465868E56A94F88E
:105FA0003E1094F83D2010298CB0D2B25FFA81FCEB
:105FB00021D0BCF1400F1ED0216C002900F093804D
:105FC0005969002511F0020FC1F3400656D086052D
:105FD00056D5226C02B19D6994F83D2002F028024A
:105FE000282A00F021826FF002010022596184F812
:105FF0003C200CB070BD99695A69D6071AD4B5F522
:106000002A0FF6D0B5F12A4FF3D016076ED58505C5
:1060100040F18480626C616BD2B21A61002900F099
:10602000F081CA6B002A00F0F1815A6842F40062E4
:106030005A60DEE785056FD5E26AB2F52A0F00F0F7
:10604000EE81E26AB2F12A4F04BF0822E26294F8BC
:106050003E20402A00F0DC812269B2F5804F00F03A
:10606000B081226D002A40F0F381626CC2F3C81245
:1060700002F0060242F0F0021A61BAE7CD067CD4C3
:1060800002F0F702212A00F0F5804E0640F132813D
:10609000450540F12F81490700F12F8194F83D100B
:1060A000628D92B2C9B2002AA3D0626A1B691370D2
:1060B000638D626A013B9BB26385638D01329BB243
:1060C0006262002B95D12A2993D122685368222538
:1060D000282123F4806353602046256384F83D1013
:1060E000FFF7C0FD85E79D6959696BE7960715D5F0
:1060F000850513D594F83E20E06A256B94F83D1091
:106100002229D2B200F0B781002209925A6909927D
:106110009B690993099B6CE71507E7D511F0040FFC
:10612000596800F0F38009053FF563AF160640F1AA
:106130001381450540F11081510700F1108194F859
:106140003D20208D94F83E10E56AD2B2C9B20028F5
:1061500040F03E82212A00F02F8340297FF449AF8E
:10616000222A7FF446AF628D92B2002A40F0AD82BF
:106170005A6822F480625A603BE7850580D594F81E
:106180003D505A6822F4E0625A600B965A690B92AD
:106190001A6842F001021A600B9A1A6822F48062AF
:1061A0001A605A681105EDB221D505F0F702222ACE
:1061B00000F07E81606B0268526892B26285628DE7
:1061C00092B21AB1226C42F0040222645A6822F49C
:1061D00000625A60FEF7D2FE012808D0606B914B36
:1061E0000365FEF7C9FD10B1606B036D9847638DC1
:1061F0009BB213B323685A6952070AD5626A1B69B6
:106200001370628D636A013A591C92B2236861620D
:1062100062855A69560609D5626A1B691370638DD7
:10622000626A013B01329BB262626385638D9BB2FD
:106230001BB1236C43F004032364236C002B40F058
:10624000DA802A2D00F0628194F83D30282B00F08E
:106250005081236B222B02D0222D7FF4CAAE002363
:1062600020222363204684F83D2084F83E30FFF747
:10627000F9FCBEE60D0628D5460526D54D0727D4E0
:1062800094F83D00618D89B2C0B200293FF4B1AEEF
:10629000616A11F8015B1D616162618D013989B22A
:1062A0006185618D89B200297FF4A3AE29287FF42E
:1062B000A0AE5968282521F48061596020462263E8
:1062C00084F83D50FFF7CCFC93E649077FF591AE8B
:1062D00082057FF58EAE628D92B2002A3FF489AEC0
:1062E000626A12F8011B1961638D6262013B9BB205
:1062F00063857EE64A077FF57CAE86057FF579AE3D
:10630000628D92B2002A3FF474AE1AE00D053FF59B
:1063100070AE510630D451077FF56BAE82057FF524
:1063200068AEE16A628D92B2042A00F04281628D09
:1063300092B2032A00F05E81628D92B2022A00F0CE
:106340008A81626A1B691370638D626A013B013244
:106350009BB2626263854CE652077FF54AAE8605C2
:106360007FF547AEBCF1100F00F0FF8020460CB067
:10637000BDE87040FFF77EBC4605CCD55507C2F39B
:106380008001CBD494F83D20222A7FF432AE628D76
:1063900092B2032A40F29F81626A1B691370638D77
:1063A000626A013B9BB26385638D9BB20132032B12
:1063B00062627FF41EAE2268536823F480635360E8
:1063C00017E694F83D20212A626C16BF42F00102C4
:1063D00002F0FE02D2B21A61626B1AB1D26B002ACD
:1063E0007FF423AEA26B002A3FF403AED26B002AE7
:1063F0007FF41BAEFDE520460CB0BDE87040FFF712
:1064000013BDA26B002A7FF40CAEF2E5A26BEDE7A0
:10641000226D52BB626C02F0FE021A61E9E50122B4
:10642000E26214E6355D00085A6822F480625A6020
:106430002E0685F004014FF0000354BFA289228B81
:1064400084F83C30C1F380012046FFF70DFCD0E515
:10645000226D012A7FF4CDAD626CC2F3C81202F046
:10646000060242F0F1021A61C3E5626C42F00102D9
:10647000D2B21A61BDE5216D11B9402A00F0A180A8
:10648000226D22B92169B1F5404F00F0A580628DDF
:1064900092B2002A42D102925A6902929A690292F9
:1064A000029A1A6842F400721A6000232365A0E57C
:1064B000A06B0268526892B26285628D92B21AB184
:1064C000226C42F0040222645A6822F400625A608C
:1064D000FEF754FD01283FF48AAEA06B9A4B03658A
:1064E000FEF74AFC00283FF482AEA06B036D98478C
:1064F0007DE600239549E16220222363204684F84B
:106500003D2084F83E30FFF7B1FB72E5282223637B
:10651000204684F83D20FFF7A5FB95E6628D92B2F8
:10652000012A76D0628D92B2022A00F017811A6891
:1065300042F480621A605A6815050ED510F5803F46
:1065400007D001381F2808D8814A22FA00F0C00776
:1065500003D55A6842F480525A60002208925A6960
:1065600008929B690893089B9FE7E16A94F83D2095
:10657000212A7FF43EAD628D92B2002A7FF4B0AE44
:10658000082900F06181202900F05E8111F5803F2B
:1065900000F05A81596821F4E061596011202023EC
:1065A000206384F83E20204684F83D30FFF754FBFA
:1065B0001FE55A68616A22F480625A601B690B7099
:1065C000C2E600915A6900929B690093009B10E516
:1065D000212A3FF4C8ADC0E501925A6901929A6937
:1065E0000192019A1A6842F480721A60236D013395
:1065F0002365FEE45A68042922F480625A603FF45D
:10660000A0AE02293FF49DAE1A6822F480621A609F
:1066100097E610F5803F00F00381082800F0BC8069
:10662000202800F0B980122D00F05181102800F2CE
:106630005181484A22FA00F0C60740F14B811A689E
:1066400042F480621A60002205925A6905929B69A1
:106650000593059B29E701291A6800F0C4801029D9
:1066600000F0C180042900F02381022900F020817C
:1066700042F400721A60626A1B691370638D626A69
:106680002168013B9BB263850B69511C61625370A9
:10669000638D2168626A013B9BB263854B6801325E
:1066A00023F44073202062624B6084F83D0094F82C
:1066B0003E30402B00F0DC800022122384F83E2084
:1066C00020462363FFF7CAFA93E494F83E20402A59
:1066D0007FF406AE4AE6E06A02283FF48AAC012A5B
:1066E0003FF687AC1C4A0A91126846F2A810B2FB2A
:1066F000F0F202EB82020A9204E01A6812F40072CD
:1067000000F0ED800A9A013A0A920A990029F4D120
:10671000226C606A42F0200222645A6822F4E0622D
:106720005A601B690370638D626A013B01329BB240
:1067300020206385626284F83D00204684F83E1084
:10674000FFF7F4FA55E400BF355D00080000FFFFD5
:106750008180008014000100CC000020102840F24D
:1067600090801A6822F480621A601A6842F400620B
:106770001A605A68110507D510F5803F40F08E80E9
:106780005A6842F480525A60002207925A6907926E
:106790009B690793079B88E61A68002122F48062B0
:1067A0001A6006915A6906929A690692069A1A68C0
:1067B00042F400721A6078E6082D18D0202D16D009
:1067C00015F5803F13D05A6822F4E0625A60112018
:1067D00000212023206384F83E10204684F83D30B9
:1067E000FFF73AFA05E422F480621A6043E7596839
:1067F00021F4E061596019680022202041F4007101
:106800001960226384F83D0094F83E3084F83E20FD
:10681000402B20467FF4CAAEFFF72AFAFFF7E9BB08
:106820001A6822F480621A605A6812F4006243D037
:106830001A68002122F480621A6003915A69039257
:106840009B690393039B30E65A6822F4E0625A6026
:106850001A680021202542F400721A602046216344
:1068600084F83D5084F83E10FFF7F6F9FFF7C1BBFE
:10687000002384F83E3020462363FFF755FAFFF7E4
:10688000B8BB284AC240D5077FF56BAF1A6842F4FF
:1068900080621A605A6812057FF576AF01381F28AA
:1068A0003FF672AF204AC240D6077FF56DAF67E76B
:1068B00042F480621A60DEE604925A6904929A6990
:1068C0000492049A1A6842F400721A60EDE50128F5
:1068D0007FF462AF1A6822F480621A60B3E6196826
:1068E000606A21F480611960596821F4E06159609F
:1068F0001B690370638D013B20219BB2638584F883
:106900003D10636A94F83E100133402963627FF4BE
:10691000D4AE84F83E2020462263FFF705FAFFF745
:1069200068BB00BF140001008180008030B503689F
:106930005C695A6890F83E10E50583B05FFA81FC07
:1069400033D5D1054FEA122E2FD56FF480725A61DC
:10695000A2053CD4620572D50121428D90F83DE03C
:10696000056BBCF1200F92B25FFA8EFE3DD06FF442
:106970008062BCF1100F41F004015A6102D0BCF1F9
:10698000400F03D11A6842F400721A60220504D540
:106990006FF4006241F008015A61036C194301640D
:1069A00003B0BDE83040FFF73FBAA50503D5D105D8
:1069B0004FEA122E17D46505C4F3802103D42405B1
:1069C00034D403B030BDD105FBD50021C5E7032188
:1069D0006FF400725A616205BFD42405DDD51EF044
:1069E000010FD5D1D9E70221F2E7CAB90EF0F702BB
:1069F000212A04D0BEF1280F12D1212D10D190F8F8
:106A00003D20C56A082DD2B21ED0202D1CD0212ACF
:106A100037D06FF480625A6125050CD50368B7E75B
:106A20006FF480625A6141F00401AFE74FEA122E21
:106A30001EF0010FACD10029AFD103B030BD250548
:106A40004FF00101F4D4A8E7282AE0D11A4AC26223
:106A50005A68019122F4E0625A606FF480625A61D0
:106A60001A68009022F480621A60002320220363D7
:106A700080F83D2080F83E30FFF7F8F8DDE90001AE
:106A8000CAE70D4DC5620263202280F83D20002236
:106A900080F83E205A68019122F4E0625A606FF457
:106AA00080625A611A68009022F480621A60FFF7CF
:106AB000D7F8DDE90001AFE70000FFFF90F83D00E7
:106AC000704700BF10B40D4C0D4A236823F0030338
:106AD000184320601369012943F0040313610AD0AD
:106AE00040BF20BF20BF064A5DF8044B136923F066
:106AF00004031361704730BFF5E700BF007000402A
:106B000000ED00E0F0B44D6A35B1B2F1406F03D052
:106B10008B6A0468013B23618B691BB30C6A002CF0
:106B200047D00068CE698F68C761002E60D02B43C4
:106B300013432343CC6A334323430C6B23434C6BF3
:106B400023430C692343CC6823430C6823434C69DB
:106B5000B2F1406F43EA844343615CD04B68836188
:106B6000F0BC70470B6A93B10068CE698C68C46151
:106B70002B43002E62D0CC6A1343334323430C6B68
:106B800023434C6B23430C692343CC68DEE7CB697A
:106B9000002B62D1002D3ED0CB6A0C6B00682B43DA
:106BA000134323434C6B4A69234343EA82434361C3
:106BB00031E0CC6945EA030C002C2ED04CEA020CE3
:106BC0004CEA040CCC6A03684CEA04000C6B2043CA
:106BD0004C6B2043CC6820430C6820434C69B2F1D5
:106BE000406F40EA8440586115D04A689A6112E0CB
:106BF00045EA030C4CEA0203CA6A0D6923430C6B95
:106C000013434A6B234313430C684A692B432343C2
:106C100043EA82434361F0BC7047CC6A4CEA02030A
:106C200023430C6B4A6B23430C684969134323438A
:106C3000026843EA8143F0BC53617047CC6A134356
:106C400023430C6B4A6B23430C6913434A69234368
:106C500043EA8243F0BC436170472B43CD6A0C6B1F
:106C6000006813432B4323434C6B8DE7704700BFF1
:106C700070B50446FDF7B2FE0646002C4CD094F8E1
:106C8000413003F0FF02002B3DD0A56C2168A268C3
:106C90000B68013A23F4F85343EA02230B608B6834
:106CA00013F0200325D1E669E268256A08683243BB
:106CB0002A436568A66920F07F4042EA056220F019
:106CC000D00002430A6062694D6818483243266961
:106CD000284042EA064202434A600A6801252A43E4
:106CE0000A601846636484F84150002384F84030F9
:106CF00070BD6B1CD3D0FDF771FE801BA8420DD870
:106D000065B12168CBE784F84020204641F2883500
:106D1000FFF7ACFFA564B9E7012070BD042384F838
:106D20004130636C012003436364DEE7FEF8E0FF5B
:106D3000704700BF10B5044670B10268136823F0B5
:106D400001031360FFF7F4FF00236364184684F81F
:106D5000413084F8403010BD012010BD2DE9F843CA
:106D600005460F461646FDF739FE95F84030012BD3
:106D7000804638D0012385F8403095F84130012B0A
:106D80005FFA83F907D04FF00209002385F84030FD
:106D90004846BDE8F88300236B64022385F8413040
:106DA0002A68946814F020040BD1224639462846FC
:106DB000FFF7A8FE7B6A2BB3012385F84130A1467B
:106DC000E3E7701CEDD0FDF709FEA0EB080086425A
:106DD00001D3002EE4D1042385F841306B6C43F0DD
:106DE00001036B64D1E74FF002094846BDE8F88320
:106DF000731C08D0FDF7F2FDA0EB08008642EAD331
:106E0000002EE8D02A6893689907F1D50221012362
:106E1000D1604FF0000985F84130B6E72DE9F84F11
:106E200006461F468A469346FDF7D8FD96F8403041
:106E3000012B80465FD0012386F8403096F8413020
:106E4000012B5FFA83F907D04FF00209002386F87F
:106E500040304846BDE8F88F00237364422386F82B
:106E600041303568AB689C0628D4DBF80030AB6253
:106E7000DBF804306B62DBF80830EB622C68DBF87F
:106E8000103024F4400C4CEA030C4CF48002DBF884
:106E90000C302A6051464FF00062CAF82830304664
:106EA000FFF730FE32689368190712D508210123D5
:106EB000D1604FF0000986F84130C7E7781CD1D087
:106EC000FDF78CFDA0EB080087420CD3002FC8D142
:106ED00009E07B1CE7D0FDF781FDA0EB08008742AD
:106EE00001D3002FDED1042386F84130736C43F0C8
:106EF00001037364AAE74FF002094846BDE8F88F22
:106F000070B50446FDF76AFD94F8412012F00202C4
:106F100006461CD00022236884F840201A685507D2
:106F20002BD41A68A56C42F002021A609A68900786
:106F30000FD50222A56CDA609A6812F0200212D1F5
:106F40005969012021F04061596184F841001046DF
:106F500070BD691CEAD0FDF741FD801B85421CD342
:106F6000DDB12368E2E76A1CE6D0FDF737FD801B40
:106F7000854212D38DB12368DEE71A68E06B22F0F8
:106F800004021A60FDF7B0FE08B92368C9E7626C15
:106F9000236842F004026264C3E7042384F84130AA
:106FA000636C012213436364D1E700BF2DE9F8430A
:106FB000044689461646FDF711FD94F840302768CF
:106FC000012B054663D0012384F8403094F841300A
:106FD000012B5FFA83F807D04FF00208002384F8F2
:106FE00040304046BDE8F88300236364B9F1000FE8
:106FF00052D0122384F841303B690133E3623B698C
:10700000C4F824900133A3627B6923F040637B6161
:10701000E36A33B339468B685B070FD5636A1B7825
:1070200087F82030E16A636A0139E162E26A01337C
:10703000636252B321688B685B07EFD4701CEAD09F
:10704000FDF7CCFC401B864201D3002EF2D1042375
:1070500084F84130636C43F0010363640AE0731CFD
:107060000CD1BB689A07FAD50223FB602046FFF7D4
:1070700047FF8046012384F84130AFE7FDF7AEFCBF
:10708000401B8642E3D3002EE1D02768E9E74FF0AA
:1070900002084046BDE8F883636C43F0080363646C
:1070A0009CE700BF2DE9F843044616468946FDF7E4
:1070B00095FC2768BA6994F84030012B054668D0E2
:1070C000012384F8403094F84130012B5FFA83F8B3
:1070D00007D04FF00208002384F840304046BDE856
:1070E000F88300236364B9F1000F57D0222384F89A
:1070F00041303B690133A3633B69C4F830900133ED
:1071000063637B6923F0406343F080637B61BA6112
:10711000A36B43B339468B6813F0060F10D0236B73
:1071200097F820201A70A16B236B0139A163A26B21
:10713000013323635AB321688B6813F0060FEED135
:10714000701CE8D0FDF74AFC401B864201D3002E9C
:10715000F1D1042384F84130636C43F0010363648C
:107160000AE0731C0CD1BB689A07FAD50223FB60B6
:107170002046FFF7C5FE8046012384F84130AAE788
:10718000FDF72CFC401B8642E3D3002EE1D027689C
:10719000E9E74FF002084046BDE8F883636C43F02E
:1071A0000803636497E700BF70B50346224E88B0BA
:1071B0000D461446F0B90190326B42F00102326381
:1071C000326B059002F0010201924FF4807203923B
:1071D00002220199049219480793032203A90692F7
:1071E000FDF7D0FEB26822F0EC622A432243B2607F
:1071F00008B070BD00230293326B114842F00402C4
:107200003263326B059302F0040202924FF4007273
:10721000039202220299049203A903220793069281
:10722000FDF7B0FEB36823F0784343EA050141EA75
:10723000C401B16008B070BD0038024000000240D7
:1072400000080240014B0122DA6470470000474207
:10725000164908B58B6803F00C03042B1BD0082BD0
:1072600017D14A684B68496813F4800302F03F0263
:1072700013D10F48C1F38811A1FB000110F01AF8D7
:107280000A4B5B68C3F3014301335B00B0FBF3F0CF
:1072900008BD074808BD074808BD0648C1F3881166
:1072A0000023A1FB000110F005F8E9E700380240D7
:1072B0000024F40000127A002DE9F0410D46044646
:1072C00060B1454A136803F00F038B4209D2CBB279
:1072D0001370136803F00F038B4202D00120BDE846
:1072E000F0812368980714D5590704D53B498A686B
:1072F00042F4E0528A601A0704D538498A6842F499
:1073000060428A603549A0688A6822F0F002024330
:107310008A60DF0721D56268012A55D0931E012BB0
:107320002E4B1B684DD99907D8D52C4EB36823F046
:1073300003031343B360FDF751FB41F2883807465E
:1073400004E0FDF74BFBC01B404542D8B3686268C0
:1073500003F00C03B3EB820FF3D11F4A136803F061
:107360000F03AB4206D9EBB21370136803F00F039F
:10737000AB42B3D123685A0706D51849E0688A683A
:1073800022F4E05202438A601B0707D5134A2169A1
:10739000936823F4604343EAC1039360FFF758FF07
:1073A0000E4A0F4C92680F49C2F303120346A25CC7
:1073B0000D48D34000680B60FDF7E0FA0020BDE8FF
:1073C000F0819801B1D489E7044B1B689E03ACD4CB
:1073D00084E7032083E700BF003C024000380240FE
:1073E00064C80108CC000020C8000020014B1868C8
:1073F000704700BFCC000020044B05499B68054A3C
:107400000868C3F38223D35CD84070470038024039
:10741000CC00002074C80108044B05499B68054A4C
:107420000868C3F34233D35CD84070470038024049
:10743000CC00002074C801080E4B0F2202609A682D
:1074400002F0030242609A6802F0F00282609A68D9
:1074500002F4E052C2609B68DB0810B403F4E0530E
:10746000054C036123685DF8044B03F00F030B60C8
:10747000704700BF00380240003C02402DE9F04157
:10748000036813F0010582B004460BD09F4945699B
:10749000D1F88C2022F0C0622A43B5FA85F5C1F8F4
:1074A0008C206D099E070BD59849A069D1F88C20D6
:1074B00022F0C05202430028C1F88C2008BF0125E9
:1074C000180700F1A4805F0705D5914B94F8382088
:1074D000C3F8E0212368DE0608D58C49606AD1F83C
:1074E000942022F440020243C1F8942098060BD560
:1074F0008649A06AD1F8942022F000620243B0F1DC
:10750000006FC1F894202AD059061ED4012D30D026
:10751000802B2ED0DA0508D57C49E06AD1F88C2082
:1075200022F000420243C1F88C2013F4007009D00D
:10753000764A216BD2F88C3023F400430B430020B1
:10754000C2F88C3002B0BDE8F0817049206AD1F8F1
:10755000942022F080520243C1F89420D6E75B06C3
:1075600007D5D1F89430226A23F080531343C1F831
:107570009430684B654E00229A66FDF72FFA054657
:1075800004E0FDF72BFA431B022B3CD833681A01A9
:10759000F7D45F4B626BC3F8D8202268D3077ED53F
:1075A0006369002B7BD1E368A06861681B0643EA2E
:1075B000801320690B43554943EA0073C1F88430B6
:1075C00010060CD5E368A068626821691B0643EACF
:1075D000801313434D4A43EA0173C2F884304D4B84
:1075E0004A4E01229A66FDF7F9F9054604E0FDF7D7
:1075F000F5F9401B022806D833681901F7D523682E
:10760000DA0592D588E7032002B0BDE8F0813F4B50
:10761000414E002201921A6C42F080521A641B6C97
:1076200003F080530193019B336843F4807333600C
:10763000FDF7D4F9074604E0FDF7D0F9C31B022B90
:10764000E1D83368D905F7D5304EE369326F12F4CB
:1076500040723DD003F44071914210D0336F2D4AF7
:107660000121C2F8401E23F440730021C2F8401EDD
:107670003367336FDA0739D4E36903F44072B2F544
:10768000407F28D021498A6822F4F8128A601F4A74
:10769000116FC3F30B030B431367236813E79707BB
:1076A00003D5A369002B3FF47EAF960604D5A36AE9
:1076B000B3F1006F3FF477AF550681D5236A002BF5
:1076C0007FF47EAFA36AB3F1006F7FF479AF6AE70E
:1076D00003F44072D3E70D48826823F0704122F42E
:1076E000F81221F440710A438260D0E7FDF776F981
:1076F00041F28838074604E0FDF770F9C01B4045A9
:1077000081D8336F9B07F7D5B6E700BF003802403A
:107710000010474200004742007000402DE9F04150
:107720000368DD0782B004462FD59F498A6802F0BE
:107730000C02042A00F0C2808A6802F00C02082AB7
:1077400000F0B8806368B3F5803F00F0F980B3F5CE
:10775000A02F00F04C81944D2A6822F480322A60D8
:107760002A6822F480222A60002B40F0EE80FDF788
:1077700035F9064605E0FDF731F9801B642800F273
:1077800002812B689B03F6D423689F0728D5864A7D
:10779000916811F00C0F00F09F80916801F00C01CE
:1077A000082900F09580E368002B00F00F817F4BE3
:1077B0007D4E01221A60FDF711F9054605E0FDF73F
:1077C0000DF9401B022800F2DE8033689807F6D5D9
:1077D0003368226923F0F80343EAC2033360236865
:1077E0001A0716D56369002B00F081806F4B6E4E2F
:1077F0000122C3F8802EFDF7F1F8054605E0FDF7FC
:10780000EDF8401B022800F2BE80736F9B07F6D58F
:10781000236858072FD5644A136C13F0805377D030
:107820000025634E3368D90540F19D80A368012B84
:1078300000F0AD80052B00F01A815B4E326F22F014
:1078400001023267326F22F004023267002B40F0EF
:10785000A380FDF7C3F841F28838074605E0FDF73D
:10786000BDF8C01B404500F28E80336F9807F6D4F8
:10787000002D40F0C680A369C3B14B4DAA6802F049
:107880000C02082A2FD0022B484B4FF000021A6638
:1078900000F0BD80FDF7A2F8044604E0FDF79EF875
:1078A000001B02286FD82B689B01F7D4002002B080
:1078B000BDE8F0814A6850027FF544AF3A4A126849
:1078C00091037FF562AF6268002A7FF45EAF0AE041
:1078D000526856023FF567AF334A1268950723D5C1
:1078E000E268012A20D0012002B0BDE8F0812F4AD1
:1078F0002D4EC2F8803EFDF771F8054604E0FDF715
:107900006DF8401B02283ED8736F9F07F7D47FE7BE
:107910000193136C43F080531364136C03F0805392
:107920000193019B01257CE71F4920690A6822F029
:10793000F80242EAC0020A601A077FF56AAF51E70F
:10794000194A136843F480331360FDF747F8164E65
:10795000054604E0FDF742F8401B642813D833685D
:107960009A03F7D510E7336843F480733360FDF76B
:1079700035F807463368DA053FF558AFFDF72EF8BE
:10798000C01B0228F6D9032002B0BDE8F081064AE8
:10799000136F43F001031367FDF720F8024F06460B
:1079A00041F288380BE000BF003802400000474237
:1079B00000700040FDF712F8801B4045E3D83B6F94
:1079C0009B07F7D5002D3FF456AF1AE02D4A2E4EF7
:1079D0001360FDF703F8054604E0FCF7FFFF401BCA
:1079E0000228D0D833689907F7D42368F8E6264BE5
:1079F0001A6842F480221A601A6842F480321A60CF
:107A0000A3E7214A136C23F08053136433E7FCF798
:107A1000E5FF064604E0FCF7E1FF801B0228B2D830
:107A20002B689901F7D4216AE369626AE06A0B4323
:107A300043EA8213A26A216B43EA0063520843EAD5
:107A40000173013A0F4943EA024301226B600A665F
:107A5000FCF7C4FF0C4D044604E0FCF7BFFF001B1D
:107A6000022890D82B689A013FF520AFF5E7064B26
:107A70001A6F42F004021A671A6F42F001021A6785
:107A80008AE700BF0000474200380240704700BF4D
:107A900010B50446A0B1437903F0FF0263B1216839
:107AA000022363710B68002243F0040301200B6082
:107AB00060711046A26010BD0271FFF7E7FFEEE7AC
:107AC000012010BD704700BF38B50446002866D0BD
:107AD000437F03F0FF02002B5DD023685322022076
:107AE000CA21607759625A62DA6855063CD59968AE
:107AF0006268256921F4E00121F040019960616923
:107B000098682A430A430243E1689A6019611A6936
:107B1000A16842EA01421A61DA6822F08002DA6062
:107B20009A6891060DD5196CA06921F48021196419
:107B30001A6C02431A64FF21012259620020627705
:107B400038BDDA6822F0A002DA60FCF747FF05468C
:107B500005E0FCF743FF401BB0F57A7F14D823689B
:107B6000DA689206DFD4F4E74FF0FF32DA60FCF710
:107B700035FF05462368DA685006B8D4FCF72EFFB7
:107B8000401BB0F57A7FF5D92268FF2104235162AA
:107B90000120637738BD0277FFF794FF9DE701204E
:107BA00038BD00BF0368503343F82120704700BF41
:107BB0000368503353F82100704700BF2DE9F041AE
:107BC00080460E4615461F46D8F8003001E07A1C64
:107BD0000CD19C6836EA04020CBF4FF0010C4FF048
:107BE000000CAC45F3D10020BDE8F081FCF7F6FEB7
:107BF000069BC01AB842E7D3D8F80030D8F8041072
:107C00005A68B1F5827F22F0E0025A6015D0D8F8A8
:107C10002820B2F5005F07D00122002388F8512008
:107C200088F850300320DFE71A6822F400521A6007
:107C30001A6842F400521A60EEE7D8F80820B2F54C
:107C4000004F02D0B2F5806FE1D11A6822F04002F5
:107C50001A60DCE730B50B4611464268B2F5827F08
:107C600083B0044608D0009100220121FFF7A6FF4F
:107C700088B9002003B030BD8268B2F5004F1ED035
:107C8000B2F5806F0ED00091002280212046FFF7D0
:107C900095FF0028EDD0636D032043F0200363655A
:107CA00003B030BD05682A6822F040022A600091C6
:107CB00000220121FFF782FF0028DAD0EBE70068FD
:107CC000026822F040020260DDE700BF30B5174BCA
:107CD000174C1B68A4FB033C436885B04FEA5C5C0F
:107CE0004FF47A7505FB0CF5B3F5827F04460395D6
:107CF00007D10CE0039B2268013B039393681B06AA
:107D000002D5039B002BF5D1002005B030BD0092B9
:107D10000B4600228021FFF751FF0028F4D0636D4D
:107D200043F0200303206365EFE700BFCC00002091
:107D3000819F5E16704700BF70B5044600283BD097
:107D400090F8513003F0FF02002B30D004F108000E
:107D500007C86368666A03430B436169E0691343BC
:107D60000B432268216A022584F8515003430B43D8
:107D70001168A069A56A21F0400111602B43010C34
:107D800000F400700343136001F004033343B5F5BE
:107D9000005F536004BFE36A1361D369002023F4DA
:107DA00000630121D361606584F8511070BD80F8D3
:107DB0005020FFF7BFFFC9E7012070BD90F8503099
:107DC000012B70B504465ED090F8513001208342FB
:107DD00084F85000DDB205D00225002384F850302D
:107DE000284670BD0029F8D0002AF6D0032384F875
:107DF000513000236365A286E286A268E387B2F56C
:107E0000004F2268A36363642364A38708BF1368D9
:107E1000216304BF43F480431360A36AB3F5005F9A
:107E200028D0A06C194EE38E0664194EC663194E15
:107E3000C66400260C329BB20665FCF715FF88B9B4
:107E400023681A68520603D41A6842F040021A6086
:107E50005A6842F020025A605A6842F00202002535
:107E60005A60BAE7636D012243F01003636584F83A
:107E70005120B2E7136823F400531360136843F4EE
:107E800000531360CDE70225284670BDC97F000866
:107E90001D800008F97F000810B5044690F85000D6
:107EA000012873D0012084F8500094F85100012873
:107EB0005FFA80FC0ED06068B0F5827F04D00220AB
:107EC000002384F8503010BDA0680028F7D1BCF121
:107ED000040FF4D1002957D0002A55D0002B53D0DD
:107EE00094F8510021630428A16AA3861CBF0520D1
:107EF00084F851000020B1F5005F60652168E386D9
:107F0000A263A387E3872064606407D10B6823F42E
:107F100000530B600B6843F400530B6094F851302E
:107F2000E06C042B3DD0214B0364214BC363214BF8
:107F3000C36400230365E38F0C319BB2FCF794FE0E
:107F400030BB2268A16C536843F001035360E38E99
:107F50000864C863C86408659BB208460C32216B8C
:107F6000FCF782FEA0B923681A68520603D41A6887
:107F700042F040021A605A6842F020025A605A6881
:107F800042F002025A609BE7012099E7022010BDEF
:107F9000636D012243F010036365104684F851209D
:107FA0008EE7054B0364054BC363C0E7E97F000818
:107FB00041810008F97F0008D97F00088D80000802
:107FC000704700BF704700BF08B5806BFFF7FAFF2E
:107FD00008BD00BF704700BF08B5806BFFF7FAFF10
:107FE00008BD00BF704700BF08B5806BFFF7FAFF00
:107FF00008BD00BF704700BF806B026808B55368BA
:1080000023F003035360436D012143F010034365E4
:1080100080F85110FFF7EEFF08BD00BF30B50546F0
:1080200083B0846BFCF7DAFC2B681B68DB05024627
:1080300021D42368586820F020005860586820F048
:108040000200586064212046FFF740FE18B1636DBE
:1080500043F020036365A36833B922680193D368B2
:10806000019393680193019B01230022E28684F827
:108070005130636D23B92046F9F718FE03B030BDC7
:108080002046FFF7B7FF03B030BD00BF30B505464F
:1080900083B0846BFCF7A2FC2B681B68D9050546EE
:1080A00021D42368A16A5A68B1F5005F22F020024A
:1080B0005A6035D0A26852B35A6822F001025A6061
:1080C0002A4664212046FFF7C5FD08B120236365D9
:1080D000012223680021E18784F851209A68D206A2
:1080E00006D4636D73B92046FFF76AFF03B030BD55
:1080F000626D4FF6EF7142F0020262659960636D46
:10810000002BF0D02046FFF775FF03B030BD62684A
:10811000B2F5827FD0D15A6822F003025A60CFE7CD
:1081200001220090642311462046FFF747FD18B155
:10813000636D43F0020363652368DA68BAE700BF42
:1081400030B5054683B0846BFCF748FC2B681B6890
:10815000D905054622D42168A26A4B68B2F5005FB2
:1081600023F020034B602DD02A4664212046FFF7E0
:10817000ADFD18B1636D43F02003636523685A6851
:10818000002122F0030201205A60E186E18784F891
:1081900051009A68D20606D4636D73B92046F9F788
:1081A0009FFD03B030BD626D4FF6EF7142F00202E9
:1081B00062659960636D002BF0D02046FFF71AFFCF
:1081C00003B030BD01220090642311462046FFF722
:1081D000F5FC18B1636D43F0020363652368DB6847
:1081E000C2E700BF30B502685168936813F0400FD2
:1081F00085B00446C3F3801505D113F0010F02D0FA
:1082000011F0400F7AD1980701D5080670D413F009
:10821000200FC3F3401049D0880645D575B194F8B6
:10822000510003286CD0606D40F0040060650020B0
:108230000090D0680090906800900098606D40F0C9
:10824000010060650020029090680290106820F0A4
:10825000400010600298C3F30023002B3ED1636DF1
:1082600013B3536823F0E003536001208B0784F8B5
:1082700051004DD05368E06C23F00303536040B1CC
:10828000254B0365FCF778FD18B1636D43F040039F
:108290006365A06C40B1204B0365FCF76DFD18B120
:1082A000636D43F04003636505B030BD95B18D0645
:1082B000FAD594F85150032D22D0656D45F0040590
:1082C00065650090D0680090906800900098C3F3B6
:1082D0000023C2E7DD05E7D58B06E5D5636D0020F9
:1082E00043F008036365039093680393039BB6E729
:1082F000636C204605B0BDE830401847036CF9E7D1
:1083000000230193D368019393680193019BCBE70A
:108310002046FFF76FFEC7E71D83000808B5806B96
:108320000023C387C386FFF765FE08BD704700BF03
:1083300070B50E461546044618B390F8493003F060
:10834000FF02CBB1214651F8080B00F035FBA268C3
:108350002068314600F070FB236BA26860682946F4
:1083600000F096FB2268A16852F8213043F0010327
:1083700042F82130002070BD80F84820FFF7D6FF7A
:10838000E0E7012070BD00BF704700BF0368DA68F6
:1083900042F00102DA609A6802F00702062A03D06E
:1083A0001A6842F001021A60002070470368DA6818
:1083B00022F00102DA601A6A41F211110A4208D170
:1083C000196A40F24442114203D11A6822F00102B4
:1083D0001A600020704700BF704700BF704700BFA1
:1083E000704700BF704700BF704700BF03681A693D
:1083F000910710B5044602D5DA6892075FD41A696E
:10840000500702D5DA68510746D41A69120702D517
:10841000DA6810072ED41A69D20602D5DA68D006B7
:1084200018D41A69D10702D5DA68D2075DD41A695F
:10843000100602D5DA6811065FD41A69520602D511
:10844000DA68500661D41A69910602D5DA68920694
:1084500043D410BD6FF010021A61DB69082213F4D7
:10846000407F2277204664D0FFF7BAFF00222368BE
:108470002277D6E76FF008021A61DB6904229907B8
:108480002277204652D1FFF7A9FF2046FFF7AAFF27
:10849000002223682277BEE76FF004021A619B690D
:1084A000022213F4407F227720463CD1FFF796FF4B
:1084B0002046FFF797FF002223682277A5E76FF099
:1084C00002021A619B6901229B07027725D0FFF700
:1084D00087FF00222368227791E76FF02002204671
:1084E0001A61BDE8104000F0B3B86FF001021A61E4
:1084F0002046FFF771FF236899E76FF080021A6149
:10850000204600F0A7F8236897E76FF040021A6151
:108510002046FFF769FF236895E7FFF75FFF2046D6
:10852000FFF760FFD5E7FFF75BFFC4E7FFF758FFF2
:10853000AEE7FFF753FF2046FFF754FF96E700BF73
:10854000344A0368904230B44CD0B0F1804F34D0FC
:10855000A2F57C42904230D002F5806290422CD04D
:1085600002F58062904228D002F57842904239D0DC
:1085700002F57052904224D002F58062904220D0E1
:1085800002F5806290421CD0A2F59832904218D039
:1085900002F58062904214D002F58062904210D0C1
:1085A0004D698C680A6823F080032B430360012324
:1085B000C462826230BC436170474A6823F0700332
:1085C0001343CC684A6923F44073234323F08003A8
:1085D00013438C680A6803600123C462826230BC62
:1085E000436170474C68CA6823F07003234323F447
:1085F000407313434A6923F08003134303608B687D
:10860000C3620B6883620B690363012330BC43615F
:10861000704700BF0000014010B50446B0B190F8AB
:108620003D3003F0FF0263B12146022351F8040BF1
:1086300084F83D30FFF784FF012384F83D300020AB
:1086400010BD80F83C20FFF79FFEEDE7012010BD34
:10865000704700BF704700BF0268116938B5044613
:10866000C068A368256921F4405101431161D168B4
:10867000E0692B43656921F416412B4321F00C017D
:1086800003430B43D3605369A16923F440730B4345
:10869000B0F5004F5361294B23D09A421ED003F509
:1086A00080639A421AD0FEF7A7FE636819219A00E8
:1086B000A0FB01019B0F0EF0FDFD214AA2FB001360
:1086C0005B092168642404FB130000013230A2FB23
:1086D00000201B0103EB5010886038BDFEF79CFEA4
:1086E000E3E79A4226D003F580639A4222D0FEF750
:1086F00083FE6268124D92184FF019014FF000038B
:108700005B41A0FB01010EF0D5FDA5FB0032510934
:10871000642303FB1103DB003233A5FB0323C3F304
:1087200042121B09246802EB011203F4F87313448C
:10873000A36038BDFEF770FEDBE700BF001001400C
:108740001F85EB51704700BF38B5044650B390F811
:10875000393003F0FF0203B32268242384F8393050
:10876000D36823F400532046D360FFF775FF2368D6
:108770001A6922F490421A615A6922F02A025A6157
:10878000DA680025202142F40052DA602846E563C9
:1087900084F8391084F83A1038BD80F83820FFF793
:1087A000D1FFD9E7012038BD704700BF704700BF37
:1087B00008B590F83A30222B22D18368B3F5805F58
:1087C0001FD0036943BB836A0268591C52688162E7
:1087D0001A70C38D013B9BB2C3858BB90368DA68FD
:1087E00022F02002DA60DA6822F48072DA605A69D4
:1087F000202122F001025A6180F83A10FFF7D6FFDB
:1088000008BD0269836A82B902685268C2F308022D
:1088100023F8022B8362DCE70368826A5B68511CE1
:1088200003F07F0381621370D3E702685268D2B20B
:1088300023F8012B8362CCE7704700BF03681A68F6
:1088400070B51607DD68596904460CD1910601D54B
:10885000AE066DD4160601D5280642D4510601D5C0
:108860006A065AD470BD01F0010105F49070084306
:10887000F0D0D00705D5EE0503D5E06B40F0010040
:10888000E063500724D529B1E06B960740F0020061
:10889000E06321D4160707D505F02000014303D07B
:1088A000E16B41F00801E163E16B0029DAD0900649
:1088B00001D5A90664D45A69E56B02F0400205F0BF
:1088C0000805154338D12046FFF7B6FFE56370BDB4
:1088D0009007DFD50029DDD0E06B40F00400E063B5
:1088E000D8E794F83920212ABCD1A268B2F5805F7C
:1088F000226A4AD0511C216212785A60E28C013AF5
:1089000092B2E284002AADD1DA6822F08002DA6005
:10891000DA6842F04002DA6070BDDA68202122F0A5
:108920004002DA60204684F83910FFF73DFF70BD41
:10893000BDE87040FFF73CBFDA6822F49072DA605D
:108940005A69202122F001025A6184F83A105A69CA
:10895000520611D55A69606B22F040025A6158B133
:10896000104B0365FCF708FA00283FF47BAF606BFF
:10897000BDE87040036D18472046FFF75DFF70BDEE
:108980002046FFF715FF236895E711882069C1F39A
:108990000801596010B902322262AFE70132226247
:1089A000ACE700BFA989000808B5806B0023C38528
:1089B000C384FFF741FF08BDF0B40C688D6850F820
:1089C00024304A681B4E4F6B1E4045EA0203CA68BA
:1089D00013430A6913434A691343CA6913430A6A72
:1089E00013434A6A13438A6A1343CA6A13430A6BDE
:1089F0001343CA6B3B4313438A6B13433343082D22
:108A000008BF43F04003B7F5801F40F8243006D07C
:108A100014B103681A4302600020F0BC7047002CB8
:108A2000FAD0036843F48013036003681A430260BA
:108A3000F2E700BF8004C0FF0B6900EB820203F184
:108A4000FF3C536810B58C6903F0404E0B6823431C
:108A50004C6843EA04138C6843EA0423CC684969F0
:108A600043EA044343EA0C53023943EA016343EA0D
:108A70000E0353600368DB024FEA0C5C05D54368C4
:108A800023F470034CEA03034360002010BD00BFD1
:108A9000B3F5804F30B406D06FF0704340F8223009
:108AA00030BC0020704750F822300A4C8D691C40C1
:108AB0000B682B434D6843EA05138D68C96843EA88
:108AC000052343EA0143234340F8223030BC002011
:108AD000704700BF0000F0CF054BD3F888204FF05F
:108AE000006142F47002C3F888209960704700BFAB
:108AF00000ED00E0DFF834D0002103E00C4B5B58C0
:108B0000435004310B480C4B42189A42F6D30B4A9F
:108B100002E0002342F8043B094B9A42F9D3FFF7E5
:108B2000DBFF0FF0B3FCF7F7ADFB7047000004204C
:108B30000819020800000020200200202002002066
:108B4000A8180220FEE737B50D4600F108010246DD
:108B5000C36A03C91C688DE803001046694601F02A
:108B60008AF8B5F90020BDF9003022449A4217DC9A
:108B7000B5F90420BDF90430121B9A4210DBB5F997
:108B80000220BDF9023022449A4209DCB5F9060000
:108B9000BDF90630041B9C42ACBF0020012000E060
:108BA000012003B030BDB0F9003070B5B0F90460F9
:108BB0001588D088948852884D80F31A9BB2181A71
:108BC0009B1A08808B80CC8070BD438E1B0713B529
:108BD0000C460FD5684601F061FBBDF802302380DA
:108BE000BDF80630A380BDF800306380BDF80430C6
:108BF000E38002E0084601F051FB02B010BD38B539
:108C000004460D4601F0F9FFE36A284629461A6832
:108C1000BDE8384005F0D0BA37B50C46054607F038
:108C200033FB428E0190944203D04486284602F0E2
:108C30002CF801A807F036FB03B030BD37B50C4661
:108C4000054678B107F020FB428E019004EA02014C
:108C50008C4204D014434486284602F016F801A83A
:108C600007F020FB03B030BD37B50D46044670B1A8
:108C700007F00AFB428E019022EA05018A4203D0E6
:108C80004186204602F001F801A807F00BFB03B073
:108C900030BD0000024B42861B68C36201867047EC
:108CA000D0000020F0B50D4685B00646002800F043
:108CB000938007F0E9FA2B680290162B52D00CDC57
:108CC000112B33D002DC0D2B3ED07EE0142B77D05D
:108CD000152B7AD1B0F9303070E01F2B6BD002DC4D
:108CE0001E2B42D071E0312B1ED0B3F5407F6CD1EA
:108CF000C36A1968EB68C3621B6802A8CD1A07F043
:108D0000D1FA304607F0C0FA04AC694244F8040DC9
:108D10000A462B46009500F034FF204607F0C2FAC1
:108D2000304601F0B2FF4EE000243FE0438ED9060A
:108D30004BD5EB681B7A002B47D002A807F0B2FA9C
:108D4000304601F017F840E0EB68DB68002B3CD0C0
:108D50001B7A002B39D002A807F0A4FA304601F0A4
:108D6000BDFA30E0EB6803862DE0EB68418E012B05
:108D700008D1CA060DD5304641F00101FFF74CFF7E
:108D8000082708E021F001013046FFF745FF0927D9
:108D900001E04FF0FF3702A807F084FA7B1C4FF088
:108DA000000405D03046394601F0B7F8EC600DE01C
:108DB0000123EB600AE0438EC3F30013EB6002E093
:108DC000E968FFF71CFF002400E00124029B23B1A7
:108DD00002A807F067FA00E00124204605B0F0BDC4
:108DE00070B50D46FE211646044601F035FA2946B7
:108DF00000F0B3FF2046FF2101F02EFA3146BDE816
:108E0000704000F0AABFF8B51C46438E069F1B07B2
:108E10000D4616460AD5002C07DB2846311BA21941
:108E200006F00CFB013C3D44F5E7F8BD002C07DBE8
:108E30002846311BA21906F089F8013C3D44F5E7AC
:108E4000F8BD37B505460C4619B9684601F026FA53
:108E50006C466B8E1B0705D5224628466946FFF7F0
:108E6000A2FE6C4628462146FFF76DFE18B1EB6A5C
:108E700020461B69984703B030BD2DE9F04F2DED1A
:108E8000028B85B00D4607F0FFF90090006905F0F0
:108E90000FFF009BD86805F039FF022005F0ECFEBB
:108EA000009CA68CE36916F001061AD0002B77D03F
:108EB000A06807F0E9F90190C26A636917681F4466
:108EC00001F01EF9A369384433B1012B70D1B5F913
:108ED000003083426CDD1CE0B5F90430834218DBBE
:108EE00066E0002B5CD0A06807F0CEF90190C36A61
:108EF000D3F8008006F004F863690746C8EB03095D
:108F000001F006F9B5F90210EA88484407448F4297
:108F100003DA01A807F0C6F942E012B29042F8DC89
:108F2000A06802A901F0FCF8019BBDF90CB0DA6D54
:108F3000D3F854A0BDF90870256AC2EB0B0BB3F847
:108F40007820D207574458BFD3F88C603D4435444D
:108F5000BD4222DDE369ED1AFAE7BD421BDDA069DF
:108F600005F094FE236AD4ED0A7AEB1ACAEB0303E8
:108F7000C8EB03039B1B08EE103AB8EEC88A2846DC
:108F800028EE278A494605F09FFFB0EE480A94F87C
:108F90002C0005F099FCE3691D445D45DDDDB8E773
:108FA000684607F07FF905B0BDEC028BBDE8F08F95
:108FB000A06802A901F0B4F8019B1D6ED3F8588097
:108FC00005F09EFFBDF90E60019BBDF80AA0D3F825
:108FD0008030761B256A751B1D44B54201DAE369B2
:108FE000FAE74FF0020990FBF9F908FA8AF39D427B
:108FF0008FDBB5421CDCA06905F048FE236AD4ED86
:109000000A7A711BC91A019BD3F880208A1808EECE
:10901000102AB8EEC88A384628EE278AC9EB05011F
:1090200005F052FFB0EE480A94F82C0005F04CFC15
:10903000E369ED1AD9E700002DE9F34781463020B6
:10904000884617461E4607F0F1FB8246D0B107F06E
:109050001BF902AD0D4A45F8040D4FF07E538362B3
:10906000C0F81490C0F818808784C66100F10C0322
:10907000044692E8030083E80300054B236028467A
:1090800007F010F9504602B0BDE8F087D400002088
:109090007B8E000800B52DED028BF0EE408A83B088
:1090A00090B107F0F1F890ED0A8A0190B4EE688A69
:1090B000F1EE10FA04D0C0ED0A8A806801F0E5FDF7
:1090C00001A807F0EFF801E09FED048AB0EE480A2E
:1090D00003B0BDEC028B5DF804FB00BF0000000094
:1090E00013B5044607F0D0F80190406A20B107F0AC
:1090F00005F9019B00225A6201A807F0D3F8204627
:1091000007F0FCF802B010BD2DE9F0438BB007F07A
:10911000BBF80790406A002860D007F0B5F8079BBD
:1091200005900646986807F0AFF8079BD0F8548082
:10913000056E876DC46D069008A9986800F0F0FF71
:10914000BDF82230079A0698BDF82010D2F820907A
:109150001F44ADF82270BDF82430BDF826701C1BEA
:109160007F1B1369D0F88C505D1B92F82830414466
:1091700089B2A4B2BFB2012BADF82010ADF82440E3
:10918000ADF82670D0F8808009B208D024B2641BF4
:109190000134A14204DD0C1B06EB44062D1B0C46DA
:1091A000002D15DD906905F0B1FD4FF0FF32012370
:1091B0008DE80C00079A3FB292F829300293C9EB70
:1091C000070930462946224609EB080306F05AF9FA
:1091D00006A807F067F805A807F064F807A807F0E5
:1091E00061F80BB0BDE8F0831FB590F82830012B73
:1091F0000446806827D102A900F092FFA06807F01A
:1092000043F8BDF80A20836D01901344ADF80A308D
:10921000BDF80E20036ED31AADF80E30426DBDF8C6
:1092200008301344226913449BB29A1E01A8013BE3
:10923000ADF80820ADF80C3007F034F8A06802A9AA
:1092400001F0E7FC01E000F05FFB04B010BD00009E
:109250002DE9F74380462C200E4617461D4607F0A1
:10926000E5FA044618B3700007F0E0FA814658B1F9
:1092700057B14DB107F008F839466A0001900FF078
:109280008FF901A807F00EF8204606F0FDFF0A4B03
:109290000190C360094B0360094BC0F82490C0F8EB
:1092A000188046610561436001A806F0FBFF204677
:1092B00003B0BDE8F08300BFE99100080991000800
:1092C000E19000081FB5ADF8061006F0DDFF029032
:1092D00068B1406A06F0D8FF0DF10602014603901E
:1092E0000223029800F03FFB03A806F0DBFF02A870
:1092F00006F0D8FF05B05DF804FB13B50C4660B16D
:1093000006F0C2FF036A0190A34203D004628068A2
:1093100001F0BBFC01A806F0C5FF02B010BDF0B51E
:109320008BB002A9044600F0FBFE204606F0ACFF1D
:10933000BDF90A20BDF90E600190B61A826D456D27
:10934000C76DB61A026EB61AB0F87820510707D466
:10935000416FB1422046D4BF0021012100F0FBFC47
:10936000019BBDF90C105A6FDA67BDF90820C3F8EC
:1093700084608A1A551BB3F878209207C7EB05055D
:1093800007D4196FA9422046D4BF0021012100F063
:10939000E0FC0198036FC0F88830C0F890507C3032
:1093A00000F08AFF0198883000F086FF019B03F1EE
:1093B0007C0207CA883307AE86E8070093E80700F7
:1093C00004AD85E8070001A806F06CFF2046314691
:1093D0002A46FFF705FD0BB0F0BD73B50C460646F7
:1093E00006F052FF0190204607F05AFB0546204642
:1093F00000F0F6FE019BFE280CBFC3F88050C3F8B6
:109400008C50304601F041FC01A806F04BFF02B041
:1094100070BD2DE9F04F44680668054697B02046B8
:109420002946FFF73FFCB6F5407F074602D12046AC
:10943000FFF775FF002F00F064822B680B2B00F004
:10944000008206DC052B40F059822046FFF767FFBB
:1094500054E20F2B03D0262B00F03D824EE2ED6844
:109460000295204606F010FFC36AC16D1B68D0F854
:109470005490D0F858B0D0F860A00D900EAD2846AA
:109480000393019100F00AFF0D982946FFF7D9FCDC
:1094900095E8030012AB83E803000398BDF84A1077
:1094A00082B25944BDF84E001144ADF84A1002EBA7
:1094B0000A01411AADF84E10BDF848101144494454
:1094C000ADF8481001990A44BDF84C108A1AADF85D
:1094D0004C2093E8030010AA82E80300104600F035
:1094E000FBFB0D9B586B05F00FFC06F09DFA0D9BE6
:1094F000D3F8943013B12046002198470D9D95F87C
:109500006C30002B00F08D80204614A900F008FE7E
:10951000EB6ABDF856001B68BDF85420BDF8521028
:1095200004930790BDF85030286C0592069308917B
:109530006E6CAF6C05F0EAFB05F0DCFC099016B927
:10954000002F4BD146E0EB6C06EB030CB5F87830FE
:10955000DB0754BFD5F88C3000230CEB0308B04573
:1095600002DBC6EB0808FAE795F87A0005F098FBED
:109570000598019A03B206984A4401B2C2F1010269
:109580005B1A13449845DBDA0498BDF95210BDF913
:10959000563095F87A20484440445944CAEB0303B6
:1095A0001AB1024605F02CFF02E01A4605F0CEFC87
:1095B000B044DDE795F87B0005F072FB0799089849
:1095C0000BB20BEB0A0201B2C2F101025B1A1344A7
:1095D0009E420CDB099805F063FB22E02E6DD5F866
:1095E00080303E44F61ABE42E4DBF61BFBE70198EE
:1095F000BDF95420BDF95610BDF95030121A95F836
:109600007B00CAEB0101891B4B4420B118460B4675
:1096100005F0F6FE03E00846194605F00FFF3E444C
:10962000CCE7039A12A80EA904F0C6FD12A800F018
:1096300053FB0D9B93F83B20FF2A00F0A380B9F168
:10964000000F08D1BBF1000F05D1019919B9BAF18A
:10965000000F00F09780DA6A14A92046156800937D
:1096600000F05EFD00F04CFD049000F051FDBDF9EE
:109670005220009BBDF9546005905A440392019A10
:10968000986BBDF95070BDF95680B61A05F03CFBD9
:10969000009BD86B4F44CAEB080805F037FBB9F1C3
:1096A000000F1BD002980499B0F9003009F1FF3285
:1096B0002A445B1A934211DCBDF95630BDF95000C3
:1096C000CAEB030305EB0B01013306F07BF9039AA8
:1096D000781E511E08F1010205F038FCBBF1000FA5
:1096E00017D002980599B0F902200BF1FF332B44F3
:1096F000521A9A420DDCBDF95000BDF95210BDF965
:10970000542006F05FF9039A791E501E721C05F072
:1097100095FE019BD3B10299BDF95420D01AB1F93D
:109720000430049901305B1A83420FDBBDF95630D7
:10973000CAEB030305EB0B01013306F043F9039A6F
:10974000701C511E08F1010205F000FCBAF1000F77
:1097500018D00298BDF95630B0F906200598CAEB2A
:1097600003010131C0EB020A8A450BDBBDF9500051
:10977000BDF9542006F026F908F10100791E721C8B
:1097800005F05CFE0D9BD3F8943013B12046012107
:10979000984710A800F0A0FA0D9B586E07F08CFCBB
:1097A00000250746BD421AD00D9B2946586E07F08A
:1097B00005FD06F069FD149078B10668304606F0A4
:1097C00063FD0C9030B103680299304698470CA8AD
:1097D00006F068FD14A806F065FD0135E2E712A861
:1097E00000F07AFA0D9B986E07F066FC002507469C
:1097F000BD421AD00D9B2946986E07F0DFFC06F09B
:1098000043FD149078B10668304606F03DFD0B909C
:1098100030B103680299304698470BA806F042FD24
:1098200014A806F03FFD0135E2E7002000F054FAED
:109830000D9BD3F8943013B12046022198470DA810
:1098400046E0204606F020FD1290406E07F034FC02
:1098500000240646B442129B18DA586E214607F0DF
:10986000ADFC06F011FD149070B10568284606F0B5
:109870000BFD109028B1476810A806F013FD28468C
:10988000B84714A806F00EFD0134E3E7986E07F020
:1098900013FC00240546AC42129B0FDA986E214659
:1098A00007F08CFC06F0F0FC149028B1006806F07C
:1098B00025FD14A806F0F6FC0134ECE716AC586E52
:1098C00007F053FC54F8103D986E07F04EFC20460C
:1098D00006F0E8FC15E0EB68052B0FD12046AE68DA
:1098E00000F0F0FB864205D02046AE6800F0E5FBB4
:1098F000864203D16868A968FFF76FFD284601F02A
:10990000EFFD17B0BDE8F08F2DE9FF41044606F0EA
:10991000BBFC034604A8D3F8548040F80C3D9F6D6F
:10992000DE6D1D6E06F0BEFC204602A900F0F8FBBD
:10993000BDF808309844BDF80A30ADF808801F44DF
:10994000BDF80C30ADF80A709E1BBDF80E30ADF8B6
:109950000C605D1B204602A9ADF80E5001F059F9CC
:1099600004B0BDE8F081F8B51D46836804460E4694
:10997000174623B30069636998420ED1421E6A43B9
:10998000084629440EF01AFE2069013800FB0560E4
:1099900039462A460EF012FE0CE0431C236100FB00
:1099A000051011462A460EF009FEE36813B1204661
:1099B0009847F8BDA068BDE8F840FFF7A5BFF8BD1F
:1099C000F0B587B00C9C00940D9C0194174C029448
:1099D000109C6C34039401F099F9064618B307F013
:1099E00000FC054607F0FDFB0446304606F04CFC43
:1099F00045660F4D84660F9905900022FFF74AF9DE
:109A000006AF0FCD57F804ED0EF134040FC40FCD9F
:109A10000FC495E80F0084E80F000E9BAEF8783075
:109A2000384606F03FFC304607B0F0BD13940008FE
:109A3000DC00002010B586B0089C0094099C0194BD
:109A40000A9C02940B9C039400240494FFF7B8FF33
:109A500006B010BD30B585B004460191D0B106F016
:109A600013FC04AB456E43F8040D184606F01AFCCF
:109A7000019806F009FC024604A8946040F8082DFD
:109A800006F010FC284601A9042207F024FB20461A
:109A900001F0FBF805B030BD30B585B0044601914A
:109AA000D0B106F0F1FB04AB856E43F8040D184607
:109AB00006F0F8FB019806F0E7FB024604A8946064
:109AC00040F8082D06F0EEFB284601A9042207F015
:109AD00002FB204601F0D9F805B030BD73B50D4644
:109AE0001446064698B106F0CFFB032C019009D826
:109AF00000EB8400446BAC4205D04563304601F076
:109B0000C4F800E0002401A806F0CCFB00E0044605
:109B1000204602B070BD73B50E46054678B106F01A
:109B2000B3FB90F86C400190B44204D080F86C60B4
:109B3000284601F0AAF801A806F0B4FB00E00446AC
:109B4000204602B070BD2DE9F3410F4690461D46F8
:109B5000064698B106F098FB044602A8089B2366C7
:109B600040F8044D6765C4F85880E56506F09AFB37
:109B70003046FFF7D4FB304601F087F802B0BDE86D
:109B8000F0812DE9F04F87B0C46903938A4693466C
:109B9000002C6DD0204606F077FB816A059001F419
:109BA0002073802BB0F8008042888688C58808D052
:109BB000B3F5207F08D108EB0A091FFA89F9039B46
:109BC00008E0039883B201E01FFA8AF303EB080967
:109BD0001FFA89F901F4A0613344B1F5807F9BB28B
:109BE00008D0B1F5A06F08D102EB0B0C1FFA8CFC6A
:109BF000109F08E010998FB201E01FFA8BF707EB76
:109C0000020C1FFA8CFC0FFA89F90FFA88F812B2CD
:109C10002F440FFA8CFCB9EB08010292BFB2C2EBE1
:109C20000C0200D142B120460193CDF800C000F0F3
:109C300008FADDF800C0019B1BB2C9EB030936B27C
:109C4000029BC6EB08083FB22DB2CCEB070C5D1BA4
:109C500019EB08010CEB050200D112B1204600F00F
:109C6000E1F806A850F8043D1C6A06F01BFB8FE7DC
:109C700007B0BDE8F08FB0F90030B0F90220084617
:109C80005242594205F0D4B810B5044670B100F004
:109C9000FCFF204600F0BBFA04463CB12046FFF72B
:109CA000F3FF204606F0E6FA046AF6E710BD13B5A6
:109CB000044670B106F0E8FA826A0190930705D471
:109CC00042F0020282622046FFF7DEFF01A806F0A2
:109CD000E9FA02B010BD0000044B10B51B685C6CC3
:109CE000586400F02BFE204610BD00BF2401002068
:109CF000F7B50D46114606461F4600F0ADFA04467C
:109D0000A5B120B93046394606F0D9FE14E006F078
:109D1000BBFA02AB826A43F8040D22F4004242F01F
:109D200002028262184606F0BDFA05E020B100F09A
:109D30008CF9204601F006FB201C18BF012003B05F
:109D4000F0BDFE220823FFF7D3BFFF220023FFF759
:109D5000CFBFFFF7FABFFFF7F4BF1FB530B129B18E
:109D6000242303916946009300F038FF05B05DF8A5
:109D700004FB0000F0B587B00446002102A81022C1
:109D80000EF036FC002C3AD01F4B204A196852F8CE
:109D90002100844216461F4631D01E238DE8110053
:109DA000029310B102A907F033FA0123204602A959
:109DB000059307F02DFA059D15BB3B6846F8234037
:109DC000204600F084F9044638B12023029302A90A
:109DD00000AB059307F01CFAF2E7009C204600F068
:109DE00032F968B1204600F072F9044640B12023F0
:109DF000029302A900AB059307F00AFAF2E70125E6
:109E0000284607B0F0BD00BF4817022038170220CF
:109E1000024B1A6818601046704700BF50170220A6
:109E200007F0E2B92DE9F04151EA02038AB0804619
:109E30000E4617466ED000286CD006F025FA034671
:109E4000039003C804AD06AC85E8030084E8030072
:109E50007EB19A6A02F42072802A05D1BDF81820DA
:109E6000961BADF8186004E0BDF81C201644ADF850
:109E70001C6087B19A6A02F4A062B2F5807F05D1B6
:109E8000BDF81A20D71BADF81A7004E0BDF81E20EB
:109E90001744ADF81E709B6ADA0302D5404600F005
:109EA00081FD94E80300039B83E803009B6A9B0702
:109EB0000AD508A82946224604F0CAFF039B08A831
:109EC00099691A6A00F072FEBDF91C40BDF91430A0
:109ED000BDF91E70BDF91600BDF91860BDF910106E
:109EE000BDF91A50BDF91220E31A381A0AACAA1AA1
:109EF0000090711A0398FFF744FE54F81C1D01F1FD
:109F0000080004F015FA4046052100F06BFE2046DB
:109F100006F0C8F90AB0BDE8F0811FB52623039109
:109F20006946009307F09AFA05B05DF804FB2DE945
:109F3000F04188B006460C46154604A800211022C0
:109F40000EF056FB36B3304606F09EF921462A46FF
:109F5000019004F06DFF0198214608302A4604F074
:109F600067FF08A850F81C2DD2F81C80176A06F06D
:109F700099F9404621462A46FFF7D9FF0323049367
:109F8000304602AB04A90793029403953E4607F0BE
:109F90003FF9D7E708B0BDE8F0812DE9F0438BB079
:109FA00006460D46144606A8002110220EF020FB9E
:109FB000002E43D00DB9002C40D0304606F064F995
:109FC0000346019003C80DF1080888E80300224603
:109FD0001846294604F02CFF01980AAF294622466C
:109FE000083004F025FF57F8243DD3F81C9038467C
:109FF00006F058F9224648462946FFF798FF3046B2
:10A0000006F042F9826A019092070AD5816941B14E
:10A01000026A00F0B6FD019B404699691A6A00F099
:10A02000B0FD384606F03EF903230693304604ABF4
:10A0300006A909930495059407F0EAF80BB0BDE86A
:10A04000F083FFF7AABF00F09DBC13B588B106F0FE
:10A050001BF9826A02AC910744F8040D06D522F080
:10A06000020282628169026A00F0A0FD204606F0C9
:10A0700019F902B010BD70B506460D4606F0FAF8A3
:10A08000C4694CB1204600F0ABF8A842204613D07A
:10A0900006F0F0F8046AF4E7304606F0EBF8C4691D
:10A0A000204644B12946FFF7E6FF28B9204606F0CE
:10A0B000E1F8046AF4E770BD70BD10B1FF21FFF74D
:10A0C000DABF704710B1FE21FFF7D5BF704708B562
:10A0D000034610B106F0CEF88369184608BD08B5EE
:10A0E00020B106F0C7F8B0F9000008BD08BD08B5FA
:10A0F00020B106F0BFF8B0F9020008BD08BD0000AD
:10A10000024B1B68986CFFF7EABF00BF24010020D8
:10A11000024B1B68986CFFF7EABF00BF24010020C8
:10A12000F0B50C4687B0064600284BD0002949D030
:10A13000FF2100F091F8FE210546304600F08CF832
:10A1400069460746304607F0B1F9304602A900F0EB
:10A150003BF8C7B1384604A907F0A8F9BDF90010CB
:10A16000BDF9022004A84942524204F061FE38467B
:10A1700000F046F800F08200822804D1BDF81030CB
:10A18000013BADF80C30CDB1284604A907F08EF99B
:10A19000BDF90010BDF9022004A84942524204F062
:10A1A00047FE284600F02CF800F48170B0F5817F5E
:10A1B00004D1BDF81230013BADF80E3002AB03CB39
:10A1C0002060616007B0F0BD1FB5039104A914239E
:10A1D00041F8103D694600F001FD05B05DF804FB53
:10A1E0001FB504461022684600210EF001FA15231F
:10A1F00020466946009300F0F1FC039804B010BDBE
:10A2000008B518B106F036F8008D08BD08BD08B5D0
:10A21000034610B106F02EF8C369184608BD37B5DD
:10A220000D4606F031F802ABC46943F8040D184638
:10A2300006F038F820466CB1FFF7D2FFA84220465E
:10A2400008D02946FFF7EBFF20B9204606F012F8A8
:10A25000046AEFE703B030BD08B1FFF7E0BF704715
:10A26000034B1B685A7C034B53F82200704700BF16
:10A27000240100202817022037B50D4658B151B1EE
:10A2800006F002F802AC294644F8040D00F0B5FCD3
:10A29000204606F007F803B030BD0000044B01462D
:10A2A000186810B9034B1B68986CFFF7E5BF00BF37
:10A2B000241702202401002002688368D31A426810
:10A2C000002ABCBF00224260426823EAE3739A423C
:10A2D000C8BF4360704700F0D8BC000073B50546A6
:10A2E000002832D005F0D0FF02AC034644F8080D38
:10A2F000006A08B968460EE09B6A1A0711D405F097
:10A30000C3FF836A02AE1B0746F8040D06D56846F4
:10A3100005F0C8FF304605F0C5FF16E0304605F0F1
:10A32000C1FF009B68469E6905F0BCFF284600F00F
:10A33000B7FA3146284600F061FA284600F0A5FC3D
:10A3400028460349002207F0D0F802B070BD00BFD4
:10A35000D7A200080A4A0B49002313700A4A0B606F
:10A3600013600A4A4B601360094A13605360094A3C
:10A370001360094A1360094A1360094A1360704761
:10A38000F8D7012038170220D0D701205C1702200F
:10A390006417022070170220241702205017022091
:10A3A0006017022010B5044605F064FF836A044A72
:10A3B00013F4803F034B204608BF1346984710BD57
:10A3C00009B20008F5B70008F0B5054685B00C469F
:10A3D0001646002D4CD0284605F056FF876A01909E
:10A3E000BB0701463DD502AD26B12846324603F0F3
:10A3F0006DFF02E003C885E803002046294604F00B
:10A40000CDFC70B317F0010F019B1ED13EB1B3F923
:10A410000220B6F902309A42A8BF134601E0B3F910
:10A420000230B4F902209342B4F9062006DDBDF8EB
:10A430000A3019B28A4214DB013B04E0BDF80E3049
:10A4400019B28A420DDDE3800BE0DF694FB1384677
:10A4500021462A46FFF7B8FF384605F00BFF076A8A
:10A46000F4E704A850F80C3D1D6A05F01BFFB0E7A7
:10A4700005B0F0BD2DE9FF4104460F46904600258A
:10A48000002C37D0204605F0FFFE866A0190B20707
:10A49000014628D502ACB8F1000F04D02046424650
:10A4A00003F014FF02E003C884E8030038462146A5
:10A4B00004F074FCB8B1F30705D4BDF80C300133D7
:10A4C0003B8001250FE0019BDE6966B130463946CD
:10A4D0002246FFF7CFFF0028304618BF012505F0C0
:10A4E000C9FE066AF1E704A850F80C3D1C6A05F0A5
:10A4F000D9FEC5E7284604B0BDE8F081F0B50446B2
:10A5000085B00E461746002C31D0204605F0BCFE23
:10A51000856A0190AA07014622D502AC27B12046E0
:10A520003A4603F0D3FE02E003C884E80300304655
:10A53000214604F033FC98B1EB0704D4BDF8083091
:10A54000013BB3800CE0019BDD694DB128463146EB
:10A550002246FFF7D3FF284605F08CFE056AF4E794
:10A5600004A850F80C3D1C6A05F09CFECBE705B032
:10A57000F0BD00002DE9F341214D2B680646986C93
:10A5800005F082FE0090304605F07EFE02AC0146EA
:10A59000019054F8080D083004F000FC074628B379
:10A5A0000199009A2B68174C1F6DD3F84C8001F16C
:10A5B0000800083203F08AFE684605F073FE019A2F
:10A5C0002B68B2F90010B2F90220D9641A6501A80B
:10A5D000266005F067FE3046FFF7E4FE00232360A7
:10A5E0002B681F65C3F84C80012705E0684605F01D
:10A5F00059FE01A805F056FE384602B0BDE8F081CC
:10A6000024010020241702202DE9F347064605F017
:10A610003BFE836A01909B0705D401A805F042FE2A
:10A6200002B0BDE8F087C469002CF6D0204605F0E2
:10A630002BFE836A02AD03F00303032B45F8080DDC
:10A6400037D10199083104F0A9FB002831D002A8C4
:10A6500050F8043DB3F80890B3F80A809F89B3F826
:10A660000EA005F01FFE684605F01CFE2046FFF711
:10A6700081FF70B1204605F0FDFD00902046FFF7F8
:10A68000C3FF204605F0F6FD0090304605F0F2FDD0
:10A690000190304605F0F8FD0190204605F0F4FDEC
:10A6A000019B0090A3F80890A3F80A809F81A3F86B
:10A6B0000EA0009B68461C6A05F0F4FDB4E700009C
:10A6C00037B5044605F0E0FD826A019040F60103CB
:10A6D0001340012B05D001A805F0E4FD2046FFF74B
:10A6E00061FE144B1B6813B32046FFF78DFF204615
:10A6F00005F0C0FD8569046ACDB194B1204605F02E
:10A70000B9FD836A03F00303032B02D12046FFF750
:10A7100031FF2046FFF778FF204605F0ABFD046AC5
:10A72000EBE7284605F0A6FD046A8569E4E703B077
:10A7300030BD00BF701702202DE9F347174D2B687D
:10A740000646986C05F0A0FD2A68B0F808A0B0F89D
:10A750000A90B0F80C80C78902AC083244F8040DA6
:10A7600000F1080392E8030083E80300204605F0A7
:10A7700099FD3068FFF7A4FF2B68986C05F084FD05
:10A780000190A0F808A0A0F80A90A0F80C80C7815A
:10A79000204605F087FD02B0BDE8F08724010020C7
:10A7A000F7B507460D46284605F06EFD836A02ACF4
:10A7B00013F00206014644F8040D04D1204605F0CA
:10A7C00071FD304616E0384603F0B2FD019B9E69EC
:10A7D000204656B905F066FD074B1A68954208D029
:10A7E00058682B1A5842584104E005F05BFD354685
:10A7F000D9E7012003B0F0BD28170220F0B50446C8
:10A8000085B00D46002949D005F03EFD00230362C6
:10A8100085610190284605F037FD019BC5690290CE
:10A820009F6A2DB9C46101A805F03CFD02A833E080
:10A83000284605F029FD04AE07F0080746F8040D88
:10A8400077B9836A1A070BD5019B1D62029B01A889
:10A85000DC6105F027FD02A805F024FD30461BE071
:10A8600002A805F01FFD304605F01CFD284605F046
:10A8700001FD0390039B1D6A0DB91C620BE0284685
:10A8800005F0F8FC002FF4D1836A1B07F1D5039B78
:10A890001C62019B1D6201A805F004FD05B0F0BD1E
:10A8A00070B5044605F0E6FC05468069A8B105F0E0
:10A8B000E1FCC369A342064605D1184605F0DAFC5F
:10A8C000036AF36170BD43B1184605F0D3FC036A17
:10A8D000A342F8D12B6A036270BD70BD03460846DF
:10A8E000B3F90220B3F9001004F0A2BA114B30B54D
:10A8F0001C68626C85B00546BAB11068516802AB3D
:10A9000003C30D4B186800B9A06C05F0BDFC04AC86
:10A9100002A944F80C0DFFF7E1FF204605F0C2FC48
:10A9200002A8294603F004FD02A802F033FF05B097
:10A9300030BD00BF24010020241702201FB50E4B9C
:10A940001B6893F854200AB10C4811E0986C05F08C
:10A950009BFC019003C802AC84E8030001A805F049
:10A96000A1FC074B196811B12046FFF719FF2046DB
:10A97000FFF7BCFF04B010BD24010020DCD701208C
:10A9800024170220064B10B50446186828B1A042CF
:10A9900004D005F06FFC4069F8E710BD012010BD40
:10A9A0004417022013B5044600B305F06DFC826A1B
:10A9B0000190930717D5406A40B10D4B1B68A34225
:10A9C00004D001F0DFFD019B00225A622046FFF710
:10A9D0001EFC04463CB12046FFF7E4FF204605F08C
:10A9E00049FC046AF6E701A805F05CFC02B010BD62
:10A9F0006C170220B0F90020B0F904309A4208DC4C
:10AA0000B0F90220B0F906309A42CCBF00200120F4
:10AA10007047002070470000F0B585B006460D462F
:10AA2000174605F027FC846A0190A30734D5284611
:10AA3000FFF7E0FF00282FD040F601032340012B51
:10AA40002AD0304605F020FC02AC0246019029468F
:10AA5000204603F03BFC2046FFF7CCFFC8B1019B2A
:10AA60009E6A44F22001314003F1080529B12846CD
:10AA70002946224604F0ECF90BE094E803003E433B
:10AA800085E803009E62054B1A8801321A8003F0A4
:10AA900015FE01A805F006FC05B0F0BD4017022028
:10AAA0002022FFF7B9BFF0B50F4685B01546064620
:10AAB00048B305F0E9FB836A04AC9B07024644F8FF
:10AAC0000C0D03D4204605F0EDFB1CE002A839462E
:10AAD00003F0FCFB0028F5D0204605F0E3FB3046F0
:10AAE00002A92A46FFF798FF3046FFF790FB04467D
:10AAF0004CB1204602A92A46FFF7D5FF204605F0B3
:10AB0000B9FB046AF4E705B0F0BD2DE9FF418046CA
:10AB100017461D460C46002930D0084605F0B4FB08
:10AB2000866A0190B307024625D502A8414603F084
:10AB3000CDFB00B340F601033340012B07D1019B4D
:10AB400002A899691A6A2B46FFF7DFFF04E0204646
:10AB500002A92A46FFF760FF019BDC695CB1BC4299
:10AB600009D0204602A92A46FFF79DFF204605F09E
:10AB700081FB046AF2E701A805F094FB04B0BDE88C
:10AB8000F08170B5054608460C46164605F072FB86
:10AB9000836A13F4803F2846214632460CBF2023A7
:10ABA0004FF48043BDE87040FFF7AFBF2023FFF7AD
:10ABB000ACBF13B5044605F067FB8169019041B154
:10ABC000026AFFF7F3FF2046FFF76AFE019B0022AF
:10ABD0009A6101A805F066FB02B010BD08B106F04D
:10ABE00017BB70471FB504AB019043F8101D6946B1
:10ABF00006F00EFB05B05DF804FB00230B80828895
:10AC00004B800388D31A8B80C2884388D31ACB80A9
:10AC10007047F0B50F4687B00546002833D005F0E1
:10AC200033FB866A0190B2072AD503C804ACF3034C
:10AC300084E8030002D52846FFF7B4FE5FB1386808
:10AC4000796802AB03C3019802A9FFF747FE2046CB
:10AC500002A903F06DFB20462946FFF7A1FD78B15C
:10AC600040F601033340012B06D1019B2046996930
:10AC70001A6AFFF79BFF03E028462146FFF710FF03
:10AC800001A805F00FFB07B0F0BD0021FFF7C1BF21
:10AC900010B5044605F0EEFA80690028F9D1054B9D
:10ACA0001A68944205D05868844214BF4FF0FF30B0
:10ACB000012010BD2817022008B5FFF7E9FF002882
:10ACC00003DBBDE8084004F035B808BD0D4A136841
:10ACD00070B59D6C0446164608B90B4A14689C640E
:10ACE0002046FFF7E9FF03F04DF9204605F0C2FAD0
:10ACF0003368B0F90010B0F90220D9641A6528460B
:10AD000070BD00BF24010020441702202DE9F74F39
:10AD10000C9D9B464B4B0746884692461E6865BB7A
:10AD2000494B1B8863B3494B1B685A7C484B53F80B
:10AD300022305A1C24D01BB31D46284605F0A4FA25
:10AD4000B0F90020B0F90230019017449844BAF1EC
:10AD5000000F05D1B0F904A0C2EB0A0A0AF1010AFA
:10AD6000BBF1000F05D1B0F906B0C3EB0B0B0BF133
:10AD7000010B01A805F096FA02E06B1CDDD100255D
:10AD80000F982C3005F052FD0446002856D00D9B3C
:10AD90001E432D4B1A8801321A8005F075FA0E9B5E
:10ADA00003610DF108092B4B826A49F8080D334005
:10ADB0000780A0F802805744D8441343013F08F1AC
:10ADC000FF3883628780A0F80680684605F06AFA3B
:10ADD000214B186848B105F04DFA0746204605F0AA
:10ADE00049FA7B6943617C6100E01C60294620468A
:10ADF000FFF704FDB50602D52046FFF767FFF00711
:10AE000003D5164B1A6801321A60710602D5204626
:10AE100006F076FBB2070DD5204605F035FA836AB9
:10AE2000009043F002038362684605F03BFA204637
:10AE3000FFF72BFF20460121FFF7D4FE204603B089
:10AE4000BDE8F08F501702202017022024010020B7
:10AE5000281702209F3F3F0044170220701702204E
:10AE600073B5044600286ED0FFF78CFD00286AD029
:10AE70002046FFF70DFF0B2105462046FFF7B2FEE7
:10AE8000204606F028FA204605F0FEF90190406AB7
:10AE900008B101F077FB2D4B2D4A002119602D4B95
:10AEA0001B6852F82300A04208BF42F823102A4A28
:10AEB00052F82310A14204BF002142F82310274B6F
:10AEC0001B682BB15A68A24204BF00225A60F7E700
:10AED00020460721FFF721F8019EF069FFF7C0FF28
:10AEE000F369002BF9D12046FFF763FE1C4B18686D
:10AEF00050B105F0BFF906464069A042F8D120469E
:10AF000005F0B8F943697361019B9B6ADA0703D5C1
:10AF1000144A1168013911609B0603D5124B1A8837
:10AF2000013A1A8001A805F0BDF9104B1A88204695
:10AF3000013A1A8005F0E2F9002D04DB0C4B53F8BE
:10AF40002500FFF7C3FE02B070BD00BFECD70120A3
:10AF50003817022048170220641702205C170220CD
:10AF600044170220701702204017022020170220E9
:10AF7000281702202DE9FF415D4F3B6893F85400EC
:10AF8000002800F0B2805B4B5A69012A1C4603DDA1
:10AF9000013A5A610020A8E004F108061B6996E80E
:10AFA0000300013302AD236185E8030023B9238840
:10AFB000ADF80830638811E0A3896289ADF80A20F2
:10AFC00001339BB2B4F90420ADF808301BB29A42A9
:10AFD00006DA2388ADF80830E3890133ADF80A308A
:10AFE000BDF90A20B4F90630DFF808819A4204DD81
:10AFF0006369013B0020636177E03B68986C05F072
:10B0000043F9BDF90820B8F9003001909A421CD1EB
:10B01000B8F80630ADF80E30B8F80430ADF80C30A2
:10B02000334B1B689A6C5AB1104605F023F98046E1
:10B030000022006A2946FFF7C7F9D8F81820F2E77E
:10B04000019B2946D869FFF7BFF9BDF80830ADF874
:10B050000C303B689A6C6AB1104605F00BF9294632
:10B0600080460022006AFFF705FA0028EDD1D8F8E3
:10B070001820F0E7019B2946D869FFF7FBF9002863
:10B08000E3D1A388BDF90820ADF80C301BB29A4279
:10B0900007DD95E8030086E8030001A805F002F942
:10B0A00097E73B689A6C52B1104605F0E3F8074603
:10B0B0000022006A2946FFF721FABA69F3E704AFD4
:10B0C000294657F80C3DD869FFF718FA384605F0BD
:10B0D000E9F8236944F62062934289DC95E803008D
:10B0E00086E80300FFF72AFC012004B0BDE8F081E8
:10B0F00024010020D4D701202DE9F041394F3B68CD
:10B1000093F8542086B0064612B9FFF717FC64E0A6
:10B11000354D6A690132012A6A612C465DDC986C02
:10B1200005F0B2F84FF0FF322A61304A00901278F1
:10B130002AB100F1080302AA93E8030005E0826A3D
:10B1400012F002080AD003C802AA82E8030002AD86
:10B1500066B12846314603F0EBF807E06B696846B4
:10B16000013B6B6105F09EF8404637E03B68204E9E
:10B170005A6CC2B1009B10685168019304AB03C3C1
:10B18000336833B101A805F08DF8306805F07CF81C
:10B190000190019804A9FFF7A1FB284604A903F038
:10B1A000C7F801A800E0684605F07CF8316819B1DD
:10B1B0002846FFF7F5FA28B13B682846996CFFF757
:10B1C000EFFA18B96369013B636107E095E8030092
:10B1D00084E80300FFF7CEFE00E0012006B0BDE8E2
:10B1E000F08100BF24010020D4D701204D17022098
:10B1F0002417022008B503F067FD024B1B680022EC
:10B200005A6408BD24010020F0B589B0044605F059
:10B210003BF80769866A0190083003C802AD85E8EB
:10B22000030001A805F03EF8002F31D0B3072FD559
:10B2300020462E21FEF7F4FD164B1A7816F4805F97
:10B2400002F101021A701E460AD00F2305940493DE
:10B250000795FFF7CFFF204604A905F0D9FF10E0BE
:10B260002846FFF749FF60B10F2304930594079523
:10B27000FFF7C0FF204604A905F0CAFFFFF77AFEDA
:10B28000F1E733782046013B2F213370FEF7C8FDEC
:10B2900009B0F0BD4D170220F0B589B006AC03909F
:10B2A00004F0F2FF00F108020346059092E8030063
:10B2B0009D6A9E691F6984E8030005A804F0F2FFF7
:10B2C00044F220032B40002B34D0BFB12046039919
:10B2D000FFF766FA90B10398FFF7F8FC69070FD5FE
:10B2E00026B105F0010585F0010500E00125009576
:10B2F0002046124903AA002300F0DAFA002403E0F2
:10B300000398FFF7DDF90124039804F0BDFF826A7A
:10B31000059022F4804323F02003920448BF43F0B9
:10B320000403836205A804F0BDFF054B1A88013AA7
:10B330001A8000E01C46204609B0F0BD39A700087D
:10B340004017022008B504F095FF836A43F40043D8
:10B350008362024B01221A6008BD00BFD0D70120D2
:10B360002DE9F04F4C4B1B689FB003B19847002666
:10B370004A4D2B68DBB14A4B1C68BCB1204604F037
:10B3800083FF826A47691EAB12F4004F43F8700DC9
:10B3900007D0184604F086FF2046FFF761FD3C46C3
:10B3A000EBE718463C4604F07DFFE6E72C603D4B9A
:10B3B0001B6803B198473C4B1B682BB93B4F3B685C
:10B3C00093F8543043B103E098470028F6D058E092
:10B3D00003F012FD002854D13B6893F854504DB14E
:10B3E000334B1D8835B1334B1B68002B4BD01B688A
:10B3F000984701253B6893F8543013B9002D37D195
:10B4000045E0DFF8AC80B8F80030002BF6D0DFF86C
:10B41000A890D9F800400CB9214B1C6802A803F091
:10B42000A9FC3B68D3F830B0D3F834A014B9002499
:10B430000DE063B92046FFF72FFF03462046019336
:10B4400004F018FF4469019B002CF2D1EFE7584645
:10B45000C9F8004003F05AFC504603F055FC02A81E
:10B4600003F092FCB8F80030002BC7D00126C1E7EA
:10B47000104B186810B14368984708E002F01EFFAF
:10B4800005E0012674E7012002F018FFB1E730461D
:10B490001FB0BDE8F08F00BF34170220D0D70120C5
:10B4A0004417022030170220B01702202401002088
:10B4B0004017022060170220ECD70120024B1B68C6
:10B4C000012283F85420704724010020034B1B689D
:10B4D000002283F8542002F055BD00BF2401002053
:10B4E00010B5044640682368E168172B0FD006DCCE
:10B4F0000E2B0ED0142B14D1FEF7BEFE11E0222B22
:10B500000CD0282B0DD1BDE81040FFF7BEBBE0608A
:10B5100010BD2146BDE8104005F0A0BF6FF070439C
:10B5200000E00023E36010BD03680E2B10B5044655
:10B5300002D00F2B09D020E0C3685A68012A21D11C
:10B540001868BDE8104003F04FBC0F4A436811680B
:10B550008B4206D05268934214BF4FF0FF33012351
:10B5600000E00023094A52F823006FF0704398422C
:10B5700003D003F0C9FB04F057FA2046BDE81040A1
:10B58000FFF7AEBF10BD00BF2817022054170220DE
:10B5900030B52B4B187885B01D4600284DD1294B6E
:10B5A0001860294B1860294B1B685864284B188079
:10B5B000284B04461880204604F012F9C0B14FF021
:10B5C000FF3202238DE80C00002043F6FF72224B6D
:10B5D0000293039013460146FFF798FB1F4B43F875
:10B5E00024001F4B6FF0704243F82420FFF74DFBFF
:10B5F0000134022CDFD11B4805F07AFF1A4805F010
:10B6000077FF1A4805F074FF194805F071FF1948D3
:10B6100005F06EFF184805F06BFF104B1868FFF738
:10B6200055FBFFF74BFF01232B701448144B0360AD
:10B6300005B0BDE8304004F007BA05B030BD00BF2A
:10B64000F8D7012044170220ECD701202401002064
:10B65000401702202017022029B5000828170220D1
:10B660005417022094180220841802207418022013
:10B670009C1802208C1802207C180220F0D7012090
:10B6800055A300082DE9F04F87B0044604F0FCFDF7
:10B6900006AFB0F800808688B0F80290B0F806B027
:10B6A00047F8040D0FFA88F836B2C8EB0606D0F852
:10B6B00024A0013638460FFA89F90FFA8BF504F009
:10B6C000F1FDC9EB0505002E05F101054DDD002D4D
:10B6D0004BDDBAF1000F4AD0504604F0D5FD06AB61
:10B6E000868843F8080DC58836B2184604F0DAFD9E
:10B6F000464502D12DB24D4532D0504641464A46CC
:10B7000000F086F82CE0836A43F480338362384685
:10B7100004F0C8FD404600F093FF0746504603F092
:10B72000F7FA404600F0B4F82D4B05FB06F2197805
:10B730002C4D2D4E920002F015FD2046D5F80080CC
:10B740003460FEF7CCFC28602046FFF75DFD00204A
:10B75000C5F80080306003F0DBFA384600F070FF77
:10B76000204604F087FD406A37E0002035E0FEF710
:10B7700077FD844212D102F09FF8824602F0A4F8CD
:10B78000564502DC854209DD00E056468542A8BFE9
:10B790000546314620462A4605F008FE134B019324
:10B7A0004FF0010A124B02934046494632462B465F
:10B7B000CDF800A000F04EFE8046204604F064FD67
:10B7C0000590C0F82480B8F1000F9CD1384604F0F1
:10B7D00069FD2046FFF718FD404607B0BDE8F08F31
:10B7E0000C0100207C1702206C170220BCC8010845
:10B7F00094F3010838B5054605242846FFF742FFB3
:10B8000010B9013CF9D138BDBDE8384006F086BB1F
:10B8100037B50D46144618B9114B1B68186EE8B1C0
:10B8200004F032FDA4B2ADB2C4808580009002F075
:10B83000A9FB009B586970B104F026FD009B0190A4
:10B840001A895B898280C38012B10BB10580448064
:10B8500001A804F027FD684604F024FD03B030BDC4
:10B860002401002013B520B9084B1B68186E04464C
:10B8700048B104F009FD02ABB0F90A4043F8040DE9
:10B88000184604F00FFD204602B010BD2401002030
:10B8900013B550B104F0F8FC044602A840F8044D7A
:10B8A00004F000FD04F11800FFE702B010BD000035
:10B8B0002DE9F04F1E4689B04E4B04921A68039151
:10B8C000547C4D4A1257012A05469B46204606DD08
:10B8D00001F0E0FF0746204601F0DFFF05E001F040
:10B8E000DFFF0746204601F0DEFF044625B306A829
:10B8F00007A903F0F1FA069BB5F900A0B5F90420F9
:10B90000B5F902801F44079B2AEAEA7A013F974271
:10B91000D4BFCAEB0707CAEB02071C44B5F90620DF
:10B9200028EAE878013C9442D4BFC8EB0404C8EB91
:10B9300002040137013401E0A846AA4606B966426E
:10B94000002F52DD002C50DD129B009350464146E3
:10B950003A46334600F038FE054620B90498039B6A
:10B960009847012042E0FFF77DFFA042064606D03F
:10B97000DBF80030986C10B1322105F035FC284618
:10B9800000F05EFE73420593A1460027B14503DA3D
:10B990002846494606F0C2FB47B12846514607EB08
:10B9A0000802FFF735FF284606F0CEFB039B0498FC
:10B9B0009847124B1B680BB100209847284600F0AF
:10B9C000B7FE3744059BA7429944DFDB284600F0C9
:10B9D000D9FD002000F034FEA64206D0DBF800308E
:10B9E000986C10B1332105F0FFFB002009B0BDE8D1
:10B9F000F08F00BF2401002074170220FCD7012023
:10BA00000248012918BF0020704700BFBCC80108C8
:10BA10000248162918BF0020704700BF2D1D0108DD
:10BA200008290CBF20200020704708B50068C368B3
:10BA30001B6A984708BD37B580680C4604F024FCA3
:10BA4000034602A89988DA881D8940F8043D5B897D
:10BA50002180628029441A440139013AA180E280A0
:10BA600004F020FC03B030BD0E4B1B6873B50546D7
:10BA7000186E0E4604F008FC034602A8B3F906400F
:10BA800040F8043D03F11801361BDC68B3F90430BB
:10BA900004FB0614ED1A04F005FC04EB85042046B3
:10BAA00002B070BD2401002008B508461146FFF71A
:10BAB000DBFF006808BD0000154B1B6873B5186EEE
:10BAC00015460E4604F0E0FB294600903046FFF78D
:10BAD000CBFF009B1B681B6904469B689847236843
:10BAE0005840009B2060586960B104F0CDFB02AC67
:10BAF000836844F8040D1B6831462A46984720465F
:10BB000004F0D0FB684604F0CDFB02B070BD00BF6E
:10BB10002401002073B51C46104B1B68186E0E469E
:10BB2000154604F0B1FB294600903046FFF79CFF14
:10BB3000009B0460586960B104F0A6FB02AC836806
:10BB400044F8040D1B6831462A469847204604F005
:10BB5000A9FB684604F0A6FB02B070BD24010020DA
:10BB60002DE9F7432C4D1E462B68186E0F461446E0
:10BB700004F08AFB00904069A94608B104F084FBF8
:10BB8000019021463846FFF76FFFD9F80020009B4F
:10BB9000D16B127CD3F80C80D1F80090D207054607
:10BBA0001FD51B681B699B6898478046019828B180
:10BBB00082683946D2F800C02246E0472B6883EA03
:10BBC00008032B60009B0134DB68B4421D44EDDDAB
:10BBD000684604F067FB019BD3B101A804F062FB47
:10BBE00016E0019B63B10198836822461B683946C1
:10BBF00001349847B442C5F800904544F3DDE7E7C7
:10BC0000341B0134013CC5F800904544FAD1DFE70C
:10BC100003B0BDE8F08300BF240100202DE9F04F00
:10BC2000DFF8ACB01446DBF8002085B0106E0F468C
:10BC30001D4604F029FB214602903846FFF714FF09
:10BC4000029ADBF80030D2F80C90DB6B06465069A4
:10BC5000D3F800A0ED1B013538B304F015FB0E9AA4
:10BC60000DF11008131B48F8040D013300933946F9
:10BC700022462B4606F03CFA404604F013FB14E043
:10BC8000DBF800301B7CDB0713D5029B1B681B69AC
:10BC90009B68984732462B461168013B81EA0001B8
:10BCA00042F8041BF8D14E4401340E9B9C42E7DD60
:10BCB00008E0002DF7DD2B463246013B42F804AB8D
:10BCC000FBD1F0E702A804F0EDFA05B0BDE8F08F73
:10BCD0002401002007B50092FFF7A0FF03B05DF834
:10BCE00004FB00002DE9F04F9D4C9A46236891B06B
:10BCF0008046186E07920E46DDF874B01F9D00282E
:10BD000000F0878304F0C0FA0E90406908B104F097
:10BD1000BBFA0F9010A850F8083DDB680A9304F0B6
:10BD2000C1FA1E9F0F983744049750B123681B7CBB
:10BD30009C0706D41A9F00970499079A534606F069
:10BD4000D7F904980799FFF78FFE1B9F172F064618
:10BD500064DD4FEA8A0706974FF000091A9F0F9893
:10BD6000B94557DA30B18368079A5C6804994A4448
:10BD70005346A047D8F81030D86828B13046594605
:10BD8000069A0CF00DFC3EE05B689847000E0590AB
:10BD9000354657465C463B4622464FF0000C52F86B
:10BDA000041B0598090E8142059808BF0CF1010C8F
:10BDB000814203F1FF3314D0BCF1000F14D04FEADD
:10BDC0008C03284621461A460393CDF808C00CF090
:10BDD000E7FB039BDDF808C01D441C44CCEB0707C0
:10BDE0000FE0002BDBD1E7E72068020EFF2A05D029
:10BDF000D2432968D2B202F0B9FA2860043504347B
:10BE0000013F002FC7D11C9FBB440A9F09F10109C4
:10BE10003E44A3E7002840F0F982FAE21B9F102F6E
:10BE200037D1061F00251A9F0F9CBD4280F2A080CB
:10BE3000079F2F443CB1A3680499D3F804C020465F
:10BE40003A465346E047ABF1020306930596D146C6
:10BE50000499D8F81030069A5B6832F8020F0692FF
:10BE60005144C9EB010103919847059B039943F89D
:10BE7000040F059324B1A36820461B683A469847EF
:10BE8000B9F10109E4D11C9FBB440A9F01353E442E
:10BE9000C9E71B9F082F00F104066DD1079F079982
:10BEA0001A9A0F9C7B1A9342A6F1040060DA2C4B7D
:10BEB0001B681B7C6DB313F0030305D0022B51D11B
:10BEC000B146DDF810801CE01BF8032055F8222055
:10BED00040F8232001335345F6D143E055F8233091
:10BEE00049F8043C2CB1A36820461B6841463A46F9
:10BEF0009847049B08F101085344434509F104099C
:10BF000030D00498C0EB0B0313F80830002BF0D0AE
:10BF1000E4E713F0030305D0022B23D1B146DDF88B
:10BF2000108015E0594652460CF03AFB1AE049F8E9
:10BF3000043C2CB1A36820461B6841463A4698470A
:10BF4000049B08F101085344434509F1040909D051
:10BF50000499C1EB0B0313F80830002BF0D0E6E78F
:10BF6000240100201C9A0A9B934401371E4496E743
:10BF7000002C40F04B824CE21E9FB24B09967F0092
:10BF80000C971E9FBF000D97079F0597002D08BFB8
:10BF90001D46099F07983C1F059F3B1A1A9FBB42ED
:10BFA00080F232821B9F022F00F0AD80042F00F040
:10BFB0004F81012F40F01E82DFF89092D9F80030B7
:10BFC000186E04F061F99BF800309F4A1E99D65C08
:10BFD000D9F800300E901B7CDDF83CC003F0030361
:10BFE000022B5746C1F1080846FA01F620D0032B70
:10BFF00061D0012B5FD05A46474538BFB846C8EBE1
:10C0000007074346214606F00100013B55F8200092
:10C0100041F8040B4FEA5606F5D104EB8804002FD3
:10C020006DD012F8013F88494FF00808CE5CE3E775
:10C030006B68DDF810900B93CDF820B0474538BF02
:10C04000B846C8EB0707BCF1000F26D01EB904EBB9
:10C050008804C14425E0F0070CD5DCF80830059AC7
:10C060001B68CDF808C06046494698470B9BDDF831
:10C0700008C02360B8F1010809F1010904F10404C2
:10C080000FD07608E2E7F10744BF0B9B2360B8F1BD
:10C09000010804F1040404D07608002EF3D104EB67
:10C0A000880467B30898684A10F8013F0890D65C86
:10C0B0004FF00808C2E703681B699B689847594618
:10C0C000474538BFB846C8EB0707231DC646F207E9
:10C0D00004D553F8042C424043F8042CBEF1010E61
:10C0E0004FEA560603F10403F1D104EB880437B19B
:10C0F00011F8013F544A4FF00808D65CE0E70EA85B
:10C1000004F0D0F876E11E9F0C9BDDF83CC0C7F12F
:10C1100004069BF800709F404C4B1B681B7C03F08F
:10C120000303012BF6B2FFB266D008D3022B40F016
:10C1300061810498CDF820B0D04606903EE05A4682
:10C1400053469E42C8BFDEB29B1B314620464FEA93
:10C15000971C013955F82CC040F804CBBF0011F0F2
:10C16000FF01FFB2F3D1013EF6B2013604EB8604C3
:10C17000002B00F03F8112F8017F0426E1E70699C9
:10C1800017F0C00F494422D109F101095FFA89F281
:10C19000BF009642FFB2F2D1069F013EF6B27B1C71
:10C1A000721C9E1904EB82040696B8F1000F00F091
:10C1B0002181089B13F8017F089304264645C8BFD8
:10C1C0005FFA88F6C6EB08084FF00009D7E7BA090E
:10C1D00055F8222044F82920BCF1000FD4D0DCF817
:10C1E000082012680B926046CDF808C0059A0B9B98
:10C1F0009847DDF808C0C7E7584653469E42C8BF77
:10C20000DEB29B1B221DB44617F0C00F05D052F8BA
:10C21000041C81F0FF0142F8041C0CF1FF3CBF003C
:10C220001CF0FF0CFFB202F10402EDD1013EF6B2A8
:10C23000013604EB8604002B00F0DC8010F8017F4F
:10C240000426DBE77CC80108FCF10108240100207A
:10C25000714A9BF8003012680D98127C0F9F02F013
:10C2600003028340012ADEB200F09C8002D3022A3E
:10C2700035D0BFE01E9F5FB136090BF1010255F8C2
:10C28000263023609BF80160099C0AF1FF3301E02E
:10C2900053465A46012B1ADD581004F1080103F0E9
:10C2A000010302EB00084FEA161C06F00F0655F8D2
:10C2B0002C7041F8087C55F8266041F8046C12F89F
:10C2C000016F424501F10801EDD104EBC004002BE0
:10C2D00000F09080360955F8263023608AE01E98D9
:10C2E000C0B113F0F00F0AD0360955F8263023609C
:10C2F0002FB1BB6804991B68059A38469847049982
:10C30000099C9BF8016001F101080AF1FF3C0BF167
:10C31000010911E0D446D946DDF810800CE016F092
:10C32000F00F0DD116F00F061BD119F8016F08346C
:10C3300008F10208ACF1020CBCF1010FEFDC21E0C6
:10C34000330955F823302360002FEBD0BB68059AE2
:10C350001B68CDF808C0384641469847DDF808C04C
:10C36000E0E755F826306360002FDED0BB68059A01
:10C370001B68CDF808C0384608F101019847DDF880
:10C3800008C0D2E7BCF1000F34D0360932D055F8DE
:10C390002630236077B3BB68059A1B683846414650
:10C3A000984727E01E9FC7F10203DBB25F46524663
:10C3B0009342C8BFD3B2D21A201D9C4616F0C00FBC
:10C3C00005D050F8041C81F0FF0140F8041C0CF16A
:10C3D000FF3C36011CF0FF0CF6B200F10400EDD179
:10C3E000013BDBB2013304EB83041AB117F8016F90
:10C3F0000223DDE7059B1C9F0133BB4405930A9F85
:10C40000099B3B440993C4E50F9B13B10FA803F0AC
:10C4100049FF11B0BDE8F08F240100202DE9F34160
:10C420000E469046074603F02FFF036802ACDB6818
:10C4300044F8040D5B6A0020162198470546204603
:10C4400003F030FF1DB1384631464246A84702B0DE
:10C45000BDE8F0812DE9F04F3E4E87B01D463368B0
:10C46000109F5B7C83468A46904611981299002261
:10C4700003F0C8F90446002833D003699B68984745
:10C4800001F0BFFA08FB00F60390073604F0C4F889
:10C4900017F001094FEAD60604D1042390FBF3F00C
:10C4A00000EB4000002D09DC1EB11838B0FBF6F09F
:10C4B00000E030466D42A842B8BF0546B9F1000F12
:10C4C00009D1CDF800905846514642462B4605F01A
:10C4D000CFFD074600E00027002D04DC204603F0D6
:10C4E0008FF9002032E006FB05F01830B9F1000F9B
:10C4F00002D004F01DF901E004F098F9814640B93A
:10C50000204603F07DF9002FEBD0384603F0F6FE0D
:10C510001BE003F0B9FE034606A8039A40F8043D69
:10C520001A611C60A3F804B0A3F806A0A3F8088061
:10C530005D81DE605F6103F0B5FE064A129B2361F8
:10C540001368C4F808905B7CA361484607B0BDE857
:10C55000F08F00BF2401002037B5054670B103F00D
:10C5600093FE036802AC1B6944F8040D9B6898476E
:10C5700001F047FA0546204603F094FE284603B032
:10C5800030BD000037B50446D0B10E4B1B681B6EA2
:10C59000834201D102F0E4FB204603F075FE0190D6
:10C5A000406908B105F090FD02AD55F8043D1868EA
:10C5B00003F026F9284603F075FE204603F09EFEA0
:10C5C00003B030BD240100202DE9FF479A46194BE6
:10C5D0000C9D1B680746587C174B53F82040884633
:10C5E0009146E3681B68042B06D02468002CF8D120
:10C5F00003F0F6F8044630B1E3682046DB6A012117
:10C600009847064608B9002010E02469A3689847B7
:10C61000013004BF45F00105084C02948DE860002C
:10C62000384641464A465346FFF714FF04B0BDE87A
:10C63000F08700BF24010020A417022094F3010812
:10C64000114BF7B51A680446166E1F4610B902F072
:10C6500087FB16E00EB102F083FBFEF737FF2046A2
:10C6600003F012FE02AD3B6845F8040D1C6600683D
:10C6700003F004F9284603F015FE01F079F801F003
:10C6800081FC304603B0F0BD240100202DE9F043C9
:10C690000C4685B015460646002841D0002002F021
:10C6A00011FB214B1B6807463046D3F8608003F02E
:10C6B000EBFD03680190986902F03CFB1B4B9C4228
:10C6C000019B04BFB3F90440B3F906501A895B8992
:10C6D000ADF80840013A013B22442B448146ADF8B5
:10C6E0000C20ADF80E30ADF80A50FEF7E7FE01A8B9
:10C6F00003F0D8FD02A8FEF7FFFC48B9484602F057
:10C7000019FB4046FFF79CFF384602F0DBFA07E0D2
:10C71000304621462A4604F077FFFEF72BFCECE773
:10C7200005B0BDE8F08300BF2401002001F0FFFF49
:10C7300001490A46FFF7AABF01F0FFFFF8B504461A
:10C740000E46D0F88C302A2115469847E16AD4F875
:10C75000903031442046C1F30F219847E16AD4F864
:10C760009030B7B239442046C9B29847E16AD4F84C
:10C77000903031442046C1F30F219847E16AD4F844
:10C78000903039442046C9B29847D4F88C302046BE
:10C790002B219847216BD4F8903029442046C1F3CF
:10C7A0000F219847216BD4F89030AEB23144204627
:10C7B000C9B29847216BD4F8903029442046C1F380
:10C7C0000F219847216BD4F8903031442046C9B2EC
:10C7D0009847D4F88C3020462C219847F8BD2DE995
:10C7E000F041044688461F462A21D0F88C30069D29
:10C7F00016469847E16AD4F8903041442046C1F388
:10C800000F219847E16AD4F8903041442046C9B2DC
:10C810009847E16AD4F8903039442046C1F30F219B
:10C820009847E16AD4F8903039442046C9B2984715
:10C83000D4F88C3020462B219847216BD4F89030C7
:10C8400031442046C1F30F219847216BD4F8903032
:10C8500031442046C9B29847216BD4F8903029441E
:10C860002046C1F30F219847216BD4F8903029441A
:10C870002046C9B29847D4F88C3020462C219847DE
:10C88000BDE8F08113B50D4A0446516810686B4647
:10C8900003C3D4F88C30204636219847636BA18CB3
:10C8A00002AA134421F0E00113F8083C1943204682
:10C8B000D4F8903089B2984702B010BD80F10108D9
:10C8C00013B50446D0F80C312E209847216AD4F8CD
:10C8D0002831684603319847226A00AB13441DF89B
:10C8E000022059789878D2088908D20242EA411287
:10C8F00042EAD00002B010BD1FB50446D0F82C317A
:10C900002E209847216AD4F848316846023198476A
:10C91000236A00A901EB43023DF81300528802F498
:10C920007C41C2F3C40242EA511200F0F80042EA2C
:10C93000002004B010BD38B504460D46D0F80C31C7
:10C94000080A9847D4F80C31E8B2984738BD08B5C2
:10C95000D0F82C310846984708BD08B5D0F81031FA
:10C96000C8B2984708BD08B5D0F830310846984796
:10C9700008BD0000082902D0102905D07047064BD9
:10C98000C0F88C30054B03E0054BC0F88C30054BEC
:10C99000C0F89030704700BF37C900085BC9000875
:10C9A0004FC9000867C90008F0B585B084680A9FC0
:10C9B0000097BD1A581A013500FB0555D4F8A87028
:10C9C0000B9E2046B847D4F80C312E209847D4F857
:10C9D0002831216A02A89847D4F8283102A80321F7
:10C9E00098479DF808309DF80920DB089208DB0283
:10C9F00043EA42139DF80A20013D43EAD20326F898
:10CA0000023BE9D105B0F0BDF0B587B084680C9F5A
:10CA10000097BD1A581A013500FB0555D4F8A870C7
:10CA20000D9E2046B847D4F82C312E209847D4F8D4
:10CA30004831216A02A89847D4F8483102A8022157
:10CA40009847BDF80A3003F47C42C3F3C40343EAB9
:10CA50005213BDF8082002F0F80243EA0223013D18
:10CA600026F8023BE8D107B0F0BD000010B504463F
:10CA700000F0A6FDA368124AC3F8AC20114AC3F81F
:10CA8000A820114AC3F8B020104AC3F8B8200022E9
:10CA9000C3F8BC20C3F8CC200D4A0E491268C3F875
:10CAA000C420DA8C0968C3F8B41022F003020A49E2
:10CAB000DA840A4AC3F8C810C3F8942010BD00BF36
:10CAC0003DC70008DFC7000885C80008C1C80008C6
:10CAD0001401002010010020A9C9000875C9000830
:10CAE00008B5D0F8B430984708BD08B5D0F8303153
:10CAF00088B2984708BD00002DE9F04F3D4F84688B
:10CB000082463868007C10F0010F85B00E4615464D
:10CB10009846C1EB030945D04FEA490B0E98854270
:10CB200065DCD4F8C4C0E76EBCF1000F01D1B44697
:10CB300007E08DE8A000504631462A464346E047CC
:10CB400011E0C4450EDCD4F8EC30CDF80CC06146E1
:10CB500050462A469847DDF80CC027F8020B0CF126
:10CB6000010CEEE7E76EBB1E09F1010C5F44BB420E
:10CB700005D0A26A59884A4023F8022FF7E70095AA
:10CB80002A46D4F8A870CDF80CC02046314643465A
:10CB9000B847DDF80CC0D4F83831E06E61469847EC
:10CBA0000135BBE70E980090851AD4F8A86020469E
:10CBB000B0473B68A76EDB6B09F10109D3F8008031
:10CBC00005FB0995012395B1FA2D34BF2E46FA26AF
:10CBD0002BB138461FFA88F1324601F095FAD4F8A5
:10CBE0003831384631469847AD1B0023EBE705B096
:10CBF000BDE8F08F240100202DE9F04F8DB085684D
:10CC0000179F05937B1E012B099008910A920B95A3
:10CC100003D9042F01D0082F06D18F4B1B681B7C32
:10CC200003F00303022B10D00A9A169F1A9D08994D
:10CC3000059B3A442944013A0B9D00920B44D5F8D8
:10CC4000A8400A9A2846013BA047DDF828B00A9F71
:10CC5000169DC7EB0B03AB4280F25182179F7B1EE0
:10CC60000F2B00F24582DFE813F01000B7004302FB
:10CC70004001430243024302D701430243024302FD
:10CC800043024302430243023D02734B099D1B686A
:10CC9000AC681B9D1B7C2F686D680795DDF820A094
:10CCA0001A9D03F00303022BAA441BD0032B6ED062
:10CCB000012B6CD0059EDDF8648098F80010D4F844
:10CCC000303180222A41114216BF0799B8B288B28A
:10CCD00001359847082D04BF08F101080025013EE1
:10CCE000EBD105E2199D0695D4F86C90DDF86880CB
:10CCF000CDF80CA0002556462B46069F4FF0800C21
:10CD00003A784CFA08FC12EA0C0C0BD013B9D4F8A0
:10CD10006C900396079FA9F80070013509F102098C
:10CD2000012317E0012B14D1CDF800B0CDF810C0CD
:10CD300020460399D4F8A8705A46731EB847D4F811
:10CD40003831E06E29469847DDF810C065466346E5
:10CD500000E0634608F10108B8F1080F06F101068A
:10CD600004D1069F013706974FF00008059A5244F8
:10CD7000B242C2D1059F7B1E5344002D00F0B88102
:10CD8000CDF800B0D4F8A860039920463DE1DDF865
:10CD900014801A9E199DDDF814902A78802333415F
:10CDA000D1441A42C8EB09090DD0D4F8EC300998E7
:10CDB00049465A469847A36AD4F8F070434049461A
:10CDC00009985A46B8470136082E04BF0135002697
:10CDD000B8F10108DFD18BE1099D1B9FAC68002FE2
:10CDE00000F086811C4B199D1B6895F800A01B7CE8
:10CDF00013F0030311D0022B40F07A811A9DDDF865
:10CE00002090E76E0397A944A846199D0795002531
:10CE1000CDF818904E462B4640E01A9D059E199F6E
:10CE2000C5F103035B00C3F10602C02141FA02F21F
:10CE300002EA0A02DA401B99D4F8303131F82200B4
:10CE400001359847042D03D197F801A0002501373B
:10CE5000013EE5D14CE100BF2401002013B9E76E8B
:10CE6000039706961B9F57F82C30039F3B80023791
:10CE700001350397012308F10108B8F1040F06F109
:10CE8000010606D1079F97F801A0013707974FF0D9
:10CE90000008059A4A44B24200F0AC80C8F103028F
:10CEA0005200C2F106014FF0C00C4CFA01FC0CEA32
:10CEB0000A0C3CFA02FCD1D1012B14D1CDF800B000
:10CEC000CDF810C020460699D4F8A8705A46731EB3
:10CED000B847D4F83831E06E29469847DDF810C0DD
:10CEE00065466346C7E76346C5E7099D1B9FAC6877
:10CEF000002F00F0FD80834B199D1B6895F800A062
:10CF00001B7C13F0030311D0022B40F0F1801A9D1B
:10CF1000DDF82090E76E0397A944A846199D079570
:10CF20000025CDF818904E462B463CE01A9D059EF4
:10CF3000199FC5F101039B00C3F10402F02141FADE
:10CF400002F202EA0A02DA401B99D4F8303131F8D1
:10CF5000220001359847022D03D197F801A0002542
:10CF60000137013EE5D1C3E013B9E76E039706969A
:10CF70001B9F57F82C30039F3B80023701350397E6
:10CF8000012308F10108B8F1020F06F1010606D1EC
:10CF9000079F97F801A0013707974FF00008059AFF
:10CFA0004A44B24226D0C8F101029200C2F1040103
:10CFB0004FF0F00C4CFA01FC0CEA0A0C3CFA02FCB3
:10CFC000D2D1012B14D1CDF800B0CDF810C020463D
:10CFD0000699D4F8A8705A46731EB847D4F8383169
:10CFE000E06E29469847DDF810C065466346C8E7FD
:10CFF0006346C6E7059F7B1E4B44002D78D0CDF8D5
:10D0000000B0D4F8A860069920465A46B047D4F834
:10D010003831E06E29466AE0099D1B9FAC68002FFD
:10D0200066D0384B1B681B7C13F0030309D0022B1E
:10D030005ED1DDF82090D4F86C8000264F46334650
:10D0400022E0199D199B059F3B445B1B002B4FDD84
:10D0500015F8012B1B9FD4F8303137F82200984780
:10D06000F0E713B9D4F86C80B9461B9D55F82A3007
:10D07000A8F80030013608F102080123089A059D3E
:10D0800001372A44BA421CD0199D08982A1A12F86E
:10D0900007A0BAF1000FE4D1012B10D1CDF800B0F8
:10D0A000204649465A467B1ED4F8A850A847D4F8D3
:10D0B0003831E06E3146984756465346DEE75346D0
:10D0C000DCE7089F6B1E3B4496B1CDF800B02046CC
:10D0D0004946D4F8A8505A46A847D4F83831E06EEB
:10D0E000314604E00B9D1998D5F8383105999847D9
:10D0F000199F189D2F4419970BF1010BA7E50DB04F
:10D10000BDE8F08F2401002010B5044600F058FA65
:10D11000A468104BC4F8E4300F4BC4F8E8300F4B50
:10D12000C4F8EC300E4BC4F8F0300E4BC4F8A0300D
:10D130000D4BC4F8A430D4F8C430C4F8FC302046F9
:10D14000D4F89430102198471023A363074B6364ED
:10D1500010BD00BFF9CB0008F9CA00080FD50008C0
:10D160007FD40008E1CA0008EBCA000820F40108D7
:10D17000084670470068401A0138704708467047F3
:10D180000068401A01387047104670474068801A9E
:10D1900001387047104670474068801A0138704760
:10D1A00010467047104670474068801A0138704733
:10D1B0004068801A01387047084670470846704733
:10D1C0000068401A013870470068401A01387047FB
:10D1D00010B58468D4F8F040A04710BD08B5836846
:10D1E000D3F8EC30984708BDF7B504460F4616460D
:10D1F0008568FFF7F3FF0190DDF804E0AB6A204695
:10D20000394632468EEA0303FFF7E2FF03B0F0BD72
:10D2100013B584680092D4F8E840A04702B010BD6E
:10D2200013B584680093D4F8E8400B46A04702B0D9
:10D2300010BD37B5069C85680094D5F8E840A04736
:10D2400003B030BD30B587B085680A9C00940B9C54
:10D2500001940C9C02940D9C03940E9C04940F9CCE
:10D260000594D5F8E440A04707B030BD70470000F2
:10D2700073B5079E84680C4D76B1286888B9069806
:10D280000090D4F8A8602046B047D4F8A8302B60AE
:10D29000064BC4F8A83004E02B6813B1C4F8A830DA
:10D2A0002E6002B070BD00BF00D801206DD2000812
:10D2B00008B5026CD0F8D4309069984708BD08B51D
:10D2C000026CD0F8D8309069984708BD2DE9F74333
:10D2D0000A9D8468009517462046D4F8A8609946B0
:10D2E0008846ED1BB047216CD4F8DC3088690B9977
:10D2F000C8EB09086A1C08FB0222984703B0BDE886
:10D30000F0832DE9F7430A9D84680095174620466F
:10D31000D4F8A86099468846ED1BB047216CD4F834
:10D32000E03088690B99C8EB09086A1C08FB0222E7
:10D33000984703B0BDE8F0830139172924D8DFE806
:10D3400001F01023232323232323230C250E15234D
:10D35000232323232323231F1A210D4870470D481D
:10D36000704703689B68D3F8FC00704703689B68AC
:10D37000D3F8F400704703689B68D3F8F80070474F
:10D3800005487047054870470020704704487047BB
:10D39000EFD6000891D60008F5D5000871D2000834
:10D3A000DBD60008013980680D2923D8DFE801F0B9
:10D3B000090B0D0F2222221107252513181D00200D
:10D3C0007047006870474068704780687047C06861
:10D3D0007047806B704788B1406B00F00100704768
:10D3E00060B1406BC0F34000704738B1406BC0F390
:10D3F000800070474FF0FF3070470120704783680E
:10D4000001290CBF586C00207047836800220A80F5
:10D410004A801A685B68013A013B8A80CB8070477A
:10D42000F0B5104D2E4607460FCE91B06C460FC496
:10D4300096E80F00203584E80F000FCD08AC0FC42C
:10D4400095E80F0084E80F007B6B10AA02EB8303C2
:10D4500053F8402CC7F8002153F8203CC7F804319A
:10D4600011B0F0BD88F1010807B580698DE80600AC
:10D4700003216A46F3F71CFA03B05DF804FB2DE9BB
:10D48000F74384689846E38C9B078946174632D554
:10D49000D4F8003120469847D4F8045106463A465D
:10D4A00020464946A8472369A2699E42ACBF002393
:10D4B00001239642D4BF1A4643F0010263699842A1
:10D4C000ACBF134642F00103054613B9E369984225
:10D4D0000ADD62682368013A00920021D4F8A8703E
:10D4E00020460A46013BB847D4F8AC702046314686
:10D4F0002A46B84703E0D4F8AC502046A847D4F8F1
:10D50000A43020464146984703B0BDE8F083F7B504
:10D510008468E38C9B070F46164645D5D4F8003146
:10D5200020469847D4F8043132460546394620460D
:10D530009847D4F8983006461BB1204601210022B6
:10D5400098472369A2699D42ACBF002301239542FD
:10D55000D4BF1A4643F0010263699E42ACBF134632
:10D5600042F0010313B9E3699E420ADD6268236851
:10D57000013A00920021D4F8A87020460A46013BE7
:10D58000B8472946D4F8AC30204632469847D4F8FC
:10D59000A03020469847D4F8983005466BB1204615
:10D5A00000210122984708E0D4F8AC302046984783
:10D5B000D4F8A030204698470546284603B0F0BD71
:10D5C00038B58568044695B94FF4BA7002F0B4FFD7
:10D5D0004FF4BA72A060294600F0C4FDA36802228D
:10D5E000DA8401221A62024A1C64C3F8082138BD99
:10D5F00021D4000870B506460D461446FFF7E0FF3B
:10D60000B368002B3BD0262D02D0272D16D070BD3D
:10D610009A6B102A02D0122A08D070BD184AC3F89B
:10D62000D440C3F8B820C3F8B42070BD154AC3F87D
:10D63000D840C3F8BC20C3F8C02070BD9A6B102A34
:10D6400002D0122A0ED070BD3CB10F4AC3F8DC40A4
:10D65000C3F8C820C3F8C42070BDC3F8C840C3F8DD
:10D66000C44070BD3CB1094AC3F8E040C3F8CC20C7
:10D67000C3F8D02070BDC3F8CC40C3F8D04070BD13
:10D68000B1D20008BFD20008CDD2000803D30008F1
:10D6900038B50546FFF794FFAC684FF4FA7002F016
:10D6A0004BFFA36BA0660733D8102368584302F0E2
:10D6B00043FF01210022E066A869F3F7F9F8D4F8E6
:10D6C00008310546204698472046D4F8B0309847A0
:10D6D000002DD4BF0020012038BD70B504460D4692
:10D6E0001646FFF76DFFA36883E8600070BD70B554
:10D6F00004460D461646FFF763FFA3689D60DE6093
:10D7000070BD38B505460C46FFF75AFFAB68226876
:10D71000DA6262681A63A2685A63520707D593E80F
:10D7200006001A605960DA689968D9609A60A2891F
:10D730009A84226912B122EAE2721A6238BD2DE996
:10D74000F04104461F4616468846FFF739FFA56894
:10D750004146682205F586700AF022FF2046B04750
:10D760002046B84723699B689847A862BDE8F081C6
:10D7700010B5074C2368186B00F05EFC00F07CFCD1
:10D780002368586B00F058FCBDE8104000F090BCD6
:10D790002401002037B5094C23685A7C084B054604
:10D7A00053F82200C2686946126B904720682946E8
:10D7B0006A46083000F08AFD03B030BD2401002025
:10D7C000A417022037B50D46144602F009F801905F
:10D7D00008B901200CE0C3680A215B6A01A89847D8
:10D7E00003460028F5D00198294622469847002094
:10D7F00003B030BD37B50D46144601F0F1FF01907E
:10D8000008B901200CE0C3680B215B6A01A89847A6
:10D8100003460028F5D00198294622469847002063
:10D8200003B030BD37B50D46144601F0D9FF019065
:10D8300008B901200CE0C36810215B6A01A8984771
:10D8400003460028F5D00198294622469847002033
:10D8500003B030BD012810B50C4608DC01F0C0FF54
:10D8600020B1C36821469B6A984710BD10BD0020B7
:10D8700010BD38B5044621460120FFF7EBFF2146D5
:10D8800005460020FFF7E6FFA842B8BF284620EA79
:10D89000E07038BD0121FFF7DDBF0221FFF7DABFDD
:10D8A0000321FFF7D7BF0421FFF7D4BF0821FFF7FB
:10D8B000D1BF0921FFF7CEBF024B1B68587CFFF791
:10D8C000E9BF00BF24010020024B1B68587CFFF712
:10D8D000E4BF00BF24010020024B1B68587CFFF707
:10D8E000E8BF00BF2401002008B5044B53F8200016
:10D8F000C36808219B6A984708BD00BFA41702208F
:10D9000008B501F06DFF20B1C3680221DB6A9847BA
:10D9100008BD08BD024B1B68587CFFF7F1BF00BF74
:10D9200024010020024B53F820301B6958687047CF
:10D93000A4170220024B53F820301B691868704767
:10D94000A41702200120FFF794BF0220FFF791BF28
:10D950000320FFF78EBF0000024B1860024B1960D6
:10D96000704700BF08D8012004D80120014B186877
:10D97000704700BF08D80120014B1868704700BFEE
:10D9800004D8012000283BD030F0010329D030F02A
:10D99000030328D030F0070327D030F00F0326D040
:10D9A00030F01F0325D030F0FF0324D020F4FF73A4
:10D9B00023F001030BB320F47F6323F00F03E3B1E3
:10D9C00020F4FF4323F07F03BBB1030C1B04A3B17E
:10D9D000830C9B049BB110F07F4F0CBF18202020BC
:10D9E00070470120704702207047032070470420D1
:10D9F000704705207047082070471020704712209C
:10DA0000704708B5FFF7BEFF01280FD0831E062B15
:10DA100009D9A0F10903072B07D91138102834BF01
:10DA20002020002008BD082008BD102008BD0000EF
:10DA300070B5084B1B681A7C80EA0201490705D5BE
:10DA40009C6BD96B26680D6825600E6018741046B3
:10DA500070BD00BF2401002008B5024B1B689B6805
:10DA6000984708BD1801002038B5144B1B680A46BA
:10DA7000B3F90A108A4204461EDBB3F90E108A423B
:10DA80001ADCB3F90810884216DBB3F90C1088428F
:10DA900012DC197C587C11F0010F094951F8200063
:10DAA00004D0C3682146DB69984738BDC168DB6B89
:10DAB0008D691B682146A84738BD00BF240100209E
:10DAC000A417022038B5104B1C68B4F90A309942EB
:10DAD0000D4617DBB4F90E30994213DCB4F9081087
:10DAE000B4F90C308842A8BF01469A42B8BF134629
:10DAF0008B4207DB607C054A52F82000C2689468BC
:10DB00002A46A04738BD00BF24010020A4170220E8
:10DB100038B5104B1C68B4F9083005469D421046D4
:10DB200017DBB4F90C309D4213DCB4F90A20B4F9C8
:10DB30000E309142A8BF0A469842B8BF03469342AE
:10DB400007DB607C044951F82000C168CC68294695
:10DB5000A04738BD24010020A417022073B50E464B
:10DB600012490C68B4F90810B4F90C508842A8BFE7
:10DB70000146AA42B8BF15468D4214DBB4F90A200B
:10DB8000B4F90E009642A8BF32468342A8BF0346AE
:10DB9000934208DB647C064850F82400C468009374
:10DBA00024692B46A04702B070BD00BF24010020AD
:10DBB000A41702202DE9F04FDFF8ACC18FB0DCF8DC
:10DBC00000C009900E4615469B461C9CDDF87880E7
:10DBD000BCF1000F0DD0189D199E009501961A9F5B
:10DBE0001B9D1D9E0297039504940596DCF800404A
:10DBF00053E0189F199847EA0003012B4FD1584B67
:10DC00001868B0F90A20511A002908DDC1EB0B038E
:10DC1000002B40F3A2801B9F07FB014401E05B4601
:10DC200032465E44B0F90E10013E761A002E03DD36
:10DC30009B1B002B40F391800999B0F90C6029449B
:10DC40000139891B099E0029C8BFC1EB0505C8EB36
:10DC50000601B0F90860B1420CDAC1EB060C08EB22
:10DC60000C078E1B2CF0070C354404EBE7046144D1
:10DC700007F00708002D70DD467C3A481A9F50F8DF
:10DC80002600C668019703941B9F1D9C0093029772
:10DC9000CDF81080059474682B46A0475DE01A9F6C
:10DCA000C7F108070C976746DC4556DA2C4B1998E4
:10DCB0001B683044B3F90A200A90411E91420B912F
:10DCC00045DBB3F90E309E4241DC4FF00008DDF831
:10DCD00024900894C246AA4539DAB8F1000F05D15C
:10DCE000089A1778013208924FF008080C981A9990
:10DCF0001B4A47FA00F3C1EB08088F4013F0FF01FD
:10DD0000FFB203D11068007C80071BD41268D26B6D
:10DD100010680D901D9810B150F8213000E0DBB272
:10DD2000189913604A1E4A440B9BCDF81CC0484604
:10DD30003146FFF713FF0A4B0D9A1B68DDF81CC034
:10DD4000DB6B1A60189B0AF1010A9944C3E71B9E1A
:10DD50000CF1010C34440A9EA6E70FB0BDE8F08F29
:10DD600024010020A4170220781702202DE9F04F8B
:10DD7000DFF80CC291B0DCF80090079205468846A7
:10DD80009B461C9E1E9CB9F1000F0CD01A9D1B9F38
:10DD9000009501971D9D1F9F02960395049405977A
:10DDA000D9F8004081E01A9F1B9847EA0003012B35
:10DDB0007DD1714B1868B0F90A20531A002B08DD89
:10DDC000C3EB0B01002940F3D4801D9F07FB0344E4
:10DDD00001E059464246D844B0F90E3008F1FF3808
:10DDE000C3EB0808B8F1000F04DDC8EB01010029FE
:10DDF00040F3BF80079BB0F90CC02B44013BCCEB38
:10DE00000303002B02DD079FFF1A0797B0F908C034
:10DE1000654533DA079FC5EB0C03FF1A082E0797F9
:10DE200027D00DDC022E14D0042E1AD0012E26D1BC
:10DE300023F0070C04EBE304654403F007031EE042
:10DE4000182E18D0202E16D0102E18D104EB430413
:10DE500013E023F0030C04EBA304654403F0030375
:10DE60000DE023F0010C04EB6304654403F00103AF
:10DE700005E01C4401E004EB830465460023079F92
:10DE8000002F76DD90F811E03C481D9F50F82E00E1
:10DE9000D0F80CE003948DE842001F9C0493029795
:10DEA0000594DEF80440079B2946A04761E0C6F1CF
:10DEB00008070E97CDF828900A9F5F4559DA2E4B38
:10DEC0001B9F1B684744B3F90A200C97013F9742F8
:10DED0000D9746DBB3F90E30984542DC4FF0000A4F
:10DEE0000B94AC465746079887423ADABAF1000FCE
:10DEF00006D10B9890F8009001300B904FF0080A73
:10DF00000E991D4A49FA01F313F0FF0109FA06F9C7
:10DF10005FFA89F9C6EB0A0A03D11068007C800712
:10DF20001BD41268D26B10680F901F9810B150F874
:10DF3000213000E0DBB21A9913604A1E6244604649
:10DF40000D9BCDF820C04146FFF708FE0A4B0F9A03
:10DF50001B68DDF820C0DB6B1A601A9B01379C44FC
:10DF6000C1E70A9FDDF8308001370A971D9F3C44C6
:10DF7000A2E711B0BDE8F08F24010020A417022011
:10DF80007817022008B5054B1968054B4A7C53F8F1
:10DF90002200C36808311B6B984708BD240100208C
:10DFA000A417022037B5FFF7EDFF04F02DFF04465C
:10DFB00000283DD10546284601F012FC019048B1E9
:10DFC000C3680C215B6A01A89847034670B30198A7
:10DFD000984704430135022DEDD14CBB04F030FFCE
:10DFE0000124204601F0FCFB0190D0B1204600F056
:10DFF000A1FE0420FFF730FD43F6FF72002001462A
:10E000001346FFF7ABFD0020FFF726FD02A80E2107
:10E0100050F8043DDB685B6A9847034608B10198F5
:10E02000984714F1FF34DCD2002002E0012000E028
:10E03000204603B030BD000008B5054B1B685A7C74
:10E04000044B53F822301B691B68984708BD00BF7A
:10E0500024010020A417022008B5054B1B685A7C38
:10E06000044B53F822301B695B68984708BD00BF1A
:10E0700024010020A4170220044B1B681A7C5207BD
:10E080004CBF9B6BDB6B1860704700BF2401002006
:10E0900008B5064B1B68196B814206D01863FFF761
:10E0A000CBFFBDE80840FFF7E7BF08BD2401002013
:10E0B000044B1B681A7C52074CBFDB6B9B6B1860D0
:10E0C000704700BF2401002008B5064B1B68596B40
:10E0D000814206D05863FFF7AFFFBDE80840FFF765
:10E0E000E7BF08BD2401002008B5024B1B685B6830
:10E0F000984708BD1801002008B5024B1B681B6833
:10E10000984708BD1801002070B5840702D501802A
:10E11000013A023055082B4605B3032D01EB0144AB
:10E1200002DC06461D4612E003462E46043E032E40
:10E130001C605C609C60DC6003F11003F6DC043D55
:10E14000AB085E1C00EB0610A5EB8303E9E71DB1ED
:10E1500046F8044B013DFAE700EB8300D30748BFC4
:10E16000018070BD70B52AB1830703D000F8011B90
:10E17000013AF8E7930801D1024417E04FF0013467
:10E1800002F003024C43032B054606DD04604460A5
:10E190008460C460043B1030F5E71E461BB145F8AF
:10E1A000044B013BFAE700EB8600E5E7904202D022
:10E1B00000F8011BFAE770BD0B8892B2134403808C
:10E1C0008B889B1A83804B8813444380CB889A1A90
:10E1D000C28070470128F7B504460D4665DC344B14
:10E1E0001B6803B19847012D04D0022D21D0002DCA
:10E1F0005BD135E02F4E56F82470B7B9204601F0B8
:10E20000EFFA0190002850D0C3680D215B6A01A885
:10E2100098470346002848D001982946984756F861
:10E220002430013346F8243018E0013746F82470D2
:10E230003BE0204601F0D4FA0190002835D0C368B5
:10E240000D215B6A01A89847044600282DD01A4B7F
:10E250001B6803B1984701980221A047002025E0E0
:10E26000144D55F82430012B01D0012015E0204633
:10E2700001F0B6FA01900028F7D0C3680D215B6A5F
:10E2800001A8984706460028EFD00B4B1B6803B146
:10E29000984701980021B047002055F82430002B02
:10E2A00018BF013B45F8243000E0012003B0F0BD69
:10E2B00018D8012010D801200CD80120024B1B686F
:10E2C0000146587CFFF786BF2401002070B5B2F9E3
:10E2D0000030B1F90040B1F90250B1F90460B1F970
:10E2E00006109C42B8BF1C46B2F902309D42A8BF3E
:10E2F0002B46B2F90450B2F90620AE42B8BF3546FB
:10E30000A4B2ADB29142B8BF0A460480858024B25F
:10E310002DB29BB292B2A5424380C28006DB10B2FE
:10E320001BB29842B4BF0020012070BD002070BD18
:10E330000B8810B5B0F900401AB29442B8BF038000
:10E340004B88B0F902401AB29442B8BF43808B8820
:10E35000B0F904401AB29442C8BF8380CB88B0F9A8
:10E3600006101AB29142C8BFC38010BD01F07F43AE
:10E37000B3F17F4FF0B527D0D343DBB2CDB2C6B2F5
:10E380005D4302FB065501F47F4600F47F445E4383
:10E3900002FB046601F47F0400F47F075C43090E6E
:10E3A000000E02FB07444B43360A02FB0032240AEC
:10E3B000C5F3072306F47F401843120404F47F03D7
:10E3C000184302F07F421043F0BD000070B50A4CC4
:10E3D0000A4D20680A4E01F043FF286801F040FF13
:10E3E000306801F03DFF074A00231360064A33609E
:10E3F0002B602360136070BD20D801201CD8012041
:10E4000024D8012028D8012038D801202DE9F8434C
:10E410001C46284B17461A680646884632B9012220
:10E4200025481A60254B036001F00EFB244D2B6834
:10E4300033B9244B1B682B6013B9FFF789FA2860A6
:10E440000CB12B68236096B11F4B1A6899460024C3
:10E450004AB92868800002F06FF8D0F10104C9F8C9
:10E46000000038BF0024D9F80030336000E03446A3
:10E47000B8F1000F0DD0154E33683BB92868800005
:10E4800002F05AF80028306008BF01243368C8F849
:10E49000003067B10E4E33683BB92868800002F047
:10E4A0004BF80028306008BF012433683B602046E9
:10E4B000BDE8F88338D8012030D80120CDE300082A
:10E4C00028D80120AC17022020D801201CD8012018
:10E4D00024D801202DE9F04F93B000241D9E0B900D
:10E4E0000C9190461F4634600FA810A9224611AB2C
:10E4F000FFF78CFF0546002840F0C380634C119A5B
:10E500002368587C624B53F8203007939742A8BF8A
:10E5100017461A690D920A97FFF7E6F923680890E3
:10E52000587CFFF7FFF95B4B0490984205D05A4B9B
:10E53000C31A18BF0123069300E0069500250A9C24
:10E54000AB4643461C9A53F8040B05939047030EC1
:10E550008146099300F08580BBF1000F3FD14B4B02
:10E560000B9F1B680A9AB3F90830DDF82CC00C9990
:10E570002F44BB42C8BFC7EB030B0BEB050AC8BF58
:10E580001F460F9B4FEA8A0A534494440093079B0B
:10E5900001930CF1FF3238460B46CDF80CC004F065
:10E5A000F9FB089A0F98DDF80CC0172A06DC5044D6
:10E5B000CBEB04010D9B04F093FC01E0069B13B927
:10E5C0004FF0010B0BE0C7EB0C078244DAF80000B8
:10E5D000049A9047013F4AF8040BF7D1F0E72F4B1C
:10E5E0000F99D3F800C0109F4FEA850ABCF1000FC5
:10E5F00024D007EB0A025144109223460F91404663
:10E60000E0470F9D109A002358F8031001F07F4057
:10E61000B0F17F4FE85801D1D05005E000F07F40C5
:10E62000B0F17F4F08BFD150013C03F10403EBD19F
:10E630003368109743F00103336020E0099BFF2B00
:10E6400004D151F80A3047F80A3011E0099B51F81B
:10E650000A10DA434846D2B2FFF788FE47F80A00AC
:10E6600002E0109B43F82500336843F00103336058
:10E67000013C05F1010502D0DDF8148061E7109836
:10E6800000E0204613B0BDE8F08F00BF2401002059
:10E69000A4170220DF090108DD0901082CD8012098
:10E6A0001FB508B103AA00E0024601A802A9002391
:10E6B000FFF7ACFE05B05DF804FB000008B5024BA7
:10E6C0001B6803B1984708BD3CD80120B5EEC00ACD
:10E6D000F1EE10FADFED0D7A48BFB1EE400A30EEF0
:10E6E000270A0020B5EE400AF1EE10FA0CD0F2EE47
:10E6F000047A20EE270A0130FCEEC07AC0B217EE91
:10E70000903A002BF3D07047704700BF5F7089309C
:10E71000B5EEC00AF1EE10FA08B5F6EE007A0AD5A9
:10E7200070EE677A17EE900A08F044FC41EC100B8B
:10E7300007F0AAFB09E070EE277A17EE900A08F0BE
:10E7400039FC41EC100B07F01FFC51EC100B08F0EA
:10E7500011FD00EE100A08BD0E4B53F8213007EEF4
:10E76000903AF8EE677A70B520EE270A05460C4617
:10E770001646FFF7CDFFBDEEC00A294610EE100A7F
:10E7800022461EB1BDE8704000F0AEB8BDE8704052
:10E7900000F09DB854F3010838B5B5EE400AF1EE2B
:10E7A00010FA2DED028B0446B0EE408A0D4652D091
:10E7B000B5EEC00AF1EE10FA24DBF7EE008AB4EEF3
:10E7C000E80AF1EE10FA1DD5FFF780FFA04202DC47
:10E7D00078EE287A46E0F6EE007AB4EEE78AF1EEBB
:10E7E00010FA09DBDFED367A002C18BFF0EE687AFC
:10E7F00008BFB0EE688A35E044B3F0EE687A9FED6A
:10E80000308A2FE0B5EEC08AF1EE10FA28D5FFEE7F
:10E81000008AB4EEE88AF1EE10FA21DDB0EE480A83
:10E82000FFF754FFA04204DCF7EE007A78EE677A37
:10E8300018E0FEEE007AB4EEE78AF1EE10FA03D8A3
:10E840004CB9B0EE688A0BE044B104E0DFED1C7A0D
:10E85000B0EE678A06E0F7EE007A03E09FED188AD3
:10E86000F0EE487A174B53F8243000EE103AB8EE29
:10E87000400A27EE800AFFF74BFFBDEEC00A10EEFC
:10E88000100A01F061FF012DC4EB000020EAE070E6
:10E8900005D1B5EEC08AF1EE10FAC8BF0130B0EE76
:10E8A000480ABDEC028B002C0CBF2346631C1844A5
:10E8B00021462A46C0B2BDE83840FFF74DBF00BF31
:10E8C0000000000054F301080021FFF765BF1FB5E9
:10E8D00004AB01AC43F8104D6B4601F059FF2046E4
:10E8E00000F0FAFE04B010BDF0B585B004AC0D46E2
:10E8F00001AE6946174644F8106D01F03DFF00284F
:10E90000C4BF05F1FF35EDB229463A466B4601F02A
:10E910003FFF304600F0E0FE05B0F0BD034A0023A3
:10E920001360034A1360034A1360704740D8012004
:10E9300044D8012050D801202DE9F043194B1F681D
:10E9400085B000259846D8F80030164C33B300F057
:10E9500091F90646206801F097FC034604A859691E
:10E9600040F8103D891B002913DC216803910196B2
:10E9700019695E68029168462660D3F8009001F03C
:10E9800091FC01A8C8474EB12368BB4205D00125C0
:10E99000D9E7684601F086FC00E00025284605B06E
:10E9A000BDE8F08344D80120F0B5254C85B005467C
:10E9B00001F06AFC2368019013B92560436039E0D7
:10E9C000184601F061FC04AB466943F8100D684637
:10E9D00001F068FC019B5A69921B002A03DC226843
:10E9E0005A60256026E02668304601F04DFC04ACF4
:10E9F000466844F8080DBEB1304601F045FC04AB52
:10EA0000476943F8040D184601F04CFC019A53691C
:10EA1000DB1B002B029B02DC56605D6007E020469A
:10EA20005E6801F03FFCDFE7019B5E6045602046C9
:10EA300001F038FC01A801F035FC05B0F0BD00BFC5
:10EA400044D8012037B50546F0B101F01DFC0F4B4D
:10EA500000901C68AC4204D142681A6011E001F0D9
:10EA600021FC74B1204601F00FFC034602A85C684B
:10EA700040F8043DAC42F2D1009A52685A6001F06D
:10EA800011FC684601F00EFC03B030BD44D80120F3
:10EA9000002337B50360094B1C68054654B1204676
:10EAA00001F0F2FB02AB026943F8040D2A6018463C
:10EAB00001F0F8FB204603B030BD00BF40D8012074
:10EAC000002373B50B600E46044690B101F0DCFBE9
:10EAD00002AD846845F8040D44B1284601F0E2FB1C
:10EAE000204601F0D1FB036901903360284601F014
:10EAF000D9FB204602B070BD2DE9F74381461C20AA
:10EB00000E4690461F4601F091FE0446002831D083
:10EB10001A4B1B4A1A6001F0B7FB009016B900F0BF
:10EB2000A9F8064602A850F8085D68466E61C5F867
:10EB30000090C5F81080AF8101F0B4FB2046FFF7CC
:10EB400033FF104B1A6832B901220F481A600F4B7D
:10EB5000036000F079FF204601F096FB0C4A01901B
:10EB6000136813B91460836001E08360146001A826
:10EB700001F098FB204603B0BDE8F083881702201F
:10EB800039E9000850D8012048D801201DE90008C3
:10EB900040D8012073B5044658B3174D2E688642FD
:10EBA0000BD101F071FB02AB826843F8040D2A60BF
:10EBB000184616E0684601F075FB304601F064FB2C
:10EBC000866802ADA64245F8080DF3D1204601F053
:10EBD0005BFB009B826801909A6001A801F062FBD8
:10EBE000684601F05FFB2046FFF72CFF204601F04E
:10EBF00085FB02B070BD00BF40D8012013B50C46A4
:10EC000040B101F041FB02AB846143F8040D1846AA
:10EC100001F048FB02B010BD13B5044698B101F0F5
:10EC200033FB019000F026F802AB53F8042D9169F4
:10EC300008445061184601F035FB2046FFF702FFFB
:10EC40002046FFF7B1FE02B010BD13B50C4668B107
:10EC500001F01AFB02AB828943F8040D14421846F6
:10EC60000CBF0024012401F01DFB00E0012420461C
:10EC700002B010BD05F016BB034B1B68B3F92A2088
:10EC800058851046704700BF24010020034B1B68C5
:10EC9000B3F92C2098851046704700BF240100204E
:10ECA000024B1B689A7E987610467047240100201C
:10ECB000034B1B68D96900B1D8610846704700BF93
:10ECC00024010020FEF7C8BE08B5002000F01CF8A3
:10ECD0006FF07F4000F01AF8012000F07DF800206E
:10ECE000FFF7D4FF0020FFF7C7FF0020FFF7EAFF80
:10ECF000044B1868FFF7DCFF0020BDE80840FFF771
:10ED0000CFBF00BF28010020FFF7EEB9FFF7F4B92D
:10ED100010B5074B1C7820B101221A704FF0FF305C
:10ED200002E018706FF07F4004F0C8F8204610BD74
:10ED30009517022070B5084D2B68012804465E7CAB
:10ED400008D800F04DFD28B12B685C7400F008F87D
:10ED5000024B1C60304670BD240100204817022081
:10ED600008B503F003FFFEF703FDBDE80840FCF71C
:10ED7000A5BB000008B5034B7022196809F010FC10
:10ED800008BD00BF2401002008B5034B01467022D6
:10ED9000186809F005FC08BD24010020B0F9022024
:10EDA000B1F906309A4214DCB1F90220B0F906300C
:10EDB0009A420EDCB0F90020B1F904309A4208DC26
:10EDC000B0F90430B1F900209A42CCBF00200120F4
:10EDD0007047002070470000024B1B681A7E1876AF
:10EDE0001046704724010020024B1A6802B91860CF
:10EDF000FFF764BC54D801200A4A0B49136809681C
:10EE00008B4210B50BD0094CA34293E8030014BF0A
:10EE10000833503B136002F02FFB012010BD00208F
:10EE200010BD00BF200100201C010020A8D8012037
:10EE300068B1038889B20B440380838819444388EE
:10EE4000818092B213444380C3881A44C2807047C1
:10EE500010B538B309B30AB3B1F90040B2F90030C4
:10EE60009C42B8BF23460380B1F90240B2F9023098
:10EE70009C42B8BF23464380B1F90440B2F9043044
:10EE8000B1F906109C42A8BF23468380B2F9063030
:10EE90009942A8BF0B46C38010BD11460B680360A2
:10EEA0004B68436010BD0000054B1B68002B18BF6A
:10EEB0000020044B0129B8BF01211954704700BF3D
:10EEC000B0D8012074170220024B1B685884998423
:10EED0000020704724010020044BB3F90030036088
:10EEE000034BB3F900300B60704700BF8C17022052
:10EEF00080170220014B1B68987E70472401002078
:10EF000003F0E4BF0A4B10B51C681CB1A047041CF9
:10EF100018BF0124FCF724FA064B1B68002818BF11
:10EF200001241BB19847002818BF0124204610BDBA
:10EF300088170220A017022010B50024FFF7E2FF77
:10EF400008B10124FAE7204610BD00000F4B73B54D
:10EF50001B68DE6C1C6D06440D19B3B21444684680
:10EF6000ADF80030ADF80430ADF80250ADF8064011
:10EF7000FCF7C2F838B1304629462246FEF7C8FDF4
:10EF8000FBF7F8FFF6E702B070BD00BF24010020D8
:10EF90001E4B1B689B7E013B032B32D8DFE803F03E
:10EFA000020D1A221A4B06300340002B03DA013BF4
:10EFB00063F00F0301330B2B08E0164B0340002BCB
:10EFC00003DA013B63F003030133012BCCBF0020C4
:10EFD00001207047142390FBF3F203FB12000B286F
:10EFE00009DC10E0182390FBF3F203FB12000B285E
:10EFF00009DD20F00400103801288CBF002001201A
:10F000007047002070470120704700BF2401002096
:10F010000F00008003000080C0F30B00B0F5006F0C
:10F02000C6BFA0F5006001210021B0F5806FC8BF08
:10F03000C0F5006000F03F0310B582110B4CC3F126
:10F0400040039BB234F81200402B00FB03F008D0C1
:10F05000102A06D00132C3F1400334F8122003FB1A
:10F0600002002030800901B1404210BD08F30108C0
:10F0700000F58060FFF7D0BF2DE9F74FDDF8308055
:10F08000171A5C1A54EA070C05460E46D8F800B069
:10F0900004D103B0BDE8F04F04F000BB87EAE7708D
:10F0A000A0EBE77084EAE471A1EBE471884204DB31
:10F0B00021463C460F46002106E011461A460B4603
:10F0C000294635460E460121009184EAE471A1EB00
:10F0D000E4718C4208D01E462B46644215467F429E
:10F0E0001A464FF0FF3A01E04FF0010A002FDFF817
:10F0F00048913ED1009BD3B1D9F800309B7E8BB9AB
:10F100003046294603B0BDE8F04FFEF701BDFFF7DA
:10F110003FFF30B9D9F800305B6E30465B68791933
:10F1200098470137A74207EB0B00F0DD1DE0D9F847
:10F130000030997E11B1DDF800A012E05B6E284628
:10F140001B683146984774E0FFF722FF38B9D9F8B9
:10F1500000305B6E0AEB05005B68314698470AF1A8
:10F16000010AA2450AEB0B00EEDD0138C8F80000E9
:10F170005FE0D9F800104FF00202897E94FBF2F2B2
:10F18000B8BF5242D9B99346A846C5EB0803A3427B
:10F190004FDC009B9BFBF4F131442BB9D9F80030D4
:10F1A0005B6E40465B6805E0D9F800305B6E5B68DB
:10F1B00008464146984708F10108BB44E5E7BAF123
:10F1C000FF3F04BF04EB0B01C8F800100192AB46EF
:10F1D000C5EB0B01A142D8F800001EDC5044C8F872
:10F1E0000000FFF7D5FE80B9DDF804C0D9F80000B3
:10F1F000009B406E9CFBF4F1314413B943685846C0
:10F2000002E04368084659469847DDF804C0BC440C
:10F210000BF1010BCDF804C0DAE7BAF1FF3F04BFF0
:10F220002418C8F80040D8F80020CAEB0203C8F838
:10F23000003003B0BDE8F08F240100202DE9F04F2D
:10F24000674D2C6894F818B0BBF1010F87B0814668
:10F25000884617461E46AA4604D1109C0094FFF724
:10F260000BFFBAE0841ACD1A54EA050300F0B5800A
:10F27000002CBABF644201230023002DBCBF6D42A5
:10F2800043F00203A5420BF1FF3B04DD224643F0AD
:10F2900004032C461546022294FBF2F202EB85256C
:10F2A00095FBF4F4A1114F4AC4F38304C4F1100593
:10F2B00032F91100102D05FB00F004D0013132F9B4
:10F2C000112004FB02001022083090FBF2F05907D5
:10F2D00048BFC0F58060DA0748BFC0F500609B07F3
:10F2E00048BFC0F5805000F580652846FFF7C0FE96
:10F2F00000FB0BF42846FFF78FFE002C00FB0BF001
:10F3000004DAC4F500739B125B4202E004F500735B
:10F310009B12002806DAC0F5007B4FEAAB2BCBF13D
:10F32000000B03E000F5007B4FEAAB2B002B03DD65
:10F33000581C40105B1005E0022293FBF2F0013BE9
:10F3400093FBF2F3BBF1000F05DD0BF1010252104C
:10F350004FEA6B0B06E002219BFBF1F20BF1FF3B46
:10F360009BFBF1FB80B21FFA89F4011992B2ADF850
:10F3700008101FFA8BFB1FFA88F15518CBEB01011F
:10F380009BB2ADF80E10B9B2E41ACB1AADF810303A
:10F39000B3B20144CBEB030B13440022ADF81410BD
:10F3A000ADF8163002A813460421ADF80A50ADF8A6
:10F3B0000C40ADF812B004F08FF8DAF800305B7E44
:10F3C0001BB94846414604F069F9DAF800305B7E23
:10F3D0001BB93846314604F061F907B0BDE8F08F3B
:10F3E000240100202AF3010830B585B004AC0025C3
:10F3F00044F8045D0094FFF721FF05B030BD000024
:10F400002DE9F8431E460C4B1C6881460020E56C34
:10F41000246D88461746FBF76FFE50B109EB0500D7
:10F4200008EB04017A193319FFF7DEFFFBF7A2FDA1
:10F43000F3E7BDE8F88300BF24010020F7B5104FC3
:10F440003B681D6DDC6C05440E19ABB21444684674
:10F45000ADF80060ADF80440ADF80230ADF806300C
:10F46000FBF74AFE48B13B685B6E30461B68294695
:10F4700022469847FBF77EFDF4E703B0F0BD00BFDE
:10F48000240100202DE9F04F9846814B8BB08A462D
:10F490001968069000209146149F159ECD6C0C6D46
:10F4A000FBF72AFE002800F0EF800AF100430698DF
:10F4B000013B00EB43030793169B002B14BF6FF037
:10F4C00001030223A9444444099327B9FBF752FDE1
:10F4D0000028FAD1D8E0002EF8D0BAF1000FF5DDFF
:10F4E0007B1C04D1012E14BF022301230AE0012F4B
:10F4F00004D1012E14BF0323002303E0012E14BF07
:10F50000052304230593624B1B685B69EBB1B3F9D8
:10F510000080B3F90200B3F90420B3F906B00490F7
:10F5200008F1FF38C14509EB0A03B8BFC9EB080869
:10F5300003F1FF33B4BF28EAE8784FF000089342A4
:10F540000ADDC9EB0202013207E04FF0FF3B5246F1
:10F55000CDF810B0984600E05246169B1BB9069BAA
:10F5600003EB480300E0079B90450393AEDA4A445F
:10F5700008920022C8440123029203980999058841
:10F5800008442DB247F6FF718D4203900DD10298C9
:10F5900000286FD1002B6FD1114608F1FF30019286
:10F5A000FEF762FA0123019A67E00598411EDBB17C
:10F5B000042917D8DFE801F00305070B0F00621BD1
:10F5C0000EE0651B00E02544B5FBF6F208E025449B
:10F5D00007FB05F204E0254407FB05F2B2FBF6F257
:10F5E00000234AE02A19FBE7042912D8DFE801F0DA
:10F5F0000305070B0E00651B0CE0651B00E02544AE
:10F60000B5FBF6F506E025447D4303E025447D4344
:10F61000F6E7254404998A4201DA8D4225DB5A45F2
:10F6200001DD5D4521DC05EB020C0221AA429CFBB9
:10F63000F1FC08F1FF300BDC114662468DE8081042
:10F64000FEF766FADDF804C0404661462A4609E046
:10F6500061468DE80810FEF75BFADDF804C040460D
:10F6600029466246FEF754FA009B029A0132029242
:10F670002A4602E0002302930123089808F10108BA
:10F6800080457FF47AAF21E70BB0BDE8F08F00BF73
:10F6900024010020F8B50B4B1B680546B3F92C007C
:10F6A00040F002000F461646FFF7F0FA39460446CE
:10F6B0003246284600F008F82046BDE8F840FFF73B
:10F6C000E5BA00BF24010020024B1B6859849A84CC
:10F6D00000F002B8240100202DE9F74F044600286D
:10F6E00079D03E4D00F0B4FC2B688046B3F82290F0
:10F6F00000F096FC2B689A8C87B2D21B9A842378F0
:10F70000002B5DD047F6FF71204600F0D7FB064680
:10F710003146204600F000FC2B689A8D02F003026F
:10F72000012A05D0022A14BF002290FBF2F200E069
:10F730000246598C8A1A92B291B259841FFA80FA01
:10F740009B8CADF800100AF1FF310A44ADF802308D
:10F750001FFA88FB013B5B44ADF80420204631468C
:10F760006A46ADF8063000F007FC2B68BDF80220B1
:10F770009A842046314603F029FE235C0A2B04EBD1
:10F78000000201D00D2B12D12B68998D01F00301DD
:10F79000013901298ABF198CA3F822905984117864
:10F7A0000A290BD1998C8B44A3F824B006E00B4BAB
:10F7B000BDF800001B688244A3F822A0137843B967
:10F7C0002B689A8C17449A8D9F8422F003029A85A5
:10F7D00001E0541C93E703B0BDE8F08F2401002042
:10F7E000012809DC054B53F8200020B1C3681B68D1
:10F7F0001BB10068F9E7704700207047A41702208A
:10F8000000F02EBD012BF8B506460D4617461C46E6
:10F8100001DD0020F8BD1C2000F08EFE0028F8D08D
:10F820000DB1056109E0094B53F8241029B10B68AB
:10F830000BB11946FBE70B69036100238360846108
:10F840008782C66003604360F8BD00BFA417022032
:10F85000094B826953F82210814204BF016843F8C2
:10F86000221043680BB102681A60026802B153604B
:10F870000023036043607047A417022070B538B3BB
:10F880008269012A24DC194951F822300D4613B946
:10F8900041F822001AE0596809B10B46FBE7C1683C
:10F8A0000E68D9680C68B44203DD1B68002BF8D1E0
:10F8B0000EE002D1818A012911D0596899B10860FE
:10F8C00041605860984208BF00230360002070BD6B
:10F8D000012070BDCB681B68A3420B46EDDB1968A5
:10F8E0000029F7D1E9E745F82200EAE7A41702204A
:10F8F00038B51D46FFF786FF044648B1FFF7BEFF47
:10F90000E3681B6823B9034B16351B6843F8254091
:10F91000204638BD2401002010B5074B07480024BD
:10F92000214670221C60FEF71DFC21460448082277
:10F93000BDE81040FEF716BC30D90120B8D8012030
:10F94000A417022038B5194D2B681A1DDA6303F18C
:10F9500008029B631B6442615A7C154B044653F8B2
:10F960002200C36804F108011B6B9847114B6366C2
:10F97000114B1B68E3612B68083363610123237615
:10F98000FAF76EFC032384F868306FF0704323634A
:10F990006363A0640020FEF7A7FB6FF07F40FEF7D3
:10F9A000ABFB064B064A1A6038BD00BF240100209D
:10F9B000A41702204CF30108280100209C17022004
:10F9C000381402082DE9F347074604209A460E46EC
:10F9D0009146FEF741F8134B1C68E56C246D2F44EB
:10F9E000264480464D4454446846ADF80070ADF856
:10F9F0000450ADF80260ADF80640FBF77DFB28B976
:10FA00004046FEF729F802B0BDE8F0873846314697
:10FA10002A462346FEF7A2F8FBF7ACFA0028F5D1F8
:10FA2000EEE700BF2401002010B500200146FFF7DB
:10FA30004BFA044843F6FF7201461346BDE81040F6
:10FA4000FFF7C0BF01C0FFFF80B483B000AF786094
:10FA5000054B1A687B685A60034B7A681A600C374A
:10FA6000BD465DF8047B7047B4D8012008B5084B4B
:10FA70001A6862B901221A60F0F71AFEF0F742FE26
:10FA80000448054B0360BDE80840FFF7DDBF08BD33
:10FA900030D9012028D9012019F9000890B583B088
:10FAA00000AF204B1F4A126822F001021A601E4B61
:10FAB00001221A601D4B1E4A1A601C4B1A681D4B0E
:10FAC0009A4200D0FEE7FFF7D1FF1B4B2E221A709F
:10FAD00004F0EAFB1948FFF735FFFEF763FA786098
:10FAE000FDF744FF0346002B04D0FDF745FF034616
:10FAF000002B09D1FDF726FF0446FDF726FF03463C
:10FB000020461946FDF728FF0020002103F070FC75
:10FB1000FBF73EFD0A4B01221A707B6818460C3732
:10FB2000BD4690BD002000E0083002400030024099
:10FB3000C2A507F4CDB5E8B576170220B8D80120E4
:10FB40009417022038B103888B4202D843888B4235
:10FB500001D28068F6E770472DE9F04F384C2368F2
:10FB6000B3F92A90DB69054689B0D8692946FFF7C1
:10FB7000E9FF002861D0B0F800804768C8EB0508AD
:10FB800007EBC806484696F802B0FDF765FF256802
:10FB900017F83820D5F81CE0B5F924109EF81AC0E3
:10FBA0009EF8183006938246B5F92200CDF800C0C1
:10FBB0009EF81BE0CDF804E04FF0010ECDF80CB03C
:10FBC000CDF808E073680493AD6B069B0595FEF7CE
:10FBD000CDF82368DA6992F819B0117E8B4520D9E7
:10FBE000B9F1020FD57E1CD0079103F04DFC814680
:10FBF00003F043FCFFF78AF8246817F83870E269CD
:10FC0000B4F92430B4F92200D27E079907FB02022E
:10FC100001FB05310BFB0533FDF7A0FF4846FFF75D
:10FC200075F85046FDF718FF054B1B68DA69598CCB
:10FC3000907E727800FB02125A8409B0BDE8F08F02
:10FC4000240100200D4B70B51B68DD6906460C468B
:10FC5000E8693146FFF776FF70B103884268F61A0B
:10FC600002EBC6035878AB7E10FB03F024B112F808
:10FC7000362012FB03F3236070BD00BF2401002077
:10FC800001230B80704708B5C069FFF75BFF0030A8
:10FC900018BF012008BD0000524B2DE9F04F1B6832
:10FCA000D9695F8CCC699D8CA28990428BB008D3B6
:10FCB000E689864205D3D4F80090821A4FF0FF3BC4
:10FCC00015E0A268D4F80490002A00F0818016881C
:10FCD000B0427DD3B2F802C0844579D35268801B0C
:10FCE00080B202EB800632F92020B6F902B0501C37
:10FCF0006ED091F81880A17CB3F82AA0267C0692D9
:10FD000018FB01F107910FFA8AF108460891FDF7F7
:10FD1000A3FE344909900B68069AD969887E009041
:10FD2000C97E019101210291A17C0391079901FBF8
:10FD3000029204929B6B05933FB22DB2384629463E
:10FD400032464346FEF712F8BBF1FF3F1BD04AF0A4
:10FD5000020000B2FDF780FE224A1368DA69917E44
:10FD60000091D27E0192012102910799A27C039217
:10FD700001FB0B9204929B6B059338462946324651
:10FD80004346FDF7F3FFDFF85C80D8F80030DB690D
:10FD90005A7E1B7E9A4217D9089A022A14D08AF0FA
:10FDA000040000B2FDF758FED8F80030DB6993F884
:10FDB00018E0D97E9A7E5B7E38460EFB015106FB29
:10FDC00002722B44FDF7CAFE099BD8B2FDF744FE30
:10FDD000044B617C1B685A8C0A445A840BB0BDE802
:10FDE000F08F00BF24010020044B1B68DB69DB6936
:10FDF00009B11A7C0A60587C704700BF24010020BA
:10FE000002230B807047C3699A898A4202D8DA8933
:10FE10008A420FD2986880B1038899420CD34288F5
:10FE20008A4209D3C91A426832F82100C043C0F39C
:10FE3000C0307047012070470020704770470000B5
:10FE400037B5154602AB1A4A43F8081D01901268EF
:10FE5000184C6946904723680190586958B90120A9
:10FE6000FEF72CFA2368DB695B69BBB19B680198DC
:10FE70000099984717E02946FEF790FF0028EED139
:10FE800014E001A803F08EFA2368DB691B680546BD
:10FE90009847094B1B680BB128469847009B013BCC
:10FEA000002B0093EDDA0020FEF708FA03B030BD16
:10FEB0002C010020240100209017022037B50D46A8
:10FEC0000190044698B10B4B1B68DB695B690BB171
:10FED0005B680BB9002408E0984709E001A803F02B
:10FEE00061FA20B10A2802D00134AC42F6DB204688
:10FEF00003B030BD2401002013B502A9002441F84D
:10FF0000044D00F0B7F8019B8342CCBFC0EB030067
:10FF1000204602B010BD000037B5154A019002AB73
:10FF2000126843F8081D694690470190F0B1114BE3
:10FF30001B68DB695B690BB11B6813B900252C4694
:10FF400002E00099984711E0009B013B002B0093D1
:10FF500007DB01A803F026FA054600F081F8044407
:10FF6000F2E72846FFF7C8FF2044FFE703B030BDA3
:10FF70002C01002024010020274B1B6873B5054687
:10FF80000C4663B10020FBF7B7F8002841D02846A3
:10FF900021466A46FFF754FFFAF7ECFFF5E71068D1
:10FFA00051681E4E6B4603C33368BDF80010B3F8AA
:10FFB0004C20B3F850301144ADF80010BDF80210D9
:10FFC0001944ADF80210BDF804100A44ADF804203D
:10FFD000BDF8062068461344ADF80630FBF78CF8F0
:10FFE000336840B9598CDA6C8A1A5A84998C1A6D24
:10FFF0008A1A9A840DE0BDF800205A84BDF80220C8
:020000040801F1
:100000009A84284621466A46FFF71AFFFAF7B2FF9C
:10001000E6E702B070BD00BF78170220240100207F
:100020000A4B1B689A8D02F00C02082A07D00C2A92
:1000300005D0042A07D1DB69187E01387047DB69D7
:10004000187E400870470020704700BF2401002040
:10005000024B1B68DB69587E704700BF24010020FB
:1000600008B5034B1B68DB6900215B68984708BD36
:100070002401002008B5034B1B68DB695B689847C7
:1000800008BD00BF24010020074B5A68596A01329D
:1000900010B55A605A6B02EBC0046160002102F88F
:1000A0003010586210BD00BFB417022038B50B4D98
:1000B000002405F140002146802285F82840FEF703
:1000C00051F828462146C022FEF74CF82146044844
:1000D0000C22BDE83840FEF745B800BFB417022037
:1000E00034D9012010B542680F230D4901EBC30438
:1000F000246CA24203D213F1FF33F6D210BD0F2BB2
:100100000CD80C68A21A0A608268C06802B15060FC
:1001100008B1026010BD01EBC3035A6410BD00BFFB
:10012000B4170220F8B5264EF3685A1EB36B054685
:100130001344081898420C4605D84B591BB943681C
:100140001D44FFF7CFFFB36B9C420AD954F8047CDF
:10015000E71B3B682BB97B6838461D44FFF7C2FF9D
:100160003C460F2306EBC302126C954203D213F1F7
:10017000FF33F7D222E00F2B20D8083306EBC3025F
:1001800061195268A260002084E82100246141F8CE
:10019000045C04F1080102B1516006EBC303E060A6
:1001A0005960336896F82910054A2B44336029B901
:1001B000D168CB1A9168994238BF93602846F8BD40
:1001C000B4170220254B2DE9F74FDA689C6B013AF2
:1001D000824602EB04099B4694E82800002B33D1A9
:1001E00004EB0508C8452FD254F805C0D8F80460C0
:1001F000BCF1000F28D0DBF83430184F13F83C3036
:10020000012B21D1FB6A20468DE80810FFF76AFF19
:10021000D8F800107A6B02EBC102204654604146C8
:10022000324608F0CBF99DE808109C4502D17B6B63
:100230005B1B7B632846A119FFF774FFBAF1000F1F
:1002400001D0824505D935462C444C45C4D3012004
:1002500000E0002003B0BDE8F08F00BFB41702201B
:1002600028B1034AD36B036003B15860D063704771
:10027000B417022028B1034B5B6B03EBC00040684E
:1002800008307047B4170220054BD9690131D96194
:100290005B6B13F83010013103F83010FFF7EABF41
:1002A000B417022030B50268094B52F8081C5A6B8B
:1002B00012F83140012C03D9DD690DB1013DDD613A
:1002C000013C02F8314000230360184630BD00BFF6
:1002D000B4170220024B21F00301186059607047E7
:1002E00034D9012030B1044B5B6B03EBC000436891
:1002F00058680C38704700BFB417022010B5044688
:1003000080B1094B5B6B03EBC00213F83030012B5B
:1003100008D151684868FFF705FF2046BDE8104046
:10032000FFF7B2BE10BD00BFB41702202DE9F041A7
:10033000224CE36A3BB9224B9D685B680835B3FBEE
:10034000F5F5023503E023691D1D05EBD305E80033
:1003500000F078F9804660B3616B2269E76A01EBCF
:10036000C003D2005E680836304608F019F92269E9
:10037000666306EBC201C4F82C8004311346681E84
:10038000834201F1080103D2013341F8083CF6E74A
:1003900006EBC30300265E60636862629B1A2B440F
:1003A0006360256138463FB1FFF7A8FF3046BDE8DE
:1003B000F0810120BDE8F081BDE8F081B417022092
:1003C00034D90120F8B5584E96F82810002940F08D
:1003D000AA80564D6A68012386F82830B2F5205F5E
:1003E00028BF4FF420522B6894080020A0420CD064
:1003F00047184FF0FF0EB7FBFEFECEEB0E2ECEEBF6
:10040000070743F820700130F0E70020A04216D023
:1004100047184FF0FF0EB7FBFEFECEEB0E2ECEEBD5
:10042000070E53F82070774507D0AA683F4B002A83
:1004300055D15A6892089A6051E00130E6E70131DF
:100440000229D2D1540800210020A0420CD0471824
:100450004FF0FF0EB7FBFEFECEEB0E2ECEEB0707E6
:1004600023F810700130F0E70020A0420FD04718A9
:100470004FF0FF0EB7FBFEFECEEB0E2ECEEB0707C6
:1004800033F810C0BFB2BC45CFD10130EDE7013128
:100490000229D9D100210020904207D04418FF271B
:1004A000B4FBF7F73C441C540130F5E700209042C0
:1004B0000BD04418FF27B4FBF7F73C441F5C04F053
:1004C000FF04A742B1D10130F1E701310229E2D1A5
:1004D00000219142A9D0002058540131F9E7144875
:1004E000144B0360FFF7B0FA5A2333620023102144
:1004F00006EBC30299400133102B0B4C1164F6D16B
:1005000068682968A16302232361A0F114030B44E6
:1005100001256363E0605D6065626560FFF702FE70
:10052000FFF704FF2563F8BDB417022034D901207A
:1005300040D90120AD0001082DE9F0410546264EC5
:100540000335FFF73FFF25F00305336CF26B0435ED
:100550009D4238BF1D4614462CB154F8043CAB42B2
:100560002CD02468F8E7F368B26B02EB030858F864
:10057000047CC7EB08073B6833B12046FFF722FE37
:1005800058F8047CC7EB08073B6813BB7B68AB4299
:100590001FDB38461C1DFFF7A5FDF36878685B1B61
:1005A000F3607369641B2B44401B3C44736102D0AD
:1005B0003946FFF7B7FD44F8045C0AE023680BB145
:1005C00061685960616801B10B60A24201D1236882
:1005D000F3632046BDE8F081B417022008B5FFF7A9
:1005E000F1FE00220B4B1344D3F8BC3013B19B68CF
:1005F00000200BE0083A12F1800FF3D1F8E75A68B7
:100600009B68904238BF104613B19B68002BF6D10F
:100610000C3808BDB417022008B5FFF7DFFFB0F5AE
:10062000800F4FF06403064A04D990FBF3F0136A7D
:10063000584308BD126A5043B0FBF3F008BD00BF39
:10064000B41702202DE9F843384D0446FFF7BAFEEF
:100650002F6C2B68BC4224BFE71C27F003070C3724
:100660009F42324C3ED8236B62689A420FD96B6826
:100670006E6A013B6B606B6B4FEAC60903EB0902C4
:1006800052686A62012203F8362056B92AE0013B1B
:100690002363FFF74BFE236B013323630028E6D06F
:1006A00020E00F2305EBC302126C97420CD213F12A
:1006B000FF33F7D208E094682CB16268974214D9EE
:1006C000A268002AF7D101330F2B03D805EBC30230
:1006D000526CF6E73846FFF775FD0028E1D030464A
:1006E000FFF7D2FC0020BDE8F883D4F804802B6C1F
:1006F000C7EB08020C3320469A4238BF4746FFF743
:10070000F1FC6B6B4B44E1195C60B8454FF00003A2
:1007100084E8C000A360246141F8047C03DDC7EBDA
:100720000800FFF7FFFC3046BDE8F883B41702204D
:1007300008B1FFF787BF704710B504460068FFF7A0
:10074000DDFD0023236010BD10B580EAE071A1EB50
:10075000E0710022531C0A2B06D0064C54F82340AB
:10076000A14201D31A46F5E70028B8BF931C1846EA
:1007700010BD00BF54F30108002807DD0B685A1CA8
:100780000A602B221A700B6800221A707047000052
:10079000B0F1004FF0B51C6809D1601C1860013938
:1007A0002D202070C9B26FF0004001260CE0002817
:1007B00006DA651C1D602D2525704042012400E0ED
:1007C0000024091BC9B200260AB30139C9B21EE0D0
:1007D0004D1E9142EDB205D11C68671C1F60114F80
:1007E0003F782770104C54F8257090FBF7F4E4B272
:1007F0000A2C0ED807FB14007DB10A2C18BF29461D
:100800001D6808BF01246F1C30341F602C70002944
:10081000DED11B6800221A70F0BD002EEDD001342D
:10082000E4B2EAE77617022054F3010873B50546EF
:10083000FFF77EFF064658B1FFF726FD02AC002108
:1008400044F8040D2A46FDF78DFC2046FFF72AFDEB
:10085000304602B070BD00002DE9F7431E4CD4F8BD
:1008600000E0DEF84C40DEF85060051914449EF8B4
:100870001820013A92B28F191E44AB1AADF800301D
:100880001319ADF804306846BB1A3244ADF8023093
:10089000ADF80620FAF730FCD0B12846394622469A
:1008A000FDF710F907F1010928463146224606F105
:1008B000FF38FDF707F9284649464246FDF728F973
:1008C000204649464246FDF723F9FAF753FBE3E792
:1008D00003B0BDE8F08300BF24010020C0F3C421B1
:1008E000064B00F01F02C0F345109A5C5B5C03EB03
:1008F0000243034A105C03EB002070471812020801
:10090000D8110208C0F30741064BC2B2C0F307205A
:100910009A5C5B5C03EBC223034A105C03EB401060
:10092000704700BF38130208381202084FF6FF70F4
:1009300070470000F8B50F4F3F6806460D46144655
:100940009C460FB1B847F8BD56F8042B0A49D3B2FC
:10095000013CC85CC2F30743C2F30722CB5C0749E2
:100960008A5C03EBC02303EB42132B806544EBD17D
:10097000F8BD00BF4CD90120381302083812020814
:10098000F8B5134E3668844614461D460EB1B0477E
:10099000F8BD501E02F18042013A03FB00C001EB9A
:1009A000820102880B4B02F01F06D70A9E5DDB5DB9
:1009B000C2F3451203EB0643074EB25C013C03EB66
:1009C000022341F80439C5EB0000EAD1F8BD00BFAD
:1009D00048D9012018120208D81102087047704740
:1009E00070474FF0FF30704710B550F8044B0C6063
:1009F000013A1944F9D110BD10B5046841F8044B0F
:100A0000013A1844F9D110BD10B59CB004466846AF
:100A1000FEF7B0F9094B1868FDF76EFBB4F900005A
:100A2000B4F90210B4F90420B4F90630FFF714FF4A
:100A30006846FEF7A9F91CB010BD00BF50D90120CF
:100A400010B59CB004466846FEF794F9094B186847
:100A5000FDF752FBB4F90000B4F90210B4F9042018
:100A6000B4F90630FFF7F8FE6846FEF78DF91CB0C2
:100A700010BD00BF50D9012007B56846F9F70EFC3C
:100A80006846FFF7C1FF03B05DF804FB07B5684691
:100A9000F9F704FC6846FFF7D3FF03B05DF804FBE9
:100AA00013B5044640B1FFF7EFFB02AB046D43F80A
:100AB000040D1846FFF7F6FB204602B010BD1FB527
:100AC00001F00803002B40F28A3440F28A5208BF3A
:100AD00022460CBFFF23FE238DE805000020029173
:100AE000039302460346014600F0AEF80621044691
:100AF000F9F713FA204604B010BD07B5FFF7C4FBA1
:100B00000190406E00F0D4FB02A8002250F8043D92
:100B10005A66DA65FFF7C6FB03B05DF804FB438E47
:100B20001B0710B512D5B0F90420B0F900300888C1
:100B30004C880C80D31A8A88CC888C8001339BB275
:100B4000C043D24318441344C8804B8010BD10B535
:100B5000044600F0B6FCFAF798F82046F9F7B7FA21
:100B60002521BDE81040F9F75BB90000F0B589B068
:100B70000E9E109C119DFAB9F3B9304606A9F9F7FB
:100B800023FB14F0080F2C4BBDF91C70BDF91EE0BF
:100B900009D0BDF91A10B3F90020781CC1EB0E037F
:100BA000801A013308E0BDF91800B3F900300EF1E6
:100BB00001013A1AC91A013200960F9E01961F4E82
:100BC0000296129E3C360396FAF7A0F806460028D5
:100BD0002FD0FFF759FB04F00802E30648BF42F0AC
:100BE0001002A5F1FE0348BF92B2012B88BF42F06C
:100BF000100229460590F8F74DF8114B08AF0FCBBE
:100C000057F80C4D04F1340585E80F006423E364C4
:100C10000C4D0A236365002323652B686364384603
:100C2000FFF740FB2B6830465B6898473046FFF77C
:100C30008EFF304609B0F0BD44010020EB0C0108E6
:100C4000300100204001002010B586B0089C0094BF
:100C5000099C01940A9C02940B9C03940024049424
:100C6000FFF784FF06B010BD37B50C46054600B34C
:100C7000FFF70AFB002C0190C16C426D05DB8A1A5C
:100C800022EAE272944202DC00E000242246016D76
:100C900091420BD002652846F9F7F7FF01A8FFF74C
:100CA00001FB28460521F9F738F902E001A8FFF712
:100CB000F9FA03B030BD73B50D46064660B1FFF7D3
:100CC000E3FA024602A8146D40F8042DFFF7EAFA91
:100CD00030466119FFF7C8FF02B070BD4FF0FF3119
:100CE000FFF7E9BF0121FFF7E6BF2DE9F04F4468A8
:100CF00080468FB020464146F7F7D4FF002800F029
:100D0000C081D8F80030232B00F082810BDC0E2B41
:100D100000F02A810F2B12D00B2B40F0AF81204620
:100D2000FFF715FFAAE140F21312934200F07F8112
:100D3000B3F5107F12D0242B40F0A08143E1204670
:100D4000FFF7A2FA0590002800F09B81436C05A8EC
:100D50001D68FFF7A7FA2046A84792E1D8F80C7063
:100D6000002F00F08B813B7A2046002B00F0D680CC
:100D7000FFF78AFA05A9836C0390066D2046984711
:100D8000039BB3F832A05D6DDA6C1AF0080FC5EB67
:100D9000020903D097E806003A6079609A6D3F68CF
:100DA000032A14D12046FFF7A8FE0D9B0C990220C0
:100DB00093FBF0F3FF1A069BFB1A581E00FB09F089
:100DC00002F049F9039B0646186603A87EE00698E0
:100DD00087420BDC022A39D05B6E13B12046FFF745
:100DE0008CFE039B0222013E9A652FE007998F42F9
:100DF00002DA761B6D422FE008998F4212DC0C99C3
:100E000000290BDD0D9B022293FBF2F3FF1A3F1A20
:100E1000013F07FB09F002F01EF90646039B03227F
:100E20009A6516E009998F4201DA2E4414E00A9976
:100E30008F420EDC012A0ED05B6E13B12046FFF705
:100E40005CFE039B012501369D6505E04FF0FF35F3
:100E500002E0002500E01546DDF80CB00C99DBF847
:100E60005C30DDF834E0069A71B102209EFBF0F0B0
:100E7000381A801A013800FB09F0019302F0EBF8F0
:100E8000019BCBF8600009E0DBF85820012A04BF81
:100E9000DBF84C1001F1FF31CBF8601003A801938F
:100EA000FFF700FA019BA5B1BBB94FF4C87240F23D
:100EB000D241204600F034FA07462046FFF7E4F915
:100EC00002460EA840F8282D5766D565FFF7EAF9C7
:100ED00003E013B12046FFF710FE2046012100F089
:100EE000A3FA20463146FFF7BFFE1AF4807F40F098
:100EF000C5802046FFF7C8F90EAB856A43F8280D78
:100F00001846FFF7CFF94FF480712046F7F796FEA9
:100F1000A90740F1B3802046012174E0FFF7B4F93E
:100F2000458E039003A8FFF7BDF9EA0540F1A680BE
:100F300020464FF48071F7F797FE2046FFF7A4F99B
:100F4000C36D059013B12046FFF7D7FD0EA8002210
:100F500050F8243D9D6A9A65FFF7A4F9AB0740F16C
:100F60008D80204602214EE02046FFF78DF90EAB22
:100F7000456D43F8240D1846FFF794F9D8F80C2076
:100F800013685268002A79DD103B122B76D8DFE80F
:100F900003F016161212757575757575757575757C
:100FA0007575750A0D002046294601E02046694204
:100FB000FFF781FE62E02046FFF794FE5EE02046E8
:100FC000FFF78CFE5AE02046D8F80C60FFF75CF97A
:100FD0000EAD034645F8240DDA6C3068B1689042D6
:100FE000726805D15E6D8E4202D11E6D96420DD0A3
:100FF000D86459651A652046F9F747FE2846FFF779
:1010000051F920460521F8F788FF37E0284633E0FC
:101010002046FFF739F9059000282FD0D8F80C307A
:10102000C26C1A60426D9A60026D5A6023E02046DD
:10103000FFF72AF9C16D059011B12046FFF73BFE7D
:10104000059BDA6D196D002A1A6E05DD9142B4BF59
:101050000021012106DD04E09142CCBF00210121E5
:1010600000DA1A6519B12046FFF747FD03E0586E14
:10107000322100F085F905A8FFF714F94046FAF788
:101080002FFA0FB0BDE8F08F0388994213B50C46D4
:101090000ED2406850B1FFF7F7F802AB50F8244089
:1010A00043F8040D1846FFF7FDF802E0044600E09F
:1010B0000024204602B010BD13B5044640B1FFF72E
:1010C000E3F802AB048843F8040D1846FFF7EAF88A
:1010D000204602B010BD2DE9F743054600283DD05B
:1010E0004AB10846114602F04FFBD0F10104074611
:1010F00038BF002401E0144617462846FFF7C4F81D
:1011000002AEB0F8008046F8080DD0F804906846AA
:10111000FFF7C8F824BB08F101014846890002F036
:1011200081F9814618B93846FFF7E8F818E0FFF76B
:10113000ABF802AB43F8040D40F828701846FFF7EF
:10114000B1F82846FFF7A0F8038800900133C0F8F3
:10115000049003806846FFF7A5F802E0044600E02B
:101160000124204603B0BDE8F08337B5054618B327
:10117000FFF78AF800904068C0B1FFF785F80024B7
:101180000190009B1B889C4206DA019800EB8400CA
:10119000FFF7D2FA0134F4E701A8FFF783F80098CB
:1011A0000430FFF7C9FA009B00221A806846FFF757
:1011B00079F82846FFF7A2F803B030BD73B50E46A4
:1011C000054658B1FFF760F802AC314644F8040D0B
:1011D000FFF75AFF05462046FFF764F8284602B09D
:1011E00070BD0820FFF722BB30B585B00446102241
:1011F0000D466846002107F0FBF92046FFF73AF854
:1012000003691BB1019400956846984705B030BD4D
:1012100070B50D4C2368132B06460D4612DCFFF704
:1012200029F803696E6043B12268284601322260C2
:1012300098472368013B236070BD2846BDE8704095
:10124000FAF74EB970BD00BF54D9012038B5054634
:1012500000F00FF8044654B1AC4207D02046FFF727
:1012600009F8036AAB4202D01C46F4E7002420468A
:1012700038BD08B5F8F72BFF18B1FEF7FBFFC069C2
:1012800008BD08BD1FB5044600216846102207F0BE
:10129000AFF9606850B1FEF7EDFF40F213134068FC
:1012A0000093694663680393F9F798FC04B010BD96
:1012B00037B5054668B1FEF7E7FF02AC44F8040D08
:1012C0000068FDF767FC2046FEF7ECFF2846FFF7B5
:1012D00015F803B030BD73B5054601A8FDF7D8FB7E
:1012E0000446DCB120460121FDF7AFFC019B83B130
:1012F00078B11846FEF7BEFF4368AB4209D12046DD
:1013000001A9019EFDF7DCFB04463046FFF7D0FF44
:10131000E7E7204601A9FDF7D3FBE1E702B070BD86
:101320002DE9F34180460C200F461646FFF77EFA62
:101330000446F0B1FDF79EFC2246811901230F48B7
:10134000FDF7DAFB0546204685B1FEF79DFF034613
:1013500002A8C3F8048040F8043D9F601D60FEF7BA
:10136000A1FF28463146FDF749FC02E0FEF7C6FF23
:101370002C46204602B0BDE8F08100BF851201086E
:1013800013B50C4680B1FEF77FFF01901CB10068D9
:101390002146FDF733FC02AC54F8043D1868FDF714
:1013A0003BFC2046FEF77EFF02B010BD2DE9E74171
:1013B0000E4690460746D0B1FEF766FF034602A8E8
:1013C000B3F90410B3F90020B3F9065040F8043D16
:1013D000B3F902308A1AED1AD243ED43164445445C
:1013E000FEF760FF384631462A46F8F71BFD03B08A
:1013F000BDE8E08130B50A4D0A4C2B6854F8230053
:1014000085B050B104A9182341F8103D6946FFF793
:10141000FFFE2B68002244F8232005B030BD00BF3A
:101420004817022064170220F8B5094B094A044600
:1014300018680F4652F82010A14215461E4601D0EA
:10144000FFF7D8FF336845F82340034B1F70F8BD02
:1014500048170220641702204C17022038B50546B1
:101460000C4641B1F8F733FE28B1A5602146BDE82E
:101470003840FFF7CDBE38BD7FB50A4A0346106835
:10148000094A52F8200048B100930E2301910293BB
:1014900002A900AB0593FFF7BBFE012007B05DF882
:1014A00004FB00BF481702203817022010B50C4675
:1014B00030B129B1FEF7DEFE034603CB2060616048
:1014C00010BD38B50546F8F78BFEFF28044603D05B
:1014D000FE2808BFFF2400E0FE242846F8F7F7FDA9
:1014E0002146BDE83840F8F7B7BE02F00ABD00005B
:1014F000024B1A6802601860704700BF5C17022038
:101500002DE9F043044687B0002839D0FEF7BCFE31
:101510000346019003C804AD85E8030001A81E6AD4
:10152000D3F82890FEF7BEFE2046FFF78FFE074651
:1015300030B32046F8F7CBFD19F0020F804604D0F7
:10154000284641463246F9F731FB2046FEF79CFE1D
:1015500001904046FEF798FE03903846FEF794FE51
:10156000039B019AD96906620290116201A8DC61AD
:10157000FEF798FE03A8FEF795FE02A8FEF792FE7E
:1015800007B0BDE8F0832DE9F84FDDF828B0DDF8AD
:101590002CA005460E4690461F461446894635F84F
:1015A000020BD847D047013C49F8040BF7D11F2F55
:1015B00006D8304641463A46BDE8F84F01F058BDDE
:1015C000BDE8F88F2DE9F84FDDF828B0DDF82CA044
:1015D00005460E4690461F468946044614F8010B00
:1015E000D847D0472B1B434449F8040B002BF5D1B7
:1015F0001F2F06D8304641463A46BDE8F84F01F065
:1016000037BDBDE8F88F00002DE9F04F9DB00646CC
:101610000F910D92002800F08683FEF735FE1CAB7B
:10162000446943F81C0D1846FEF73CFE3046FAF7B5
:1016300093FF0828014602DD002C00F0C38101223F
:101640004FF0000830461B920B92CDF86880FEF7F1
:101650001BFE0368DFF80CA61B69B0F90A105B6873
:101660000E930DF1700BDAF800304BF8140D04698D
:101670004569D0F80C90B0F90870587C1291FCF7CD
:1016800033F9DAF800301090587CFCF74BF9034638
:1016900058460993FEF706FE082C51460B9A099B03
:1016A00004D9102C8CBF0422022205E0012C03D1A6
:1016B00011940DF1680800E011920E98984200F024
:1016C000E2800B68587CFCF735F91390B800FFF7FF
:1016D0002FF80C90002800F026833046FAF7D8F84F
:1016E0000646002D00F0BE802846FEF7CDFDDDF851
:1016F00034B018904FF0000A129A924580F2AE80F2
:10170000189800231993836819A95B695246984772
:10171000B84205462FD10C98FEF7B6FD082C0146BD
:10172000169009D90E9A139B0092019330463A46BF
:10173000109BFFF728FF08E00E98139A0090019283
:1017400030463A46109BFFF73DFF01231098029068
:101750001CAD002200930193039255F8182D0492BA
:101760000F98CDF8148059463A46FCF7FFFA284600
:10177000FEF798FD60E0012C5CD1002D5CD019983B
:101780000F99CDF80C90082290FBF2F2324401231D
:10179000049200F00702009308440193029306921A
:1017A00059462A46CDF81480FCF704FA199B18987C
:1017B0001D44836819955B6919A9524698470546E7
:1017C000DBE70C98FEF760FD082C0146169019988F
:1017D00038D90E9A0092119A139B019300FB026074
:1017E000109B2A46FFF7CFFE01230DF1700C1098D5
:1017F00000930022019302900F99039219985CF8CC
:10180000182D049208442A465946CDF81480CDF884
:101810002CC0FCF7ABFADDF82CC06046FEF742FDA9
:10182000199B18981D44836819955B6919A952463C
:1018300098470546002DC4D14E440AF1010A0BF128
:10184000010B59E70E9B0093119B139A019200FB29
:1018500003602A46109BFFF7B5FEC5E718A8FEF700
:1018600021FD0EE001230093019304900294CDF832
:101870000C90CDF814800F980D99129B3A46FCF706
:1018800075FA0C984DE23046FAF702F80646002D3C
:1018900000F08A802846FEF7F7FC00251890129B7E
:1018A0009D427DDA189800231993836819A95B6912
:1018B0002A469847B842824624D1AA461898836897
:1018C0000AF1010B5B6919A95A469847B84201D140
:1018D000DA46F3E7C5EB0A0B0D99049601230BF1E9
:1018E000010B0093019329440294CDF80C90CDF89C
:1018F00014800F983A465B46FCF738FA09FB0B66F2
:1019000055464BE0012C27D1BAF1000F22D019988F
:101910000F99CDF80C90082290FBF2F23244049219
:1019200000F0070208440D990692012352460093E5
:10193000019302932944CDF81480FCF73BF9199BDD
:10194000189853441993836819A95B692A469847E4
:101950008246D9E74E4421E0BAF1000FFAD0199837
:101960001199029400FB016204920D990F9ACDF82F
:101970000C90012310440093524601932944CDF862
:101980001480FCF7F3F9199B189853441993836852
:1019900019A95B692A4698478246DDE701357EE74B
:1019A00018A8FEF77FFCBEE1012300930193049089
:1019B0000294CDF80C90CDF814800F980D99129BDD
:1019C0003A4641E030460A91FEF75EFC82461CA88A
:1019D000BAF80A2040F810ADDAF800401092D4F8B6
:1019E0001090BAF808709E4C13B2DAF80C200B92E3
:1019F0000993FEF757FCD9F804000E909948006847
:101A0000407C54F820402569D5F80080FBF76CFF36
:101A100008280FFA87FB0A990B9A099B04D910280A
:101A20008CBF0424022400E00124A9450FD1012029
:101A300003920AF1180200900190029104920F980B
:101A40000D99002205925A46FCF790F96BE1202986
:101A500040F08E800BFB04F0FEF76AFE0E9000282B
:101A600000F06181FEF710FC1A903046FEF70CFC86
:101A700018902B6900F1180A4FEA8B064FEAC40947
:101A8000002B2FD0DDF83480022C03D0042C01D0A1
:101A9000012C06D150462F691A995A462346B84759
:101AA000B244012300221A990093019303920491F6
:101AB000059241465A46CDF808900F98FCF756F922
:101AC00010990D9A08F1010702FA81F3BB4207D180
:101AD00018A8FEF7E7FB1AA8FEF7E4FB0E9820E132
:101AE000B846D1E70D9D022C1A9F0ED0042C18D0B9
:101AF000012C25D100235AF823000993C047099BE4
:101B0000F85401339B45F6D119E000235AF823001D
:101B10000993C047099B27F8130001339B45F5D172
:101B20000DE05A4600235AF803000B920993C04770
:101B30000B9A099B013AF85003F10403F3D1B24424
:101B4000012300221A9900930193039204910592B4
:101B50000F98CDF8089029465A46FCF707F91098D7
:101B60000D996F1C01FA80F3BB42B1D03D46BAE734
:101B7000102940F0D8800FFA87FA0AFB04F0FEF72C
:101B8000D7FD1290002800F0CE80FEF77DFB1A9062
:101B90003046FEF779FB18902B6900F1180613B157
:101BA000D9F814302BB9E2003FB211927F000D9D9D
:101BB00088E0B0F908008000FEF7BAFD119018B176
:101BC000FEF762FB199001E0119B1993199B002B02
:101BD00000F0A0803FB27F000E97E70013970D9FA3
:101BE0000C97022CDDF8688004D0042C07D0012C5F
:101BF00014D104E0304619995246234603E019995E
